:020000040800F2
:1080000000A0002069560108910D0108930D010898
:10801000950D0108970D0108990D01080000000059
:108020000000000000000000000000009B0D01089F
:108030009D0D0108000000009F0D0108F58100085A
:10804000AD560108AD560108AD560108AD56010800
:10805000AD560108AD560108AD560108018800086B
:10806000AD560108AD560108AD560108AD560108E0
:10807000AD560108AD560108AD560108AD560108D0
:10808000AD560108AD560108AD560108E5070108D7
:108090007D06010831070108AD560108AD560108FB
:1080A000AD560108AD560108AD560108AD560108A0
:1080B000AD5601084FF30008AD560108AD56010852
:1080C000AD560108AD560108AD56010861EF000834
:1080D000AD560108AD560108AD560108AD56010870
:1080E000AD560108AD560108AD560108AD56010860
:1080F000AD560108AD560108AD560108AD56010850
:10810000000000000000000000000000AD56010863
:10811000AD560108AD560108AD560108AD5601082F
:10812000AD560108AD560108AD560108AD5601081F
:10813000AD560108AD560108000000000000000027
:10814000AD560108AD560108AD560108000000000B
:10815000000000000000000000000000000000001F
:108160000000000000000000AD560108AD560108F7
:10817000AD560108000000000000000000000000F3
:0881800000000000AD560108EB
:1081880010B5054C237833B9044B13B10448AFF349
:1081980000800123237010BDA4000020000000000F
:1081A800888100080C4B43B10C480D4910B5AFF35A
:1081B80000800C48036823B910BD0A48036833B926
:1081C8007047094B002BF7D0BDE810401847064B05
:1081D800002BF5D0184700BF000000008881000878
:1081E800A8000020A400002000000000684620F03D
:1081F80007018D4619B5114B1A781C46DAB15B6830
:108208000F4A013363601368013313600D4B1A681A
:108218005AB11A68013A1A601B6833B90A4B1B68CD
:108228001BB10A4B187800F0C9F900232370BDE888
:1082380019408546704701221A70F8E7C0000020EF
:10824800E00D0020200C0020FC0B00206E0D00200B
:108258000A4B10B541F29312094C5A60F02284F887
:10826800232000229A6007221A606FF004000AF0A7
:108278008DFC302384F8233010BD00BF10E000E0EF
:1082880000ED00E0014B5868704700BFC0000020B7
:1082980038B5002205460C460220CF2100F074FCB8
:1082A80029460022022000F06FFC2146012202200C
:1082B800BDE8384000F068BC08B501200BF0ACFB05
:1082C800000A05280AD101200BF0A6FBC0B26228DB
:1082D80004D10220BDE808400BF09EBB002008BD79
:1082E8000020704708B501200BF096FB000A05280E
:1082F80001D0012008BD01200BF08EFBC0B262281E
:10830800F7D103200BF088FB000A431E584258415E
:1083180008BD002070472DE9F043012187B04FF4D4
:10832800003000240AF096FE032640F6420302A914
:108338004FF0904001274FF0904502938DF80D6063
:108348008DF80C408DF80E408DF80F400AF09EF91C
:1083580048F2BD0302A94FF090404FF480280293E1
:108368008DF80C708DF80D608DF80E408DF80F406B
:108378000AF08CF948F21803C5F81880AB614FF47D
:108388008073AF6102A90293284602238DF80C304E
:108398008DF80D608DF80E408DF80F400AF076F9D3
:1083A80006200AF085FC4046DFF8B08139460AF01D
:1083B80051FE40464BF2072302A902938DF80D6047
:1083C8008DF80C408DF80E408DF80F400AF05EF9DC
:1083D80040464FF4506302A902938DF80C708DF853
:1083E8000D608DF80E408DF80F400AF04FF94FF4EC
:1083F8000063C8F818304FF0A063C8F81830394641
:1084080008F580684FF400200AF024FE4FF420435A
:10841800404602A902934FF480498DF80D608DF80B
:108428000C408DF80E408DF80F400AF02FF94046A9
:1084380002A98DF80C708DF80D60CDF808908DF8B4
:108448000E408DF80F400AF021F9C8F8189002A9DB
:108458004FF4005828468DF80C708DF80D60CDF853
:1084680008808DF80E408DF80F400AF00FF902A928
:1084780028468DF80D608DF80F70CDF808908DF8AE
:108488000C408DF80E404FF000570AF0FFF82E46CA
:108498000A2122464346AF614FF47A7000BF013883
:1084A800FCD1288AB361400458BF01324FF47A7076
:1084B80000BF0138FCD1288A400448BF0134013983
:1084C800E9D10A2A244B45D10A2C43D101221A703A
:1084D8004FF4C043002402930226032302A94FF05D
:1084E80090408DF80D308DF80C608DF80E408DF8A9
:1084F8000F400AF0CBF822460D214FF090400AF0C9
:108508003DF922460E214FF090400AF037F9134BFF
:108518004FF480629A61012120460BF055FD012538
:108528000C2304A88DF8153004958DF814408DF8A7
:10853800165009F0DBFC072301A88DF804308DF8EC
:1085480005608DF806408DF807500AF0DBFA07B091
:10855800BDE8F0830022BAE7180C002000040048A8
:10856800F7B5134B1B7803B31249134C4FF09042E5
:108578004FF400274FF4804E002008254FF0804626
:108588009761C1F818E00190019BA34209D9956150
:108598008E610190019BA342F2D8019B01330193A4
:1085A800F8E7019B01330193EEE703B0F0BD00BF8C
:1085B800180C0020000800483F0D030001280E4B4E
:1085C8000ED008D302280FD01A784FF090437AB112
:1085D80004229A6170471A7822F001021A70F3E7B0
:1085E8001A7822F00202F9E71A7822F00402F5E775
:1085F8004FF48022EDE700BFC800002001280E4B91
:108608000ED008D302280FD01A784FF090437AB1D1
:1086180004229A6170471A7842F001021A70F3E74F
:108628001A7842F00202F9E71A7842F00402F5E7F4
:108638004FF48022EDE700BFC800002010B50021EC
:10864800044644FA01F3DB07C8B205D5FFF7D6FFA5
:1086580001310829F5D110BDFFF7B0FFF8E718B1CF
:10866800012806D000207047044B188AC0F3403018
:108678007047034B188AC0F3003070470008004861
:1086880000040048012809D003D302280BD0002099
:108698007047074B187800F001007047044B1878B2
:1086A800C0F340007047024B1878C0F38000704751
:1086B800C8000020054B188AA3F58063C0F340303A
:1086C8001B8ADB0448BF40F00200704700080048DE
:1086D800064B1B7803F001009A0748BF40F00200E0
:1086E8005B0748BF40F00400704700BFC800002087
:1086F800704701207047034B10B1034ADA60704796
:10870800024AFBE700ED00E00400FA050100FA0563
:1087180000224FF0FF31930003F1604303F56143FA
:108728000132082AC3F88010C3F88011F3D100235E
:1087380004481946C2180133F02B82F80013F9D106
:10874800704700BF00E100E0024B1844002343706B
:10875800704700BFC8000020024B18440123437033
:10876800704700BFC8000020014B1844407870478C
:10877800C8000020014B01229A707047C8000020F1
:10878800014B00229A707047C8000020024B98786D
:10879800B0FA80F040097047C800002014490B184F
:1087A80010B5DC78012C0A4603D01ED3022C14D055
:1087B80010BD897811B95B7823B910BD0D4B4FF402
:1087C8000061996113185B781BB10A4B4FF4006183
:1087D800996102440223D37010BD8A783AB95A7855
:1087E8002AB9044A4FF0006191610122DA7010BD84
:1087F800C800002000040048684620F007018D46A4
:1088080019B5012009F01AFC012801460ED1094CBE
:10881800236843B1084B1878FFF7F0FE074B22682E
:108828001A60074B1970012009F01BFCBDE81940BC
:1088380085467047FC0B00206E0D0020200C0020A0
:108848006D0D00202DE9F04385B0814688464148EA
:108858009DF830404FF480511E4617460BF09BFAA6
:108868004FF4E0613B480BF08EFA0022B021022061
:1088780000F08AF901228321022000F085F9364BA5
:10888800002201ADA3F10C01B9F1000F5FD0505CDB
:10889800A85401320C2AF7D1B9F1000F28D19DF85C
:1088A80008109DF8092008F07F0321F07F01194383
:1088B8008DF808109DF80D1006F07F0321F07F0158
:1088C8000B438DF80D309DF80A3003F00F0343EA8F
:1088D800041322F07F0207F07F073A438DF80A302D
:1088E800E3064CBF62F07F0202F07F028DF8092098
:1088F80000270224E95DF8B20B46082684EA030241
:10890800640012F0800FE4B206F1FF3618BF84F05D
:108918001D045B0016F0FF06DBB2EFD10137FFF74D
:10892800B7FC0C2FE6D121463846FFF7B1FC0121F0
:108938007420FFF7ADFC314606480BF02CFA0548C9
:108948004FF4706105B0BDE8F0430BF01CBAD05C81
:108958009EE700BF003C0040AA570108800000F1D4
:10896800006000F55E30006870470000F0B5012136
:1089780089B04FF400400AF085FB00243823022711
:10898800032601214FF4802001938DF808708DF89B
:108998000A408DF809608DF80B400AF05BFB01A9CD
:1089A800754809F073FE06223146734809F0E6FE61
:1089B80006220421704809F0E1FE062205216E48CE
:1089C80009F0DCFE6D480BF0D1F84FF48273ADF876
:1089D8000E304FF4E063ADF810304FF4007301250A
:1089E800ADF8163003A908236448ADF81830ADF87F
:1089F8000C40ADF81270ADF81450ADF81A40ADF84F
:108A08001C400BF0F3F84FF480515C480BF0C3F9AD
:108A180029465A480BF093F9FFF762FC002850D01A
:108A280029464FF480400AF02DFB4FF47043294645
:108A38004FF4802001938DF808708DF80A408DF866
:108A480009608DF80B400AF005FB01A94A4809F0B6
:108A58001DFE05220C21484809F090FE05220D2133
:108A6800454809F08BFE05220E21434809F086FE91
:108A780005220F21404809F081FE41480BF076F8A5
:108A88004FF47063ADF8103003A910233C48ADF8DB
:108A98001830ADF80C40ADF80E40ADF81240ADF806
:108AA8001450ADF81640ADF81A40ADF81C400BF064
:108AB8009DF8214632480BF06EF9294630480BF0F4
:108AC8003EF901214FF480500AF0D0FAE023002447
:108AD80001930225032301214FF400308DF809305A
:108AE8008DF808508DF80A408DF80B400AF0B2FA5C
:108AF80001A94FF0904009F0C9FD052211464FF039
:108B0800904009F03BFE052206214FF0904009F005
:108B180035FE052207214FF0904009F02FFE194835
:108B28000BF024F84FF48273ADF80E304FF4E06385
:108B3800ADF810304FF40073ADF81250ADF81630A0
:108B48000125182303A90F48ADF81830ADF80C40DB
:108B5800ADF81450ADF81A40ADF81C400BF046F8CB
:108B68004FF4805107480BF016F9294605480BF0D9
:108B7800E6F809B0F0BD00BF00040048003C004022
:108B880000380040003001400128F8B505460E467F
:108B9800144604D008D3022827D00020F8BD4FF08F
:108BA80090434FF000429A61234F022138460BF060
:108BB800ACF90028F9D0F1B21F481F4E0BF04DF95F
:108BC800012130460BF0A1F90028F9D074B3012D2A
:108BD80025D029D3022DE0D14FF0904310229A617D
:108BE80016480BF03EF980B2F8BD4FF090434FF4B1
:108BF8008012124D9A61022128460BF086F900284E
:108C0800F9D0F1B20D480D4D0BF027F90121284696
:108C18000BF07BF90028F9D0002CE1D0DCE74FF00D
:108C280090434FF400429A610348DAE7012DFBD9DB
:108C3800022DB2D1D4E700BF00300140003C004013
:108C480010B5FFF71FFB0446FFF71CFB001B0028AD
:108C5800B8BF40420628F7DD10BD07B5030A8DF8F6
:108C680004308DF805008DF80610A023032201A911
:108C7800034808F053F8FFF7E3FF03B05DF804FB7F
:108C8800005400402DE9F0411546154F00228AB0E6
:108C98000E461446AC4202D10AB0BDE8F0810AABD8
:108CA8001344315D03F8221C531C00EB030818F031
:108CB8001F0F02D0691E8C420ED1030A8DF80430B2
:108CC8008DF80500A023033201A9384608F026F8DC
:108CD800FFF7B6FF4046002301341A46DAE700BF23
:108CE8000054004013B50B4C8DF80500030A8DF8AD
:108CF800043001A9A0230222204608F00FF8A0237F
:108D0800022201A9204607F0D3FF9DF8040002B013
:108D180010BD00BF005400402DE9F341124F064634
:108D280088461446054614B902B0BDE8F0812B0AFE
:108D38008DF804300222A02301A938468DF8055089
:108D480007F0ECFFFF2CA5EB060122464FF0A0032D
:108D580028BFFF224144384607F0AAFFFF2C05F13F
:108D6800FF05E1D9FF3CDEE700540040C0EBC0003E
:108D7800072200F50060FFF785BFC0EBC00007229F
:108D880000F50060FFF7C8BF70B500238AB001ADD9
:108D98001A465A550133222BFBD10B4E4FF400646F
:108DA800230A8DF804308DF80540A0232222294695
:108DB8003046203407F0B2FFFFF742FFB4F5005FFA
:108DC800EED10AB070BD00BF0054004013B50C4688
:108DD800C0EBC0000722694600F50060FFF79CFF62
:108DE8009DF8002023789A4212D19DF801206378DB
:108DF8009A420DD19DF80220A3789A4208D1DDF855
:108E08000300D4F80330C31A5842584102B010BDC9
:108E18000020FBE7704737B540F2FF70FFF762FFAD
:108E2800422802D1254B1B788BB3002140F2FF70FA
:108E3800FFF713FFFFF7A8FF402221490020FFF7A3
:108E480021FF02AD80221F494020FFF71BFF0023AE
:108E580045F8043D4FF4C3642046042229460434EF
:108E6800FFF710FFB4F5FF6FF6D1002301934FF41D
:108E7800A7642046042229460434FFF703FFB4F50B
:108E8800C36FF6D1422140F2FF70FFF7E6FE4022A1
:108E98000B490020FFF740FF80220B494020FFF7D5
:108EA8003BFFFFF71DFA4C2228B9084908480CF087
:108EB80067FC03B030BD0749F8E700BF180C002075
:108EC8000400002050580108280C0020B857010859
:108ED800AC0C002004580108034B53F82000431E33
:108EE80058425841704700BFCC000020F8B541F007
:108EF80080011746012000221E469DF818509DF853
:108F08001C40FFF741FE394600220120FFF73CFED6
:108F1800314600220120FFF737FE294600220120B2
:108F2800FFF732FE012221461046BDE8F840FFF760
:108F38002BBE10B541F08001144601200022FFF736
:108F480023FE2116002289B20120FFF71DFE210C05
:108F580000220120FFF718FEC4F30F210022012090
:108F6800FFF712FE0122E1B21046BDE81040FFF7FC
:108F78000BBE10B5002201200C46FFF705FE0022AB
:108F880011460120FFF700FE002211460120FFF7DD
:108F9800FBFD002211460120FFF7F6FD012200210A
:108FA8001046FFF7F1FD214600220120FFF7ECFDF6
:108FB800002211460120FFF7E7FD002211460402B6
:108FC8000120FFF7E1FD0022114604430120FFF7CD
:108FD800DBFD24020122044300211046FFF7D4FDE3
:108FE8002402204310BD70B504460D461646FFF70F
:108FF800C0FF294640EA06022046BDE87040FFF758
:1090080098BF70B504460D461646FFF7B2FF2946CD
:1090180020EA06022046BDE87040FFF78ABF2DE926
:10902800F8439DF8209098460F46064614460025BA
:10903800FFF79FFFC1444146012349450BD304FA7A
:1090480008F444402C4080EA040239463046BDE822
:10905800F843FFF76EBF03FA01F215430131ECE75D
:1090680010B50C2104464FF0FF32FFF762FF20468F
:109078000E21BDE81040FFF77CBF10B5CA43044677
:109088000C21FFF756FF20460E21BDE81040FFF7E0
:1090980070BF10B5074BC4B201221A5420212046D4
:1090A8000022FFF746FF204600222421BDE8104099
:1090B800FFF73FBF090C002013B57F210020FFF701
:1090C80058FF704C002120604FF480520846FFF78B
:1090D80030FF4FF0051210210020FFF72AFF236808
:1090E800012B40F0B380684A04210020FFF721FFDC
:1090F800032205210020FFF71CFF04222021002065
:10910800FFF717FF002210463721FFF712FF002252
:1091180010462121FFF70DFF4FF4480224210020BB
:10912800FFF707FF594C4FF4483228210020FFF77A
:1091380000FF4FF4483229210020FFF7FAFEA37DF3
:10914800A27A0193637A0093002318460621FFF759
:10915800CDFEA38A4E4A4F4C5A4315210020FFF7F3
:10916800E8FE626860210020FFF7E3FEA268612143
:109178000020FFF7DEFEE389227B1C2143EA02423E
:109188000020FFF7D6FE226959210020FFF7D1FE03
:10919800226A5A210020FFF7CCFE626A5B21002078
:1091A800FFF7C7FEA26A94F82C30D1B2C2F30722A7
:1091B80000920022019110465D21FFF797FE226B75
:1091C8005E210020FFF7B5FEA26918210020FFF7F5
:1091D800B0FEE26919210020FFF7ABFE626B5C214B
:1091E8000020FFF7A6FEA26B5F210020FFF7A1FE7B
:1091F800E26B52210020FFF79CFE94F84030626C2D
:10920800019394F8413000936321D3B20020C2F354
:109218000722FFF76BFE94F84830002422462046C8
:10922800019400947D21FFF761FE02212046FFF79B
:1092380024FF022220460D21FFF7D5FE12212046E9
:10924800FFF797FE144B186002B010BD134A0421B3
:109258000020FFF76EFE6FF000720C210020002442
:10926800FFF767FE0E210020FFF783FE22466D21DF
:109278002046019400942346FFF738FE22466C21CD
:10928800204633E7CC0000200D003083280C002056
:1092980000710200AC0C00201C0C00208D124084D0
:1092A800054B4FF080629A6100BF00BF00BF4FF4CA
:1092B80080629A61704700BF00040048000270474E
:1092C800800070470012704780107047704700BFD9
:1092D8000F4A1048002330B5194613705370141DF7
:1092E8004FF0FF3544F82350C15401332F2BF9D1E7
:1092F800094B82F8C0101960084B82F8CC1019602D
:10930800074BC2F8C410C2F8C810196030BD00BFBE
:10931800D00000203E0D0020D00D0020EC0D0020D4
:10932800780D002070B5044CA278637842B1034BE5
:1093380004221A7070BD00BF700D0020E40D0020DB
:10934800FF2B00F26B85DFE813F0000130014F01BD
:1093580060017201810186018B0190019901A001D0
:10936800A901B201C601DA01EA01F501FA01FF011A
:109378000A020F021A021F022C023902590266025F
:109388006D027402880269056905690591029D02EA
:10939800A4026905690569056905AA02BF02C40234
:1093A800C902690569056905690569056905CE0286
:1093B8006905690569056905690569056905690535
:1093C8006905690569056905690569056905690525
:1093D8006905690569056905690569056905690515
:1093E8006905690569056905690569056905690505
:1093F80069056905690569056905690569056905F5
:1094080069056905690569056905690569056905E4
:1094180069056905690569056905690569056905D4
:109428006905D402D902DE02E302E802ED02F20283
:10943800F702FC02010306030B0310031503690579
:109448001A03210326032B033003690536033B0364
:1094580041034F0356035C036905610367036D030A
:109468006905690569056905690569056905690584
:109478006905690569056905690569056905690574
:1094880069056905690569056905690569058A0444
:10949800900496049C04AB04BA04C004C604E10416
:1094A800E704ED04F304F904690569056905FF0497
:1094B800690506050B0515056905210528052F050C
:1094C8004C0553055A056905690569057203770353
:1094D80091039A039F0369056905A403A903AE03D1
:1094E800690562056905B2036905B703BC03CE03C4
:1094F800D303D903DE03E303E803690569056905B6
:10950800F803690569056905690569056905690556
:10951800690569056905FE0305040C0413041A04AA
:10952800210428046905690569056905690569054E
:1095380069056905690569056905690569052F04EE
:10954800750469057B0480048504002004F014FA7E
:10955800A14EA24D3721C8B9A078FFF70AFDA3781C
:1095680005EB8305D5F8D030584370609C4B1B78C9
:109578005BB1994B5A689B4B1A609B4B002A40F091
:1095880052841A6842F008021A6070BDA078FFF78A
:10959800F0FCA278954B05EB820553F82230C01AEF
:1095A800D5F8D03058437060E0E7914B8A4E187870
:1095B8008A4D212148B9FFF7DCFCA37805EB830528
:1095C800D5F8D03058437060D0E70020FFF7D1FCC1
:1095D800A278864B05EB820553F82230C01AD5F8DD
:1095E800D03058437060C1E77C4D24210020D5F865
:1095F800D460FFF7BEFCB047A37805EB8305D5F828
:10960800D0305843744B5860B0E7744D2221002085
:10961800D5F8D460FFF7ADFC0002B047A37805EB9E
:109628008305D5F8D03058436B4B58609EE76B4D97
:10963800D5F8D430D5F8D8009847A37805EB83053A
:10964800D5F8D0305843644B58608FE7694B9A6A15
:10965800614B5A608AE7674B5A7A5F4B5A6085E7D5
:10966800644B9A7A5C4B5A6080E70F210020FFF721
:1096780080FC594B00F00100586077E75E4B564A72
:109688001B8AC3F34033536070E70F210020FFF7B4
:1096980070FC514BC0F30020586067E70F21002091
:1096A800FFF767FC4C4BC0F3C01058605EE7012120
:1096B8000020FFF75EFC810741BF474A536843F02B
:1096C8000103536002077FF551AF434A536843F0E3
:1096D800020353604AE701210020FFF74AFCC30751
:1096E80041BF3D4A536843F00103536046077FF585
:1096F8003DAF394A536843F00203536036E7FEF73B
:10970800F1FD40B13B4AA378842101FB0323DA7DB4
:10971800314B5A602AE7304B03221A7026E72F4B49
:1097280025210020D3F8D440FFF723FCA0472A4B7B
:1097380058601BE72F4B1A6B274B5A6016E72D4BC7
:10974800DA6A254B5A6011E7244B27210020D3F809
:10975800D440FFF70EFCA0471F4B586006E7254B87
:109768005A6B1D4B5A6001E71C4B26210020D3F889
:10977800D440FFF7FEFBA047174B5860F6E61D4B99
:109788009A6B154B5A60F1E6FEF7ACFD0028C2D083
:10979800184AA378842101FB03231A6C0E4B5A60E4
:1097A800E4E6FEF79FFD0028B5D0124AA37884218D
:1097B80001FB03235A6C084B5A60D7E6FEF792FD6B
:1097C8000028A8D00B4AA378842101FB03239A6CB4
:1097D800014B5A60CAE600BFE40D0020D00000200B
:1097E800DF0D0020D00D0020780D0020F40B0020A4
:1097F800AC0C0020280C002000080048FEF772FD81
:10980800002888D0914AA378842101FB0323DA6CCD
:109818008F4B5A60AAE633210020FFF7AAFB8C4B36
:109828005860A3E634210020FFF7A3FB884B58605B
:109838009CE601210020FFF79CFB450641BF844AB6
:10984800536843F00103536004067FF58FAE804AE6
:10985800536843F00203536088E601210020FFF7B4
:1098680088FB7B4BC0F3012058607FE60121002074
:10987800FFF77FFB10F0100F754B14BF0122002279
:109888005A6073E601210020FFF773FB10F0200FE8
:10989800F2E76E4B93F83F206D4B5A6066E6002066
:1098A80004F06AF86A4D322120B9A078FFF761FB0D
:1098B80068605BE6A078FFF75CFBA278654B53F81D
:1098C8002230C01A686051E6634B1A68604B5A60D0
:1098D8004CE6624B1A785E4B5A6047E6604B1A6852
:1098E8005B4B5A6042E6002004F004FF584B586076
:1098F8003CE65C4B5A68564B5A6037E6594B9A68B7
:10990800534B5A6032E6574B1A7B514B5A602DE63F
:10991800544BDA894E4B5A6028E6524B1A694C4B25
:109928005A6023E64F4B1A7D494B5A601EE64D4B51
:109938005A7D474B5A6019E64A4B1A6A444B5A609B
:1099480014E6484B5A6A424B5A600FE6454B9A6AEE
:109958003F4B5A600AE6434BDA6A3D4B5A6005E6CC
:10996800404B1A6B3A4B5A6000E63E4B9A69384BAB
:109978005A60FBE53B4BDA69354B5A60F6E57C21CA
:109988000020FFF7F6FA324B5860EFE5354B5A6B7B
:109998002F4B5A60EAE5334B9A6B2D4B5A60E5E53D
:1099A800304B9A7D2A4B5A60E0E52F4B93F8DC2028
:1099B800274B5A60DAE52B4B1A78254B5A60D5E5C8
:1099C800284B93F84920224B5A60CFE51F4B204C77
:1099D800D86918B906F01CF96060C7E5662100204F
:1099E800FFF7C7FA6060C1E565210020FFF7C1FAFB
:1099F800174B5860BAE5002003F0BEFF144B5860BF
:109A0800B4E5184BDA6B124B5A60AFE5154B93F877
:109A180040200F4B5A60A9E5124B93F841200C4B9C
:109A28005A60A3E50F4B5A6C094B5A609EE5074BE9
:109A38001A7A074B5A6099E5044A0B4B1068D3F819
:109A4800D4309847024B586090E500BF280C00209E
:109A5800E40D00200C0C0020FC0B00206E0D0020F3
:109A6800E40B0020AC0C0020D00000209D4A9E4B47
:109A78005068D3F8D43098479C4B586076E59C4B97
:109A88001A689A4B5A6071E59A4B1A68974B5A6054
:109A98006CE5944B9A7D954B5A6067E5914B9A7E9D
:109AA800924B5A6062E5914BC8225A605EE5924B30
:109AB8001A688E4B5A6059E5904B1A788B4B5A604E
:109AC80054E550210020FFF754FAA2788C4B53F844
:109AD8002230C01A844B03EB8203D3F8D0305843AA
:109AE800824B586042E57F4BDA69804B5A603DE50E
:109AF8007C4B93F83C207D4B5A6037E5794B1A6ACA
:109B08007A4B5A6032E5774B5A6A784B5A602DE5A2
:109B1800744B9A8A754B5A6028E5724B734C93F8CC
:109B28003D0018B905F094FD60601FE5002005F0C0
:109B38008FFDC0F58040606018E5002005F08CFDC1
:109B48006A4B586012E50021084605F090FD674B06
:109B580058600BE50121002005F089FD634B586032
:109B680004E50221002005F082FD604B5860FDE409
:109B78000321002005F07BFD5C4B5860F6E40421CE
:109B8800002005F074FD594B5860EFE405210020D2
:109B980005F06DFD554B5860E8E40621002005F0FE
:109BA80066FD524B5860E1E4504D00236B60FEF7B0
:109BB80081FD2871FEF78CFD524B68711B8A980451
:109BC80048BFAB79A07848BF43F001034FF00F01BD
:109BD80048BFAB71FFF7CDF9C10542BFAB7943F080
:109BE8000203AB71020648BFAB79064648BF43F093
:109BF8000403A07848BFAB71FEF7B6FD18B1AB7986
:109C080043F00803AB71F30748BFAB79A07848BFAE
:109C180043F010034FF0220148BFAB71FFF7A9F9D9
:109C280018B1AB7943F02003AB71A378334AD35C06
:109C3800EB719BE42B4B93F83D202C4B5A6095E439
:109C4800314B1A68294B5A6090E4264B5A7E274BB1
:109C58005A608BE4234B1A7E244B5A6086E400201A
:109C680006F0C5FA214B586080E4002006F0E9FAB6
:109C78001E4B58607AE4002006F0F1FA1B4B58603E
:109C880074E4002006F0DDFA184D20B9A07806F03B
:109C980000FB68606AE4A07806F0E8FA686065E4AA
:109CA800002006F0CEFA114D20B9A07806F098FAF7
:109CB80068605BE4A07806F0E5FA686056E4002086
:109CC80006F07CFA094B586050E4002006F08CFB43
:109CD800064B58604AE4002006F066FB034B5860C8
:109CE80044E400BF280C0020D0000020E40D002030
:109CF800EC0B0020F80C0020140C0020260C00208F
:109D08000C0C0020000800481C0C0020002006F065
:109D180052FB474B586029E4002006F03EFB444BB9
:109D2800586023E4002006F04DFB414B58601DE4C9
:109D3800002006F060FB3E4B586017E4002006F058
:109D480048FB3B4B586011E40B21002006F0E8F873
:109D5800374B58600AE4374B1A78354B5A6005E49C
:109D6800354A364B1069D3F8D4309847304B586091
:109D7800FFF7FCBB314B14210020D3F8D44006F088
:109D8800CFF8A0472A4B5860FFF7F0BB002006F039
:109D98005FFA274B5860FFF7E9BB002006F02EFA60
:109DA800234B5860FFF7E2BB1321002006F0B8F8F8
:109DB8001F4D90B1224BB3FBF0F06860A3781E4AA8
:109DC800842101FB03231B7E002B7FF4CFAB686843
:109DD800FFF774FA6860FFF7C9BB6FF07F436B60E9
:109DE800ECE7002006F092FB114B5860FFF7BEBB72
:109DF800002006F092FB0E4B5860FFF7B7BB7121AD
:109E0800002006F08DF80A4B5860FFF7AFBB002022
:109E180006F060FB064B5860FFF7A8BB044B032213
:109E28001A70FFF7A3BB1A6822F00802FFF7ACBB51
:109E3800E40D0020F80B0020280C0020D0000020A2
:109E48000024F40038B5B04A9378022B144600F089
:109E58001681032B00F01A81002B40F09381537870
:109E68004D2B00F0BE8043D8452B00F0928019D8C6
:109E7800422B00F0848006D8402B74D0412B79D037
:109E88000322A24B6DE0432B7ED0442BF8D1A0498E
:109E9800D2F8033041F81C3F04221C20BDE83840AA
:109EA800FEF7F0BE482B00F0818014D8462B75D001
:109EB800472BE5D1964DD2F803302946042241F8C4
:109EC800083F0820FEF7DEFE2A69A9686879BDE820
:109ED800384006F0E9BC4B2B79D07DD8492BCFD13F
:109EE800D2788B4B002A6DD1DA75D97D17203DE0E9
:109EF800552B00F0A0801BD8512B7ED008D84F2BB3
:109F080074D0502BBCD1824BD178997516202DE096
:109F1800532B00F087807DD9D2F80330012B00F253
:109F280031817B49D37801F81A3F01221A20B5E71D
:109F3800832B00F093800BD8572B00F088805C2B84
:109F48009ED17349D37801F8273F01222720A5E73E
:109F5800852B00F08E80C0F08780FF2B90D1D278BF
:109F68006C4B1A7038BDD17840F2FF70BDE83840AC
:109F7800FEF773BE664BD17819700020F6E7644B84
:109F8800D17859700120F1E7614BD178197104201B
:109F9800ECE75F4BD17859710520E7E75C49D2F8C7
:109FA800033041F80C3F04220C2077E75849D37856
:109FB80001F8243F01222420FEF764FEBDE8384062
:109FC80003F0A4BC51490122DA754A608DE7504B71
:109FD800D178D9700320C9E74D4BD1789970022008
:109FE800C4E74B4BD17859751520BFE7D2F8031059
:109FF800474BC9B259761920B8E7454D2A7DD20793
:10A0080004D5E378DB0701D4FEF7BEFEE1782975B5
:10A018001420ABE73E49D2F8033041F8203F042230
:10A0280020203BE73A4DD2F803302946042241F874
:10A03800103F102046E7D2F80330012B00F2A2802F
:10A048003349D37801F81B3F01221B2026E730490A
:10A05800D37801F8253F012225201FE72E4BD2F89F
:10A068000320C3F8E02038BD2C4BD2F803201A6037
:10A0780038BD294BD2F80320C3F8E42038BD517805
:10A08800274BD2F8032043F8212038BD5378272BDB
:10A0980060D018D8022B47D00DD853B3012B7FF4CA
:10A0A800EFAE204BD2F803205A60FEF7EBF81A4BBC
:10A0B800C3F8EC0038BD1B2B40D01C2B44D0092B17
:10A0C8007FF4DEAE38BD2B2B4DD007D8292BD2F824
:10A0D8000320144B45D042D9DA6138BD2D2B4CD022
:10A0E80046D32E2B7FF4CCAE0E4BD2F80320DA6287
:10A0F80038BD0C4BD2F803201A60FEF7C3F8064BA4
:10A10800C3F8E80038BD00BF700D0020E40D002042
:10A1180004000020DE0D0020D0000020E00D00200B
:10A12800F00D0020FC0C0020174BD2F803209A6099
:10A13800FEF7A8F8154BC3F8F00038BDD2F8033085
:10A14800114ADBB2137338BDD2F803300E4ADBB2C2
:10A15800537338BD0C4BD2F803201A6138BD5A61CD
:10A1680038BD9A6138BD084BD2F803201A6238BD51
:10A17800054BD2F803205A6238BD034BD2F80320AE
:10A188009A6238BD04227CE6FC0C0020D000002036
:10A1980038B5254CA078002844D103F0A9FB18B1A4
:10A1A8000622224B1A7038BDA07803F065FC012501
:10A1B800A0781F4B4FF0006229461D54FEF713FF8D
:10A1C800A0781C4A842303FB0023DB7D43BB2A467B
:10A1D8002021FEF7AEFEA578174BD4F8032003EB39
:10A1E8008503D3F8D000D3F8F4305043984724219E
:10A1F80002462846FEF79DFEA0784FF080520721C0
:10A20800FEF7F1FEA0784FF000620721FEF7F9FE95
:10A21800A0784FF000620121BDE83840FEF7F1BE9A
:10A228000222D5E70422BCE7700D0020E40D0020CF
:10A23800090C0020280C0020D000002038B5264C3E
:10A24800A078002845D103F053FB18B10622234B10
:10A258001A7038BDA07803F00FFC0125A078204BB8
:10A268004FF0006229461D54FEF7BDFEA0781D4A36
:10A27800842303FB0023DB7D4BBB2A462021FEF70A
:10A2880058FEA578184BD4F8032003EB85035242F7
:10A29800D3F8D000D3F8F43050439847242102462D
:10A2A8002846FEF746FEA0784FF080520721FEF7B9
:10A2B8009AFEA0784FF000620721FEF7A2FEA07870
:10A2C8004FF000620121BDE83840FEF79ABE022235
:10A2D800D4E70422BBE700BF700D0020E40D002086
:10A2E800090C0020280C0020D0000020F8B5A24C52
:10A2F800A078002840F03E8103F0FAFA18B106224F
:10A308009E4B1A70F8BD6178012949D003D3022900
:10A3180000F0A780F8BD4FF00062A0780121FEF799
:10A3280062FEA078964A842303FB0023DB7D6BBB87
:10A3380005222021FEF7FDFD924EA078924D335C58
:10A348004BB105EB80032421D3F8D820FEF7F1FDAB
:10A35800A3780022F2544FF080520721A078FEF72C
:10A3680050FE4FF000620721A078FEF73CFEA0786F
:10A37800864AD4F803104C234343D25C83001D441F
:10A3880032B9D5F8D0204A43372150E00622D0E729
:10A39800D5F8D0207E4B53F8203001FB0232F3E78A
:10A3A8004FF00062A078FEF71EFEA078744A84235E
:10A3B80003FB0023DB7D7BB905222021FEF7B9FDD5
:10A3C800714EA078331893F8DC30012B36D005D3C2
:10A3D800022B35D000250DE00622EEE73721FEF7E7
:10A3E800C8FDA378D4F8035006EB8303D3F8D03024
:10A3F80003FB0505A078634F3B5C4BB106EB800679
:10A408002421D6F8D820FEF794FDA3780022FA5428
:10A418004FF080520721A078FEF7F3FD4FF000625D
:10A428000721A078FEF7DFFDA0782A463721FEF73E
:10A4380080FD4FF000620121A07849E02121CEE79C
:10A448005021FEF796FDA3785249D4F8035006EB45
:10A45800830251F82330D2F8D020C01A02FB050538
:10A46800C8E7A3781A0646D5DB077FF54BAF444B00
:10A47800DB7D8BBB0522434E434D2021FEF759FD62
:10A4880033783BB1D5F8D82024210020FEF751FDC0
:10A49800002333704FF0805207210020FEF7B1FDF2
:10A4A8004FF0006200200721FEF79DFD374BD4F8DE
:10A4B80003201878384B88B953F82230D5F8D020C3
:10A4C80037215A43FEF735FD4FF000620121002085
:10A4D800BDE8F840FEF795BD0622CCE753F82220E8
:10A4E800A0782B4BD5F8D01053F82030002001FB72
:10A4F80002323721E6E72249842202FB0312D27D89
:10A508008ABB052218462021FEF713FD1D4EA078B0
:10A518001D4D335C4BB105EB80032421D3F8D820C3
:10A52800FEF707FDA3780022F2544FF0805207216E
:10A53800A078FEF766FD4FF000620721A078FEF7CD
:10A5480052FDA078114A14494C234343D65CD4F8F1
:10A5580003308200034415443EB951F82330D5F83E
:10A56800D0205A4310E70622CCE751F82320D5F82B
:10A57800D0100FE70422C3E6700D0020E40D002080
:10A58800280C0020090C0020D0000020AC0C002072
:10A59800F40B00200C0C00207C0D0020014B93F8DC
:10A5A800F8007047D000002070B5674E674B8425CF
:10A5B80005FB00650446A96A99420CD8EA6A9A42E2
:10A5C80009D82A6B9A4206D86A6B9A4203D8AA6BB2
:10A5D8009A4240F28380842505FB0465022200210B
:10A5E8002046FEF700FDD5ED0A7AF8EE677A17EEF9
:10A5F800900A0AF049FC0022554B0AF099FC50A336
:10A60800D3E900230AF0BEFD0AF0A4FE2821024681
:10A618002046FEF78EFCD5ED0B7AF8EE677A17EE3A
:10A62800900A0AF031FC0022494B0AF081FC44A34D
:10A63800D3E900230AF0A6FD0AF08CFE2921024680
:10A648002046FEF776FCD5ED0C7AF8EE677A17EE21
:10A65800900A0AF019FC00223D4B0AF069FC38A365
:10A66800D3E900230AF08EFD0AF074FE2A2102467F
:10A678002046FEF75EFCD5ED0D7AF8EE677A17EE08
:10A68800900A0AF001FC0022314B0AF051FC2CA37D
:10A69800D3E900230AF076FD0AF05CFE2B2102467E
:10A6A8002046FEF746FCA86B07EE900AF8EE677A9C
:10A6B80017EE900A0AF0E8FB0022254B0AF038FC56
:10A6C8001FA3D3E900230AF05DFD0AF043FE02460A
:10A6D8002C212046BDE87040FEF72BBC1D4E06EB32
:10A6E800840602220021FEF78CFCD6F8FC30A86A0A
:10A6F8009847282102462046FEF71BFCD6F8FC3076
:10A70800E86A9847292102462046FEF712FCD6F847
:10A71800FC30286B98472A2102462046FEF709FCA0
:10A72800D6F8FC30686B98472B2102462046FEF786
:10A7380000FCD6F8FC30A86B9847C8E7AFF3008058
:10A74800000000A2941AED42280C0020FFFF3F00F1
:10A7580000004042D00000202DE9F74F564A8423DC
:10A7680003FB0023824693F83F401A6C5E6CA4FBFF
:10A7780002899A6CDB6CA4FB0212CDE900126FF01F
:10A788007F42A4FB06674245A4FB03454FF0000344
:10A7980073EB09010CDBB24273EB070108DBDDE95F
:10A7A80000BC5A4573EB0C0102DBA242AB4163DAF1
:10A7B800042200215046FEF716FC494640460AF09E
:10A7C80011FF0AF061FB38A3D3E900230AF0B0FBBC
:10A7D80037A3D3E900230AF0D5FC0AF0BBFD2D21ED
:10A7E80002465046FEF7A5FB394630460AF0FAFE07
:10A7F8000AF04AFB2CA3D3E900230AF099FB2CA307
:10A80800D3E900230AF0BEFC0AF0A4FD2E2102467B
:10A818005046FEF78EFBDDE900010AF0E3FE0AF080
:10A8280033FB21A3D3E900230AF082FB20A3D3E959
:10A8380000230AF0A7FC0AF08DFD2F21024650469E
:10A84800FEF777FB294620460AF0CCFE0AF01CFBEF
:10A8580015A3D3E900230AF06BFB15A3D3E9002362
:10A868000AF090FC0AF076FD02463021504603B00B
:10A87800BDE8F04FFEF75DBB04220021FEF7C1FBE7
:10A8880042462D215046FEF754FB32462E215046B3
:10A89800FEF74FFB009A2F215046FEF74AFB22464F
:10A8A800E3E700BFAFF3008020FCFFFFFFFF3F435B
:10A8B80000C84E676DC16B44280C002073B5034C6B
:10A8C800A278637822B1042200F058BC700D0020F1
:10A8D800FF2B00F2C385DFE813F0000118014401E3
:10A8E800C105560173017D019E01C105C105C10560
:10A8F800C105AA01BD01CE01DF01E801ED01F201A8
:10A90800FB01000209020E0220022E023C024A024A
:10A918004E0252026402C105C105C10571028B02D3
:10A928009902C105C105C105C105A502B602BE024D
:10A93800C202C105C105C105C105C105C105C702DE
:10A94800C105C105C105C105C105C105C105C105CF
:10A95800C105C105C105C105C105C105C105C105BF
:10A96800C105C105C105C105C105C105C105C105AF
:10A97800C105C105C105C105C105C105C105C1059F
:10A98800C105C105C105C105C105C105C105C1058F
:10A99800C105C105C105C105C105C105C105C1057F
:10A9A800C105C105C105C105C105C105C105C1056F
:10A9B800C105D402E302F2020E031E03240331038D
:10A9C800420348034E035C0368036E037403C10526
:10A9D800C1057A03800386039103C1059B03A50380
:10A9E800C105C105C105AF03C105B503BF03CD034B
:10A9F800C105C105C105C105C105C105C105C1051F
:10AA0800C105C105C105C105C105C105C105C1050E
:10AA1800C105C105C105C105C105C105C105B80408
:10AA2800C104CA04D304E604F90402050B0514059D
:10AA38001D0526052F053805C105C105C105C10538
:10AA4800C105C10541054A05C10553055C056505F4
:10AA58009705AF05C105C105C105C105D403D903D3
:10AA6800E203C105C105C105C105EB030504C10524
:10AA7800C105B805C105C105C105C10509043004F2
:10AA8800530458045E046304C105C105C105C1052A
:10AA9800C105C105C105C105C105C105C105C1057E
:10AAA800C105C105C105C105C105C105C105C1056E
:10AAB800C105C105C105C105C105C105C105C1055E
:10AAC800C105C105C105C105C105C105C105C1054E
:10AAD8006B047D0480048E049C04BF4BD4F80320CF
:10AAE8001878BE4B40B9D3F8D03037215A4302B05A
:10AAF800BDE87040FEF71DBAD3F8D010B84B1B68FC
:10AB080001FB023237210020F1E7B34BB34D18782F
:10AB180030B9D4F80330D5F8D02021215A43E6E7DC
:10AB280021210020FEF725FAA378D4F8032005EBAD
:10AB38008301D1F8D01001FB1200A94A502142F834
:10AB480023001846FEF715FAA278D4F8033005EB6F
:10AB58008205D5F8D01001FB1300A24B43F8220060
:10AB680046E0A14B9D4DD4F8030001221A70D5F898
:10AB7800F4309847A37805EB83052421D5F8D02035
:10AB880042431846B3E7954DD4F80300D5F8F4309E
:10AB980098470028B8BF4042C5F8D8002021A078BF
:10ABA800FEF7E7F9400723D5A678D4F8030005EBAC
:10ABB8008605D5F8F430984724210246304696E7B2
:10ABC8008A4BD4F803209A62002002B0BDE8704096
:10ABD800FFF7EABC804B85491B78E07848724BB98F
:10ABE8008A7A897D8DE8030006211846FEF77EF9EA
:10ABF80002B070BD1021002005F092F9E37820F42E
:10AC0800F852DB0842EA03221021002002B0BDE816
:10AC1800704005F059B9704B74491B78E2788A7214
:10AC2800002BE5D1887D0190497A0091DCE701216C
:10AC38000020FEF79EF9D4F8033020F00A02D90765
:10AC480048BF42F002029E0701D542F008020121E6
:10AC5800A0784CE701210020FEF78BF9D4F80330E7
:10AC680020F00502DD0748BF42F001029807EED543
:10AC780042F00402EBE7FDF735FB002800F0EE8315
:10AC8800D4F80320012A3FF61EAEA3785749842042
:10AC980000FB0313DA75ABE7504BD4F80300D3F885
:10ACA800F4309847252102462DE7504BD4F803206D
:10ACB8001A6389E74D4BD4F80320DA6284E7474BDF
:10ACC800D4F80300D3F8F4309847272102461AE74E
:10ACD800464BD4F803205A6376E7404BD4F8030078
:10ACE800D3F8F4309847262102460CE73F4BD4F8B6
:10ACF80003209A6368E7FDF7F5FA002800F0AE83B1
:10AD08003A4AA078842303FB0023D4F803201A646A
:10AD180002B0BDE87040FFF71FBDFDF7E3FA002859
:10AD280000F09C83314AA078842303FB0023D4F8E5
:10AD380003205A64ECE7FDF7D5FA002800F08E836B
:10AD48002A4AA078842303FB0023D4F803209A64BA
:10AD5800DEE7FDF7C7FA002800F08083234AA078D1
:10AD6800842303FB0023D4F80320DA64D0E7D4F863
:10AD780003203321C7E6D4F803203421C3E6012198
:10AD88000020FEF7F6F8D4F8033020F0C002D90707
:10AD980048BF42F040029B077FF559AF42F080025E
:10ADA80055E701210020FEF7E4F8D4F803301B0230
:10ADB80020F4407203F440731A4348E7012100204D
:10ADC800FEF7D7F8D4F8033020F01002002B3FF438
:10ADD8003EAF42F010023AE7AC0C0020D000002051
:10ADE800F40B00200C0C0020090C0020280C00207B
:10ADF80001210020FEF7BDF8D4F8033020F020022E
:10AE0800002B3FF424AF42F0200220E7D4F80330AF
:10AE1800013BFE2B3FF657ADAA4BE27883F83F2063
:10AE2800002075E7002002F0A7FD18B9D4F8032028
:10AE380032210DE7A078A44BD4F8032053F8203032
:10AE480032211A4453E6D4F80330002BFFF63BAD09
:10AE58009E4A1360CCE6E2789D4B1A70C8E69D4B7B
:10AE6800D4F803201A60C3E69B4B1B78002B3FF4F1
:10AE7800BFAED4F80310002002B0BDE8704002F065
:10AE8800CDBD954BD4F8030058608E4BDD6925B9CC
:10AE980004F016FC2A466021DAE60246602132E612
:10AEA8008D4BD4F803009860864BDD6925B904F012
:10AEB80019FC2A466121CBE60246612123E6864B2E
:10AEC800D4F8030018737F4BDB694BB904F022FCFC
:10AED8001C21A078FEF74DF8C0F308021C21B7E644
:10AEE8001C210020FEF745F8D4F80320C0F3080021
:10AEF80040EA0242F2E7784BD4F80320DA811C21B9
:10AF08000020FEF736F8D4F8033000F47F02C3F3CC
:10AF180008031A43E2E7704BD4F803201A61592159
:10AF2800F1E56D4AD4F803101378C9B21175002BF6
:10AF38003FF45EAE937D0191527D0BE06649D4F8F3
:10AF480003200B78D2B24A75002B3FF451AE8B7DAB
:10AF5800097D0191009206210022002046E65E4B01
:10AF6800D4F803201A625A21CDE55B4BD4F80320AC
:10AF78005A625B21C7E5D4F80320574BD1B29A62D5
:10AF8800C2F3072293F82C300191009200225D2130
:10AF9800E3E7514AD4F80330D362926AD1B2C2F3DC
:10AFA800072201910092DBB2F0E74B4BD4F8032063
:10AFB8001A635E21A7E5484BD4F803209A6118214B
:10AFC800A1E5454BD4F80320DA6119219BE5424BF2
:10AFD800D4F803205A635C2195E53F4BD4F803204D
:10AFE8009A635F218FE53C4AD4F803301178DBB2CD
:10AFF800937500293FF4FCAD117D9CE7D4F803302C
:10B00800022B3FF660AC354BE27883F8DC20EFE5A5
:10B01800D4F80330304A012B0ABF314900230B70A2
:10B028001370E5E5D4F80330012B3FF64CAC2A4BFE
:10B03800E27883F84920DBE5274BD4F80320DA636C
:10B04800522160E5244BE1785A6C83F84010019155
:10B0580093F84130009308E01F4BE17883F84110E2
:10B068005A6C93F840308DE80A00D3B26321C2F3DA
:10B07800072272E7184BD4F803205A6493F840105B
:10B08800E5E7104BD4F803201A72B1E5134BD4F856
:10B098000300D3F8F43098470A4B1860A8E50F4B23
:10B0A800D4F80300D3F8F4309847064B58609FE56E
:10B0B800094B04491B78E0788875002B7FF498AD1C
:10B0C8008A7AB0E5280C00200C0C0020FC0B00202C
:10B0D8006E0D0020E40B0020AC0C0020D0000020F6
:10B0E800090C0020B94BE2789A7681E550210020BE
:10B0F800FDF73FFFB64DA378D4F8032005EB830195
:10B10800D1F8D01001FB1200B24AB34942F823002B
:10B118004C225A438A5C002A3FF46AAD2121184622
:10B12800FDF727FFA278D4F8033005EB8205D5F8A0
:10B13800D01001FB1300A94B10E5A44DD4F803204F
:10B14800E9698A423FF454ADA34B1878A8B9002A9C
:10B1580010DD012004F0F0FAD4F80320A07854217F
:10B16800FDF7E7FEA378842202FB0353D4F80320FB
:10B17800DA613DE504F0E0FAF4E70622984B6CE664
:10B18800924BE27883F83C2032E5904BD4F80320C8
:10B198001A625321B7E48D4BD4F803205A6227E58D
:10B1A8008A4AD4F8033093828E4A15215A43AAE476
:10B1B800D4F80300864B854A012120B982F83D0066
:10B1C800C3F8D01014E582F83D104FF0FF32C3F8F1
:10B1D800D0200DE5E278844B3FE6844BD4F8032079
:10B1E8001A60002002F084FB00287FF401ADD4F837
:10B1F800032012212CE5D4F803300F2B3FF663AB64
:10B20800E178724B0020597602B0BDE8704002F038
:10B21800BDBBD4F803306BB1012B7FF454AB6B4A40
:10B2280013766B4B724AC3F8F420724AC3F8D420E1
:10B23800714A07E0654A1376654B704AC3F8F420F3
:10B24800C3F8D420C3F8FC20D2E4D4F803100020BB
:10B25800C9B202B0BDE8704004F0CEBED4F8031005
:10B268000020C9B202B0BDE8704004F031BFD4F884
:10B2780003100020C9B202B0BDE8704004F04CBF12
:10B28800002004F0DEFFD4F80310C9B228B9A07872
:10B2980002B0BDE8704004F07DBFA07802B0BDE800
:10B2A800704004F04BBF002004F0CBFFD4F803102B
:10B2B800C9B228B9A07802B0BDE8704004F08ABECF
:10B2C800A07802B0BDE8704004F052BFD4F8031073
:10B2D8000020C9B202B0BDE8704004F061BED4F8E5
:10B2E80003100020C9B202B0BDE8704005F031B8C3
:10B2F800D4F803100020C9B202B0BDE8704004F0D1
:10B30800E3BFD4F803100020C9B202B0BDE8704012
:10B3180004F0ECBFD4F803100020C9B202B0BDE8B5
:10B32800704004F0BFBFD4F803100020C9B202B0C7
:10B33800BDE8704004F0ECBFD4F803100020C9B297
:10B3480002B0BDE8704005F016B8D4F8031000202C
:10B35800C9B202B0BDE8704004F0EBBF1C4BD4F892
:10B368000300D3F8F4309847184B186140E4184BA1
:10B37800D4F80300D3F8F43098471421024644E483
:10B38800D4F803100020C9B202B0BDE8704004F040
:10B39800B1BED4F803100020C9B202B0BDE87040B5
:10B3A80004F03CBED4F803000028FFF68CAA074B33
:10B3B8001B7E012B01D0FDF785FF28B1104AB2FB97
:10B3C800F0F21321A07821E40E4AFAE7280C0020B5
:10B3D800D00000200C0C0020AC0C0020F40B002046
:10B3E800E40D0020007102002C0D00201C0C002030
:10B3F800C5920008CD920008C9920008D5920008AD
:10B408000024F400B5001000D4F803100020C9B2DD
:10B4180005F040F80021A07804F082FDD4F803106C
:10B428000246A07821B142F004020021FFF7EEBBEA
:10B4380022F00402FFF7EABBD4F803100020C9B2D7
:10B4480002B0BDE8704005F035B8D4F8031000200C
:10B45800C9B202B0BDE8704004F0D4BF03228DE643
:10B468002DE9F341AD4CAE4D2378D4F803006B7051
:10B4780064222A2B2A70686001F0CC8000F2EB80ED
:10B48800162B00F0E38472D8092B00F04B8226D8E3
:10B49800042B00F01B820AD8022B00F0F98100F27D
:10B4A800FA81012B00F0E58102232B70E3E1062BE2
:10B4B80000F01282C0F00D82072B00F01082082BDA
:10B4C800F2D1A378002B40F0FE816378C92B00F0FD
:10B4D8001D82D22B00F0208203232B70CBE10E2B90
:10B4E80000F0838319D80B2B00F03D83C0F01D8238
:10B4F8000C2B00F04D830D2BD6D1A078002840F0FE
:10B50800E2816378012B00F05883C0F05383022B4B
:10B5180000F0568303232B70ADE1132B00F0B783A3
:10B528000DD80F2BC0D1A378012B00F0A383C0F056
:10B538008283022B00F0A28304232B7086E3142B52
:10B5480000F0EF83152BAFD163780C2B00F29381B9
:10B55800DFE813F006040F04180421042A04330456
:10B568003D0446044F04580461046A047304202B04
:10B5780000F0008637D81A2B00F095840CD8182BC9
:10B5880000F07A8440F2668463782E2B00F284847B
:10B59800644A0121D1546EE11C2B00F08585C0F06E
:10B5A80090841E2B00F086851F2B7FF47DAF60787A
:10B5B800142800F2E782A378002B40F0BC855A4B90
:10B5C80053F82020594B6A601B78002B00F05381F8
:10B5D800574B1A60574B002A40F0A7851A6842F06B
:10B5E80008021A6047E1252B00F0A48616D8222B02
:10B5F80000F05886C0F00086232B00F05B86242BD1
:10B608007FF452AF6378052B00F23581DFE813F041
:10B6180068066F0676067D0684068B06272B00F0E3
:10B62800BB86C0F09186282B00F0C586292B7FF4B5
:10B638003BAF63780B2B00F2E987DFE813F05A077A
:10B64800650770077B0787079507A007AB07B6074D
:10B65800BF07D507E007472B01F04D836ED8372B7E
:10B6680001F0118239D82E2B01F0EE8116D82C2B3F
:10B6780001F0E58041F2558063780B2B01F2E081FF
:10B68800DFE813F07D0986098F099809A209AE0938
:10B69800B709C009C909D209DE09D809312B01F057
:10B6A800DB810DD8302B7FF4FFAEFDF711FE224B66
:10B6B800012283F8C020D4F80320C3F8C420DAE0BC
:10B6C800322B01F0D881332B7FF4EEAE184B1B6878
:10B6D800C4F80330FEF75CFDCDE0422B01F0FB829D
:10B6E8000DD8392B01F0F281C1F0D781402B01F040
:10B6F800EE82412B7FF4D8AE02F0B2F8BBE0442BC7
:10B7080001F0F182C1F0EB82452B01F0F082462B6B
:10B718007FF4CAAE02F0EAF8ADE000BF700D002079
:10B72800E40D00203E0D00207C0D0020DF0D0020E0
:10B73800D00D0020780D0020D0000020872B01F0CC
:10B74800618362D8822B01F0F98220D8802B01F026
:10B75800D68201F2DA82502B7FF4A6AEAF4BD3F833
:10B76800C820072A00F2878061780C2900F28380BC
:10B77800DFE811F0B809CA09DC09F8090A0A1C0A45
:10B788002F0A410A530A650A770A890A9B0A842BF9
:10B79800A34A01F0DD82C1F0D782852B01F0EB824C
:10B7A800862B7FF481AE9F4B9F4E01271F70B0F50B
:10B7B8005B7F9378337081F0E482127D12EA070888
:10B7C80041F0DF826946FDF7D8FA9DF800307370C2
:10B7D8009DF80130B3709DF80230F3709DF8063083
:10B7E80033719DF8053073719DF80430B3719DF87D
:10B7F8000330F37186F808803B46F15C327A0133F6
:10B808000A44082B3272F8D135E08C2B01F06B8397
:10B818000FD8892B01F02483C1F0BD828A2B01F057
:10B8280049838B2B7FF440AE7C4B012283F84D215A
:10B8380021E0992B01F0C6830CD88D2B7FF434AE10
:10B848006378032B01F2BA83DFE813F08D0B740BD6
:10B85800A60BB40BF22B01F00184FF2B7FF424AE6E
:10B8680040F2D243984206D16C4B012283F87C21E6
:10B8780001E0FEF78DFC6A4B93F827302BB194F961
:10B888000030002BA4BF63782B7002B0BDE8F081B4
:10B89800FEF7D4FCEFE7A378ABB9644901220A703C
:10B8A8006349C87D58B92021FDF743FBA0780022E1
:10B8B8002421FDF73EFBA07802F0DEF8DBE7022248
:10B8C80020211846F0E704232B70D4E7FEF70EFD7D
:10B8D800D1E7FEF7F3FFCEE7FDF724FDCBE7A3782A
:10B8E800002BF0D16378C92B04D0D22B08D00323C6
:10B8F8002B70C0E701224F495A20FDF7C3F9BAE778
:10B9080004224D495C20FDF7BDF9B4E701224949FD
:10B918005A20FDF701FAAEE7042247495C20FDF7FB
:10B92800FBF9A8E7FEF78EFAA5E7A378022B00F04B
:10B93800CF80032B00F0D180002B40F00D8163787D
:10B94800374A502B00F0958026D8462B00F084808B
:10B958000ED8422B7AD006D8402B45D0412B59D04F
:10B9680003232B7045E0442B74D071D9537952E0EE
:10B978004B2B78D009D8482B72D06FD3492BEFD1F5
:10B98800D37D003318BF012345E04D2B6FD06CD316
:10B998004F2BE5D1537E3EE05C2B74D010D8532B4F
:10B9A8006BD005D8512B66D0522BD9D1136A32E00F
:10B9B800552B66D063D3572BD2D192F825302AE085
:10B9C800832B71D008D8812B60D069D8802BC7D140
:10B9D800124B93F8C0301EE0852B6CD068D3FF2B38
:10B9E800BED1164B1B78CCE740F2FF70FDF77AF911
:10B9F8006860134B1B78002B3FF43DAF114B6A680E
:10BA08001A60114B002A40F0A9801A6842F0080217
:10BA18001A6030E713786B60EBE700BFD0000020B6
:10BA280004000020D40D0020D50D0020090C0020B2
:10BA3800280C0020420C0020440C0020DE0D0020C1
:10BA4800DF0D0020D00D0020780D00205378E2E7AC
:10BA58001379E0E7D369DEE7D368DCE79368DAE7D0
:10BA680092F82430D7E7D378D5E79378D3E7537D96
:10BA7800D1E7937DCFE7137DCDE71369CBE7937EBD
:10BA8800C9E7D37EC7E792F82730C4E7994B93F804
:10BA9800C030A3F1040CDCF1000343EB0C03BAE75C
:10BAA800944BD3F8C430B6E7924BD3F8E030B2E702
:10BAB800914B1B68AFE78F4A9048D2F8E43043F2C5
:10BAC800390100FB0313C2F8E43023F00043A2E776
:10BAD80062788B4B53F822309DE76378282B2CD063
:10BAE80012D8022B26D006D813B3012B7FF438AF17
:10BAF800844B5B688FE7092B3FF47BAF272B7FF4E0
:10BB08002FAF804B1B6986E72B2B1CD007D8292B1E
:10BB180016D02A2B7FF424AF7A4BDB697BE72D2BD9
:10BB280017D013D32E2B7FF41BAF764BDB6A72E74B
:10BB3800744BBEE7734B9B686DE7724B5B696AE7B2
:10BB4800704B9B6967E76F4B1B6A64E76D4B5B6AD9
:10BB580061E76C4B9B6A5EE7042302E71A6822F0F0
:10BB680008021A6087E6A378022B0ED1607837287E
:10BB780008D800F5A7706449800004220144FDF745
:10BB880081F878E603232B7075E604232B7072E6A0
:10BB9800A378022B0BD160783728F3D800F5A7706B
:10BBA8005949800004220144FDF7B6F863E60423EE
:10BBB8002B7060E603F0D8F85DE603F0DDF85AE68E
:10BBC80003F0E2F8514B68601B78002B3FF453AE4A
:10BBD8004F4B18604F4B1A6818B942F008021A60A8
:10BBE80049E622F008021A6045E6A37823B1022B41
:10BBF8000BD004232B703EE6FCF78BFB0028C1D04A
:10BC0800D4F80300FCF774FD35E66378072B08D8F1
:10BC180018B91846FCF7D2FC2DE61846FCF7EEFCDE
:10BC280029E6FF2BAED1471C0ABF394BC0B21878A2
:10BC3800FCF704FD1FE66078082803D8FCF70FFD21
:10BC4800686003E00A2810D100236B602F4B1B7833
:10BC5800002B3FF410AE2E4B6A681A602D4B8AB940
:10BC68001A6842F008021A6005E6FF28EED1FCF7D0
:10BC780021FDE5E7607804F0A3F8E1E76078FCF7D8
:10BC880001FDDDE71A6822F008021A60F3E5627820
:10BC98001F4B092A26D8DFE802F005090C0F1319F3
:10BCA8001C1F22071A68104418601BE01A68101A33
:10BCB800FAE71A685043F7E71A6892FBF0F0F3E7DF
:10BCC800196891FBF0F200FB1210EDE71A681040BA
:10BCD800EAE71A681043E7E71A685040E4E71A6889
:10BCE800D2431A601A680B4BB2B91A6842F00802BC
:10BCF8001A60C0E5D0000020E00D00206D4EC6415E
:10BD0800F00D0020FC0C0020B8080020DF0D0020FA
:10BD1800D00D0020780D00201A6822F008021A6061
:10BD2800A9E5AC4BAC4A1968136888420ADA23F0D3
:10BD3800030343F004031360136869B943F008036D
:10BD4800136098E50BBF23F0060323F0050343F0C7
:10BD5800010343F00203EEE723F0080313608AE5CA
:10BD68009D4B1B681E077FF586AD9C4BC3F8C4002E
:10BD780081E5994B1B6819073FF57DAD974BC3F8D3
:10BD8800C40078E5944B1B68DA077FF574AD934BD4
:10BD9800C3F8C4006FE5904B1B68DB073FF56BAD3C
:10BDA8008E4BC3F8C40066E58B4B1B685F077FF5B5
:10BDB80062AD8A4BC3F8C4005DE5874B1B6813F07E
:10BDC800050F3FF458AD854BC3F8C40053E5824BCB
:10BDD8001B689E077FF54FAD804BC3F8C4004AE54A
:10BDE8007D4B1B6899073FF446AD7C4BC3F8C400F4
:10BDF80041E5794B1B68DA067FF53DAD774BC3F813
:10BE0800C40038E5744B1B689B067FF534AD734B53
:10BE1800C3F8C4002FE5704B1B685F067FF52BAD98
:10BE28006E4BC3F8C40026E56B4B1B681E067FF5F6
:10BE380022AD6A4BC3F8C4001DE5674B1B68D905E2
:10BE48007FF519AD654BC3F8C40014E5634BC3F81F
:10BE5800C40010E5614BD3F8C820072A3FF60BADA4
:10BE6800511C03EB8202C3F8C810D3F8C410C2F8FF
:10BE78000011C3F8C400FEE4584AD2F8C830002BB9
:10BE88003FF4F9AC013BC2F8C83002EB8303D3F8A6
:10BE98000031C2F8C430EEE4FF2B7FF473AE4F4B91
:10BEA80001221A70E7E463782E2B03D84C4A00214C
:10BEB800D154E0E4FF2B7FF465AE484B00221A70A2
:10BEC800D9E4464E96F8CC309BB9421C04BF414A8F
:10BED80010684FF00A030BBF43435843C6F820319C
:10BEE800C6F82001FCF7CEF90123C6F8240186F82C
:10BEF800CC306378042B3FF6BEACDFE803F0034494
:10BF080079A61A00FCF7BEF9D6F82431C01A002821
:10BF1800D6F82031B8BF4042984295BFD6F8C43011
:10BF2800002303F1FF3386F8CC3098BFC6F8C4303D
:10BF3800A1E4A07802F028FF38B9274A86F8CC0097
:10BF4800136823F01003136095E4D6F82031A3B1E9
:10BF5800FCF798F9D6F82431C01A0028D6F8203111
:10BF6800B8BF4042984208D91B4A002386F8CC3013
:10BF7800136843F0100313607DE4D6F8C430013B26
:10BF8800C6F8C43077E40F21A078FCF7F2FF10F070
:10BF9800010708D0104A002386F8CC30136823F034
:10BFA8001003136067E4D6F82031DBB1FCF76AF9B7
:10BFB800D6F82431C01A0028D6F82031B8BF40423C
:10BFC80098420FD9044A86F8CC70136843F01003DE
:10BFD800136050E4D00D0020780D0020D000002020
:10BFE8003E0D0020D6F8C430013BC6F8C43042E408
:10BFF8000F21A078FCF7BDFF10F0800708D0B14AE8
:10C00800002386F8CC30136823F01003136032E461
:10C01800D6F820319BB1FCF735F9D6F82431C01A8F
:10C028000028D6F82031B8BF4042984207D9A54A1F
:10C0380086F8CC70136843F0100313601BE4D6F83D
:10C04800C430013BC6F8C43015E40F21A078FCF7D2
:10C0580090FF10F4807708D09A4A002386F8CC30F5
:10C06800136823F01003136005E4D6F82031A3B158
:10C07800FCF708F9D6F82431C01A0028D6F8203180
:10C08800B8BF4042984208D98E4A86F8CC701368E7
:10C0980043F010031360FFF7EEBBD6F8C430013B42
:10C0A800C6F8C430FFF7E7BB874B002283F8C020EF
:10C0B800FFF7E1BB6378142B3FF664ADA278AAB909
:10C0C800824A8349927E41F82300002A3FF4D3AB89
:10C0D800002B3FF4D0AB03F285108000A0F214636C
:10C0E80004221944FCF7CEFDFFF7C5BBFF2A7FF4F5
:10C0F800EAAB774F73B94FF4C366A6F214613046C2
:10C10800042239440436FCF7BDFDB6F5CD6FF4D1F1
:10C11800FFF7B1BB03F285108000A0F2146104227E
:10C128003944FCF7AFFDFFF7A6BB1A6822F00802F6
:10C138001A60FFF7A0BBFF2B7FF4C5AB644F70B943
:10C148004FF4C366A6F2146130460422394404361B
:10C15800FCF7E2FDB6F5CD6FF4D1FFF78CBB00F22A
:10C1680085108000A0F2146104223944FCF7D4FD44
:10C17800FFF781BB6678142E3FF604ADA078534FC5
:10C1880010F0800F1AD0C30706D521210020FCF734
:10C19800F0FE4F4B43F82600BB7E002B3FF46BAB01
:10C1A800607800283FF467AB00F2851049498000A9
:10C1B80004220144FCF766FDFFF75DBB00287FF40D
:10C1C80082AB2121FCF7D5FE4149BB7E41F8260010
:10C1D800002B3FF450AB6378002B3FF44CABA078B6
:10C1E8001E1803F285131844042201EB860180000F
:10C1F800FCF748FDFFF73FBB6278374B0A2A0CD89B
:10C20800DFE802F006151A1F252D32373C4145009C
:10C2180032491A6809680A441A601A68294B002AC0
:10C228003AD11A6842F008021A60FFF724BB2B497A
:10C238001A680968521AEFE7284A196812684A43C7
:10C24800EAE726491A68096892FBF1F2E4E7234A0B
:10C258001868116890FBF1F201FB1202DCE71F4934
:10C268001A6809680A40D7E71C491A6809680A4326
:10C27800D2E71A491A6809684A40CDE717490A6897
:10C28800D2430A60C9E71968144A1160C5E7134A1E
:10C29800196810681860F8E71A6822F008021A602E
:10C2A800FFF7E9BA0C4B1B68C4F80330FEF706FB2E
:10C2B800FFF7E1BA084B1B68C4F80330FDF7C2FD6D
:10C2C800FFF7D9BA780D0020D00000200400002024
:10C2D8007C0D002068070020D00D0020EC0D002008
:10C2E800BA4A136803F00F031360FFF7C4BAB74ADA
:10C2F800136823F010031360FFF7BDBAB34A13683D
:10C3080023F020031360FFF7B6BAB04A136823F08E
:10C3180040031360FFF7AFBAAC4A136823F08003F9
:10C328001360FFF7A8BAA94A136823F4807313604F
:10C33800FFF7A1BA62782E2A3FF624ACA44B03EB90
:10C3480082035860FFF797BAA14BA24AD3F8281185
:10C358001160A14AD3F82C111160D3F83021C3F829
:10C36800C4209A4AD3F834111160D3F8382183F8DD
:10C37800CC20D3F83C21C3F82421D3F84021C3F8BA
:10C388002021964993F84421885C08B101208854FB
:10C3980000225A70FFF76FBAA378002B7FF493AA94
:10C3A8006378142B3FF6EEAB8A4A11688C4A42F840
:10C3B8002310FFF760BAFF283FF75DAA63780B2BBD
:10C3C80000F29380DFE803F006111C2733414C5735
:10C3D800626B737F834BA17853F8200053F82120B8
:10C3E800024443F82120FFF746BA7E4BA17853F860
:10C3F800200053F82120121A43F82120FFF73BBAF6
:10C40800784BA17853F8202053F82160724343F801
:10C418002120FFF730BA734BA17853F8200053F866
:10C42800212092FBF0F243F82120FFF724BA6D4B4C
:10C43800A17853F8200053F8216096FBF0F200FB36
:10C44800126243F82120FFF716BA664BA17853F819
:10C45800200053F82120024043F82120FFF70BBAAF
:10C46800604BA17853F8200053F82120024343F889
:10C478002120FFF700BA5B4BA17853F8200053F84E
:10C488002120424043F82120FFF7F5B9554AA17809
:10C4980052F82030DB4342F82130FFF7ECB9514B1A
:10C4A800A27853F8201043F82210FFF7E4B94D4B57
:10C4B800A27853F8206053F8221043F8226043F81A
:10C4C8002010FFF7D8B9474BA27853F8222053F829
:10C4D80020309A4240F341823C4A136823F0030318
:10C4E80043F004031360FFF7C6B903232B70FFF76B
:10C4F800C2B9A1783B4A374852F821300068034452
:10C5080042F82130FFF7B7B9A178364A314852F8D6
:10C51800213000681B1A42F82130FFF7ACB9A17826
:10C52800304A2C4B52F821001B68434342F8213013
:10C53800FFF7A1B9A1782B4A264852F821300068A4
:10C5480093FBF0F342F82130FFF795B9A178254A1B
:10C55800204B52F82160186896FBF0F300FB136338
:10C5680042F82130FFF787B9A1781E4A194852F8D6
:10C5780021300068034042F82130FFF77CB9A178E8
:10C58800184A144852F821300068034342F8213011
:10C59800FFF771B9A178134A0E4852F821300068A4
:10C5A800434042F82130FFF766B90A4BA1781B686F
:10C5B8000C4ADB4342F82130FFF75DB9054BA278FE
:10C5C8001968084B43F82210FFF755B9780D002079
:10C5D800D0000020D00D0020EC0D00203E0D0020E2
:10C5E8007C0D0020F00D0020A1789B4A9B4B52F84F
:10C5F80021001E6842F821601860FFF73CB9964B8D
:10C60800A27853F82220954B1B6862E703232B700E
:10C61800FFF731B96278914B91490B2A78D8DFE856
:10C6280002F006161D242C363D444B51565FA07867
:10C63800894A52F82020186802441A601B68002BA7
:10C6480069D10B6843F008030B60FFF714B9A678AB
:10C6580081481A6850F82600121AEEE77E4AA07838
:10C6680052F820001A684243E7E7A6787A481A6821
:10C6780050F8260092FBF0F2DFE7774AA0781E68B0
:10C6880052F8200096FBF0F200FB1262D5E7A07882
:10C69800714A52F8202018680240CEE7A0786E4A06
:10C6A80052F8202018680243C7E7A0786A4A52F86F
:10C6B800202018684240C0E7A078674A52F8202036
:10C6C800D243BAE7A078644A52F82020B5E7A078A8
:10C6D800614A1F6852F820601E6042F82070ADE77A
:10C6E8005D4AA07852F820001A6890420A6805DA74
:10C6F80022F0030242F004020A609FE70BBF22F017
:10C70800060222F0050242F0010242F00202F3E7BB
:10C7180003222A7092E70B6823F008030B60FFF7E7
:10C72800AAB863780B2B00F28680DFE803F00611C5
:10C738001C2733414C57626B737EA178464A49489F
:10C7480052F821300068034442F82130FFF793B8CB
:10C75800A178414A434852F8213000681B1A42F830
:10C768002130FFF788B8A1783B4A3E4B52F82100A8
:10C778001B68434342F82130FFF77DB8A178364A59
:10C78800384852F82130006893FBF0F342F8213022
:10C79800FFF771B8A178304A324B52F82160186817
:10C7A80096FBF0F300FB136342F82130FFF763B800
:10C7B800A178294A2B4852F821300068034042F8F2
:10C7C8002130FFF758B8A178234A264852F821307B
:10C7D8000068034342F82130FFF74DB8A1781E4A9C
:10C7E800204852F821300068434042F82130FFF7D2
:10C7F80042B81C4BA1781B68174ADB4342F821302A
:10C80800FFF739B8174BA2781968134B43F8221071
:10C81800FFF731B8A178104A124B52F821001E6870
:10C8280042F821601860FFF726B80B4BA27853F83E
:10C8380022200C4BE8E603232B70FFF71CB8637823
:10C848000B2B00F29880DFE803F00F19232D3845F1
:10C858004F59636C747F00BFF00D0020D00D00208D
:10C86800780D0020EC0D0020B94AA178B94B53F897
:10C87800213011680B441360FEF7FDBFB44AA0785D
:10C88800B449136851F820105B1A1360FEF7F3BF20
:10C89800AF4AB04BA17853F8211013684B4313608B
:10C8A800FEF7E9BFAA4AA078AA49136851F82010F0
:10C8B80093FBF1F31360FEF7DEBFA54AA54BA17801
:10C8C800106853F8211090FBF1F301FB1303136078
:10C8D800FEF7D1BF9E4AA1789E4B53F821301168CC
:10C8E8000B401360FEF7C7BF994AA178994B53F8DC
:10C8F800213011680B431360FEF7BDBF944AA1783D
:10C90800944B53F8213011684B401360FEF7B3BFC6
:10C91800A278904B53F822308D4ADB431360FEF720
:10C92800AABF8C4BA27853F82220894B1A60FEF7D5
:10C93800A2BFA178874A864B52F821001E6842F8A8
:10C9480021601860FEF797BF824BA27853F8222027
:10C958007F4B1B689A42FFF6BFAD7F4A13680BBF37
:10C9680023F0060323F0050343F0010343F0020319
:10C978001360FEF780BF03232B70FEF77CBFA178FE
:10C98800744A52F82130184442F82100FEF773BF68
:10C99800A178704A52F82130181A42F82100FEF79F
:10C9A8006ABFA1786B4A52F82130584342F82100F7
:10C9B800FEF761BFA178674A52F8213093FBF0F087
:10C9C80042F82100FEF757BFA178624A52F8216069
:10C9D80096FBF0F300FB136042F82100FEF74BBF13
:10C9E800A1785C4A52F82130184042F82100FEF73D
:10C9F80042BFA178574A52F82130184342F8210023
:10CA0800FEF739BFA178534A52F82130584042F80E
:10CA18002100FEF730BFA1784E4A52F82130DB439F
:10CA280042F82130FEF727BFA2784A4B43F822008C
:10CA3800FEF721BFA278474B53F8223098428AE785
:10CA480003232B70FEF717BF444B1B68C4F8033051
:10CA5800FDF74CFCFEF70FBF61783E4A52F82130D3
:10CA6800013B002B42F821307EF705AF3C4BC3F861
:10CA7800C400FEF700BF394B1B68C4F80330FDF74C
:10CA8800DDFBFEF7F8BE324B1B68FF2B3EF6F3AE1C
:10CA9800304A42F82300FEF7EEBE2D4B1B68FF2BF1
:10CAA8003EF6E9AE2B4A52F823202C4B6A601A60F6
:10CAB800294B2AB91A6842F008021A60FEF7DBBE51
:10CAC8001A6822F008021A60FEF7D5BE204B1B68D0
:10CAD800FF2B3EF6D0AE214A11681E4A42F82310B9
:10CAE800FEF7C9BE1C4909680F077EF5C4AE511C84
:10CAF80003EB8202C3F8C810D3F8C410C2F80011BF
:10CB0800C3F8C400FEF7B7BE134909680E073EF51F
:10CB1800B2AE511C03EB8202C3F8C810D3F8C4109C
:10CB2800C2F80011C3F8C400FEF7A5BE0A49096897
:10CB3800C9077EF5A0AE511C03EB8202C3F8C810EA
:10CB4800D3F8C410C2F80011C3F8C400FEF793BEAE
:10CB5800EC0D0020F00D0020780D0020D00D0020F5
:10CB6800D0000020CA490968CF073EF584AE511CA1
:10CB780003EB8202C3F8C810D3F8C410C2F800113E
:10CB8800C3F8C400FEF777BEC14909684E077EF5B1
:10CB980072AE511C03EB8202C3F8C810D3F8C4105C
:10CBA800C2F80011C3F8C400FEF765BEB8490968A9
:10CBB80011F0050F3EF45FAE511C03EB8202C3F87F
:10CBC800C810D3F8C410C2F80011C3F8C400FEF7A7
:10CBD80052BEAF49096889077EF54DAE511C03EB7B
:10CBE8008202C3F8C810D3F8C410C2F80011C3F801
:10CBF800C400FEF740BEA64909688F073EF43BAE65
:10CC0800511C03EB8202C3F8C810D3F8C410C2F851
:10CC18000011C3F8C400FEF72EBE9D490968CE0670
:10CC28007EF529AE511C03EB8202C3F8C810D3F875
:10CC3800C410C2F80011C3F8C400FEF71CBE944922
:10CC4800096889067EF517AE511C03EB8202C3F80A
:10CC5800C810D3F8C410C2F80011C3F8C400FEF716
:10CC68000ABE8B4909684F067EF505AE511C03EBD9
:10CC78008202C3F8C810D3F8C410C2F80011C3F870
:10CC8800C400FEF7F8BD824909680E067EF5F3ADCB
:10CC9800511C03EB8202C3F8C810D3F8C410C2F8C1
:10CCA8000011C3F8C400FEF7E6BD79490968C90553
:10CCB8007EF5E1AD511C03EB8202C3F8C810D3F82E
:10CCC800C410C2F80011C3F8C400FEF7D4BD00F0C8
:10CCD800A3FDFEF7D0BD00F005FEFEF7CCBD00F0C9
:10CCE80002FEFEF7C8BD00F0FFFDFEF7C4BD00F070
:10CCF800FCFDFEF7C0BD00F0FAFDFEF7BCBD654BBC
:10CD0800002283F8C020FEF7B6BD63782BB1012B53
:10CD180009D003232B70FEF7AEBD5E4B012283F8CA
:10CD2800C020FEF7A8BDB0F55B7FBEF4CCAD594A74
:10CD380082F8C030C2F8C400FEF79DBD554B0222F0
:10CD480083F8C020FEF797BDFCF7C2FAFEF793BD43
:10CD5800137D9B070BD4B0F55B7FBEF4B4AD4D4B90
:10CD6800042283F8C020C3F84801FEF784BD0823D5
:10CD78002B70FEF780BD474B002283F8C020FEF7DA
:10CD88007ABD3B460022F2540133082BFBD133789D
:10CD98003372FEF770BD6378012B19D03E4905D375
:10CDA800022B1ED003232B70FEF765BD3B4B0122DF
:10CDB8001A703B4A8B7813703A4B19680023013973
:10CDC800013311F8010FD054082BF9D1FEF753BDE8
:10CDD8000522EA716B7162222623AA712B71FEF774
:10CDE8004ABD2E4B304801221A702D4A8B78137099
:10CDF800002301331918082B11F8091CD154F8D154
:10CE0800FEF739BD6378032B3EF635ADDFE803F056
:10CE180002101E231F4B93F8C020EA7193F8CC2010
:10CE2800D3F84831AA711A0A6A712B71FEF723BD2B
:10CE3800184B93F8C020EA7193F8CC20D3F8C4308B
:10CE4800AA711A0A6A712B71FEF715BD174B1B6878
:10CE58006B60FEF710BD164B1B686B60FEF70BBDD1
:10CE68006378002B7EF407ADA17800297EF403AD2A
:10CE780040F2D24398427EF4FEAC40F2FF70FBF7DA
:10CE8800ECFEFBF781FF0120FBF735FCFEF7F3BC56
:10CE9800780D0020D000002004000020D40D0020D0
:10CEA800D50D00200000002000800008D00D0020D3
:10CEB800EC0D00206278894B9AB91A70884AE37899
:10CEC8001370884A92F84C11874A117087490022DA
:10CED8000A7087490A70874A11780B431370FEF766
:10CEE800CABC0122E9E766782EB1012E13D00323CC
:10CEF8002B70FEF7C0BC0422694640F2FB70FBF7BA
:10CF08000BFF009BD4F803209A4206BF01236B60F5
:10CF18006E60FEF7B0BCA3782A2B07D104227649AD
:10CF280040F2FB70FBF7AEFEFEF7A5BC03232B70A7
:10CF3800FEF7A1BC6B4ED6F85011002206F5AA7375
:10CF48008A423EF498AC53F82270874202F10107F6
:10CF580020D103EB8703043B01398A4214D3C6F876
:10CF68005011FEF788BC5F4BD3F85021092A9DBFAA
:10CF7800511CC3F8501103EB8203092394BFC3F873
:10CF880054012B70FEF777BC53F8040F43F8040CD8
:10CF98000132E2E73A46D3E7524A0023C2F8503159
:10CFA800194602F5AA7242F8231001330A2BFAD166
:10CFB800FEF761BC0A236B60FEF75DBC03232B7090
:10CFC800FEF759BC6378072B44D8DFE803F0040C5C
:10CFD80011161B31393E494B98427EF474AC02F06D
:10CFE800F7FDFEF748BC02F0FBFD6860FEF743BCA6
:10CFF80002F002FE6860FEF73EBC02F003FE6860C5
:10D00800FEF739BCB0F5005FBEF65DAC400080B2FB
:10D0180002F0F5F900046860D4F80300400001301C
:10D0280080B202F0ECF96B6818436860FEF723BC25
:10D03800324B98427EF447AC02F0C2F9FEF71BBCB3
:10D0480002F012FB6860FEF716BC02F0F3FD6860A0
:10D05800FEF711BC03232B70FEF70DBC6378812B00
:10D068007EF409ACA378922B7EF405ACA379A32BAC
:10D078007EF401AC6379B42B7EF4FDAB2379C52B28
:10D088007EF4F9ABE378D62B7EF4F5AB1C4B4FF46A
:10D0980000629A6172B6FBF73BFB1A4B1A480026EE
:10D0A8001E60314604F0D5FE3146184804F0D1FE22
:10D0B800154804F029FE154804F026FE4FF0A0405C
:10D0C80003F01EFF124803F01BFF124806F0E1FFB1
:10D0D8003046FBF710FBFEF7CEBB00BFF00B00207D
:10D0E800100C0020D00000203A0D00200A0C00206F
:10D0F8006F0D0020F10B0020730D00204E61BC0065
:10D108000004004810E000E05800024058040240C3
:10D118000004005000040040F7B50F4C07460E46C7
:10D1280094E803008DE803000C49C1F803300C4B68
:10D138008A7000220F704E701A70FEF791F9094A32
:10D14800217882F8F8109DE80300636884E80300FA
:10D15800184603B0F0BD00BFE40D0020700D00209C
:10D16800DF0D0020D0000020F8B50420FBF7F6FB07
:10D17800013010D00420FBF7F1FBB0F5803F0ADB4B
:10D188000420FBF7EBFB80B2252804DD0B4F0025BC
:10D19800ECB23E5D06B9F8BD05342046FBF7DEFB70
:10D1A800FF2808D02046FBF7D9FB0022034631466A
:10D1B8000520FFF7B1FF0135EAE700BFD4580108A1
:10D1C800F7B504461F4A63781370A3785370E37861
:10D1D80093702379937163795371A3791A4D1371FD
:10D1E800E379D3700E4695E80300184B00221A70B5
:10D1F8008DE80300FEF734F9154B1A786F462B4675
:10D208009AB9327072702A78B2706A78F270EA79D4
:10D218003271AA7972716A79B2712A79F27197E8D2
:10D22800030083E8030003B0F0BD012AF7D10948E1
:10D23800721EF11D10F8014F02F8014F8A42F9D110
:10D24800EDE700BF700D0020E40D0020DF0D002089
:10D25800D40D0020D50D0020F0B5AC4BAC4C1B789C
:10D2680089B013B994F87D316BB1AA4B1B78063B92
:10D27800DBB2192B04D8A84A22FA03F3D90702D43F
:10D28800002384F84C3194F84C31A44D5A1E012ADD
:10D2980040F26281A24F3A7842B3A24BA24E1B7869
:10D2A800013B012B1FD8A14A317893688DF81830BB
:10D2B80080238DF819308A238DF81A3000238DF8D1
:10D2C8001B308DF81C308DF81D308DF81E108DF830
:10D2D800113007218DF8123004A8D3688DF810108A
:10D2E800059303F025FC002333703B70002384F87A
:10D2F8004C312B7084F87D3194F87C3113B10120C6
:10D30800FBF7F9F994F84D314BB194F87F31B3FA42
:10D3180083F35B0984F87F31002384F84D31684634
:10D3280003F056FC002800F056819DF80030062BCB
:10D3380040F25181774B9DF808201A709DF809201A
:10D348005A709DF80A209A709DF80B209A719DF8E2
:10D358000C205A719DF80D201A719DF80E20DA7074
:10D368009DF8013084F87E31704B019A1B699A420E
:10D3780004BF012384F87D31FAF784FF6C4B1860F1
:10D388006C4B00221A709DF8003094F8C020072BCF
:10D398000CBF0123022384F84C31531E012B664B2A
:10D3A80040F21781052A00F0148101221A7094F8BE
:10D3B800C030042B04D1574B19780A0640F1368146
:10D3C80094F84C21082A04D840F25113D340DF07BF
:10D3D80001D4FEF745F894F84C31092B74D1FAF7CB
:10D3E80051FFD4F8E830554DC01A00282A68B8BF54
:10D3F8004042904209D9524B1A78012A04BF0222AE
:10D408001A70FAF73FFFC4F8E800FAF73BFFD4F8C0
:10D41800EC306A68C01A0028B8BF4042904209D967
:10D42800474B5A78012A04BF02225A70FAF72AFF9A
:10D43800C4F8EC00FAF726FFD4F8F030AA68C01A4E
:10D448000028B8BF4042904209D93D4B9A78012A3A
:10D4580004BF02229A70FAF715FFC4F8F000237887
:10D4680093B3637883BB364A36481D46D15C02299C
:10D4780040F0D28050F823104E1C00F0CC80324A85
:10D4880084F844311268C4F82821304A1268C4F874
:10D498002C21D4F8C420C4F830212D4AC4F8C41073
:10D4A8001268C4F8342194F8CC20C4F83821002339
:10D4B800D4F82421C4F83C2184F8CC30D4F82021B5
:10D4C800C4F840210123637094F84C31092B06D12C
:10D4D80094F8C020022A04BF052284F8C020D4F89A
:10D4E8005021002A68D0092B66D194F8C030012B4E
:10D4F80062D1D4F8C4101748002350F823508D4245
:10D5080040F08F80052384F8C03055E0DE0D002000
:10D51800D0000020700D002011020002D40D002060
:10D528006F0D00203A0D00200A0C00200400002096
:10D53800300D0020E80B0020DF0D0020FC0C00203F
:10D548003E0D0020D4000020D00D0020EC0D00205E
:10D55800780D0020240200204949012BCA68019255
:10D5680014BF082307238DF800302A7894F87E31F9
:10D578008DF8013000238DF80230FAB98B688DF8E8
:10D588000830404B8DF80F2019788DF8091059781C
:10D598008DF80A10D9798DF80B1099798DF80C103F
:10D5A80059791B798DF80D108DF80E30684603F007
:10D5B800BFFA00287FF46EAE09B0F0BD012AF5D19C
:10D5C800314801330DEB0302195CD171082BF8D1F6
:10D5D800ECE70022EAE694F8C030013B012B3FF665
:10D5E800E6AED4F8C430B3F55B7F10D2FBF781F810
:10D5F80068B1D4F8C4002549431CC4F8C430FBF70B
:10D60800BCFB092384F84C310122214BCEE60023D0
:10D6180084F8C030CBE6D55401332F2B7FF426AFE6
:10D6280052E701339A427FF468AFC5E794F84C019A
:10D63800082804D840F25112C240D207BCD4D4F80A
:10D648004801104DD3F803306970B0F55B7F6B600B
:10D6580012D20E49FBF78AFB0C49D4F84801FBF7B4
:10D66800B5FB38B1D4F848310133C4F848316523E3
:10D678002B70A1E70723FBE707232B70002342E762
:10D6880004000020E40D0020D50D0020700D0020BE
:10D69800DF0D0020464A00232DE9F0411360454A7A
:10D6A800454C1360454AC4F8C4301360444AC4F872
:10D6B800C83084F8CC3023706370211D4FF0FF30E0
:10D6C8001D4641F82300D55401332F2BF9D12421CD
:10D6D8000020FBF74EFC3B4BC4F8D8001D703A4DB8
:10D6E8002B7EC3BB394BC4F8F430C4F8D4300020C7
:10D6F800C4F8FC30FCF758FF95F83F3013B9012304
:10D7080085F83F300020FDF727F895F83D3053BBEA
:10D718000123C4F8D030FFF727FD2D4A002319460E
:10D72800174642F823100133B3F5807FF9D1294D0C
:10D73800AB7EDBB9EB7E4BB32B7903F0EF02012A0A
:10D7480032D1012384F87F316B7D03B1012384F842
:10D75800C030BDE8F081204BC4F8F4301F4BC4F84A
:10D76800D4301F4BC3E74FF0FF33D2E7DFF87480A4
:10D778004FF4C366A6F214613046042241440436CD
:10D78800FBF7CAFAB6F5CD6FF4D1D3E74FF4A76625
:10D79800A6F5A7613046042239440436FBF7BCFAE3
:10D7A800B6F5C36FF4D1C7E7212BCAD00023C9E768
:10D7B800D00D0020EC0D0020D0000020780D0020B6
:10D7C8003E0D0020090C0020280C0020D5920008EE
:10D7D800F00D002004000020C5920008CD9200083A
:10D7E800C99200087C0D0020704710B5094CFAF763
:10D7F80049FD2368C01AB0F5FA7F09D94FF0904265
:10D80800938A9BB283F008039382FAF73BFD20606A
:10D8180010BD00BF5002002010B50F4B0F4C5A78B6
:10D82800042A15D8DFE802F003070A0D1000FAF7FA
:10D8380043FD606010BDFAF753FDFAE7FAF752FDB1
:10D84800F7E7FAF766FDF4E79878FBF745FBF0E7AA
:10D858000323237010BD00BF700D0020E40D0020CD
:10D8680038B51D4B9C781D4694BB5A782AB1012ABD
:10D878001A4D21D003232B7038BDD3F8030018B9F3
:10D88800BDE83840FAF768BF1046FAF76DFF70B187
:10D898005021A878FBF76DFB212102460446A878A1
:10D8A800FBF747FB22463721A878FBF742FBA8780D
:10D8B800BDE83840FAF748BF2046FAF755FF28B9BF
:10D8C800074B9C8A84F40064C4F3C0246C6038BDA0
:10D8D800024B04221A7038BD700D0020E40D0020A0
:10D8E800000400487047704770477047704770479A
:10D8F800054A135C02440033527818BF01230AB169
:10D9080043F00203184670475402002010B5184B24
:10D91800184C00201870587094F82430DA0704D591
:10D9280013F0080317D0FAF769FE94F82430980723
:10D9380005D5D9064FF0010011D5FAF75FFE94F826
:10D9480024305A0712D59B064FF002000AD5BDE8CD
:10D958001040FAF753BE1846FAF730FEE5E7FAF733
:10D968002DFEECE7BDE81040FAF728BE10BD00BF59
:10D978005402002004000020034B18448078431F01
:10D9880058425841704700BF5402002038B5054638
:10D998000C46A1B9FBF7EDFA214620F4E0722846BF
:10D9A800FBF7C7FA4C236B431B4AD35C9BB328464F
:10D9B8004FF000620721BDE83840FBF714BB002197
:10D9C800FBF7D7FA04F00303022B20F4E0721CD013
:10D9D800032B1DD0012B01D142F04002630748BF41
:10D9E80042F4807214F0080418BF42F40072002157
:10D9F8002846FBF79EFA002CD9D128464FF0006242
:10DA08000721BDE83840FBF7FCBA42F08002E5E7A1
:10DA180042F0C002E2E738BDAC0C002073B5144CEC
:10DA280023180646DB780D4623B94FF0C05207216C
:10DA3800FBF7E7FA0F4A4C2303FB062301229B7DE1
:10DA4800019285EAE572A2EBE572D2B20092062154
:10DA580000223046FBF74AFA002D04EB060304EBDC
:10DA68008604B4BF01220222DA70656002B070BD7C
:10DA780054020020AC0C0020184B1A1873B5D1784A
:10DA8800044641B303EB80030025D57007214FF00E
:10DA980080525D60FBF7A7FA4FF00062072120462D
:10DAA800FBF7AFFA4C230E4A6343D618D35C93B105
:10DAB80050212046FBF75DFA212102462046FBF75C
:10DAC80038FA327DB37D0192727D009206212A4692
:10DAD8002046FBF70BFA02B070BD00BF54020020CD
:10DAE800AC0C00202DE9F04FA94D2C7A87B005F138
:10DAF80009084CB9E0B2FAF7B2FD08F8040001349D
:10DB0800082CF7D101232B72DFF8A4A2A14F2724F8
:10DB180000264FF00209F0B2FAF7A1FD18F8063016
:10DB2800834216D0331D08F806005AF82330022B1A
:10DB38000AD0032B02D0012B0BD150B13B5D012B36
:10DB480008BF07F8049004E018B93A5D012A00D12B
:10DB58003B550136082E04F10104DCD18E4FFB69D8
:10DB680093B18E4C26787EB9FAF78CFB8C4B1B68E8
:10DB7800C01A0028FB69B8BF4042984204D9304611
:10DB8800FBF787FA012323703B6A93B1854C26780B
:10DB98007EB9FAF777FB844B1B68C01A00283B6AEA
:10DBA800B8BF4042984204D93046FBF772FA0123C5
:10DBB8002370687C7D4EFAF7F1FD2221687CFBF723
:10DBC800D8F90390687CFBF74BFA0F218146687CF3
:10DBD800FBF7CFF90490687C842303FB00631B697F
:10DBE80023B3039A002AB8BF5242002BB8BF5B4246
:10DBF800B3EB022F1ADA2B189B7C43B94FF08062E3
:10DC08000121FBF7F0F96B7C01222B449A7419F07F
:10DC1800010F1BD0687C5F4AC31CD15C012912D15B
:10DC28000221D1540121FBF728FA0FE02B189B7C25
:10DC3800002BECD04FF080620121FBF7E2F96B7CFE
:10DC480000222B44E2E7D35C002BEBD019F0005FF5
:10DC58000CD0687C4F4A00F10F03D15C012904BF46
:10DC68000221D1544FF00051FBF707FA19F4006F65
:10DC780006D0039B23B94FF40061687CFBF7FDF9DC
:10DC880019F4805F06D0039B23B94FF48051687C58
:10DC9800FBF7F3F919F4005F06D0039B23B94FF49F
:10DCA8000051687CFBF7E9F919F4804F06D0039B13
:10DCB80023B94FF48041687CFBF7DFF919F0020FB4
:10DCC8000BD0687C334A00F10903D15C012904BFF9
:10DCD8000221D1540221FBF7D0F9049B13F08000F4
:10DCE8006B7C4FF00101E97405EB03026AD0107DEB
:10DCF80078B911752E4A1A44127B12F0010F08D018
:10DD080002211B2211FB0323224AD05C012808BFF1
:10DD1800D154049B13F480716B7C05EB03025BD038
:10DD2800517D81B901215175214A1A44527B12F063
:10DD3800010F08D00E33174A12F81310012904BF37
:10DD4800022102F81310FAF79DFAAB69C01A0028ED
:10DD5800B8BF40420A2840F3AB80687C154B164A8E
:10DD68001649DFF85C800344024401EB800102F0AD
:10DD7800DAFB6C7C2B199A784C23052A63D8DFE8E8
:10DD880012F0350099010502B102D6022C0300BF3A
:10DD9800540200203E0D002004000020390D002010
:10DDA800340D0020E80B0020300D0020280C002046
:10DDB800FC0C0020260C0020F80B0020140C00207E
:10DDC800AC0C0020117D0029A3D01075B14A1A446B
:10DDD800127B12F0020F92E7507D0028B3D05175E4
:10DDE800AC4A1A44527B12F0020FA2E703FB04FA72
:10DDF80008EB0A0B18F80A302BB3204600F0C4FFD2
:10DE080008BB9BF84930022B06D1842303FB04632B
:10DE18001B7A093B012B14D81021204602F080F808
:10DE2800842303FB046320F4F8525B7ADB0842EA9C
:10DE380003222046102102F047F82C440123A37046
:10DE480001E008F80A00687C00F080FC687C842304
:10DE580003FB00635B7EC3B15021FBF78AF86B7C40
:10DE68004C249A0004FB0384A918E46B096AA1EB0B
:10DE7800040E86452B4403D82144884240F205838A
:10DE88002A44012183F8241010626C7C4C236343DC
:10DE980018F803303BB12B19DB78012B00F0F9821D
:10DEA800022B00F0028300236B74FAF7EBF9A861E8
:10DEB80095F811A0BAF1000F16D1774C23789BB1D1
:10DEC800039BDFF8E881002B4FF032015046C0F287
:10DED8000183FBF74EF8D8F800200244322150465F
:10DEE800FBF727F80023237097F92430002B80F2E2
:10DEF800F7826A4B1B8A4FF0000897F82430DC073A
:10DF08002CD56C7C2B5D4BB3DFF8A4A1B8F1000FC6
:10DF180003D195F82530012B03D01AF80430D8071F
:10DF28001CD5002320462B55FFF7E2FC30B95C4B8B
:10DF3800122153F824202046FAF7FBFF6A7C97F851
:10DF480024001AF8023010F0080023F001030AF840
:10DF5800023000F0CA820020FAF750FB97F824300C
:10DF6800990713D56A7C842101FB026103F0100331
:10DF7800497E002940F0BC82049AD20740F1BE8253
:10DF8800002B00F0BE820120FAF718FB97F8243026
:10DF98005B0740F145836C7C2B195B78002B00F004
:10DFA800B482DFF80C91B8F1000F03D195F8253051
:10DFB800012B03D019F804305E0744D54C23394EA1
:10DFC8006343F35C43B950212046FAF7D2FF21217D
:10DFD80002462046FAF7ADFF6C7C19F8043023F0AE
:10DFE800040309F804302B19002220465A70FFF761
:10DFF8007FFC30B92A4B122153F824202046FAF727
:10E0080098FF687C4C234343F35C8BB1FAF7ACFB75
:10E0180070B15021687CFAF7ACFF21210246044612
:10E02800687CFAF786FF22463721687CFAF781FF79
:10E03800687CFAF789FB97F82430980640F1E58266
:10E048000220FAF7DBFABB7D85F82580002B00F06B
:10E05800458395F82640002C00F00B83012C00F036
:10E068001783114C95F826202178914200F03683C9
:10E07800EB7C002B00F03283BB7D012B40F0148336
:10E08800002A00F01783687CFBF703F8FAF772FBA5
:10E0980021E300BFFC0C00206D0D002000080048A3
:10E0A8001C0C0020AC0C002044000020E40B0020D5
:10E0B8002C0D00204FF04C0A0AFB048A002205218F
:10E0C8002046FAF736FF9AF814209AF8163001928B
:10E0D8009AF815200092062100222046FAF706FF3A
:10E0E800842303FB04639AF849A0DB6973B1BAF18E
:10E0F800010F12D019D3BAF1020F7FF4A4AE204653
:10E108002C4400F031FE84F802A09CE6BAF1000F1E
:10E118000BD0BAF1010F7FF496AEFAF7B3F805EB1E
:10E1280084032C44D861022389E679212046FAF732
:10E1380020FF7F2816DCC0F1800A20460422202117
:10E14800FAF7F7FEDD4A20462421FAF7F2FE2121EC
:10E158002046FAF70EFF372100EB0A022046FAF7AD
:10E16800E8FEDAE7B0F5C07F02DAC0F5C07AE4E786
:10E17800B0F5207F02DAC0F5207ADEE7B0F5607FDF
:10E18800B4BFC0F5607AC0F5906AD6E7842303FB74
:10E198000463D3F81CB04C23BBF1000F71D003FB10
:10E1A80004FB08EB0B0393F849A0BAF1010F2FD039
:10E1B800C0F08580BAF1020F7FF445AE204600F02A
:10E1C800E3FD8246002851D1024620212046FAF775
:10E1D800B0FE524624212046FAF7ABFE79212046AC
:10E1E800FAF7C7FE2121824602462046FAF7A1FE29
:10E1F800524637212046FAF79CFE524650212046C7
:10E20800FAF797FEAE4B01221A552C44032316E663
:10E21800FAF738F805EB8403DB69C01A0028B8BFA1
:10E22800404264287FF70FAE002220212046FAF7EB
:10E2380080FE002224212046FAF77BFE7921204621
:10E24800FAF797FE2121834602462046FAF771FE27
:10E258005A4637212046FAF76CFE5A465021204686
:10E26800FAF767FE964B03F804A0CEE718F80B30D0
:10E27800002B7FF4E8AD204600F07EFD2C440523FA
:10E28800DDE503FB048393F849A0BAF1000F16D02B
:10E29800BAF1010F7FF4D7ADF9F7F4FF05EB84036A
:10E2A800DB69C01A0028B8BF404264287FF7CBADAD
:10E2B8005A4620212046FAF73CFE5A46BAE7F9F7B3
:10E2C800E1FF05EB8403DB69C01A0028B8BF4042B0
:10E2D800B0F57A7F7FF7B7AD21212046FAF749FEDE
:10E2E80002468BE74FF0C05207212046FAF789FE15
:10E2F8004C2303FB048393F84930012B10D009D336
:10E30800022B12D0F9F7BEFF05EB84032C44D86129
:10E31800042394E56B4A07212046FAF764FEF1E7E7
:10E32800694A07212046FAF75EFE674AF3E7F9F7DC
:10E33800A9FF05EB8403DB69C01A0028B8BF404277
:10E34800B0F57A7F7FF77FAD4FF01942072120465D
:10E35800FAF757FE842303FB04635B7E0BB11B07AC
:10E3680038D54FF0206207212046FAF73CFE80227C
:10E3780005212046FAF7DDFD4FF000720121204605
:10E38800FAF731FE59212046FAF7F3FD4FF04C0A0F
:10E398000AFB048A4D4BCAF810000022502120467F
:10E3A80043F824200592FAF7E4FD2121834620460C
:10E3B800FAF7DFFD464B059AABEB000043F8240063
:10E3C8009AF84930022B7FF459AF59212046FAF7C1
:10E3D800B0FD53E74FF00072C5E7634318F803B088
:10E3E800BBF1000F7FF42FAD20464FF0840AFFF7F2
:10E3F80043FB0AFB046A4FF0046207212046FAF740
:10E4080000FE032205212046FAF793FD9AF81630FC
:10E418009AF80A2001939AF80930009306215B467E
:10E428002046FAF763FD1021204601F079FD1021FE
:10E4380040F4F852204601F047FD2B1983F802B04A
:10E448009AF81730FBB9012220212046FAF771FD0E
:10E45800002224212046FAF76CFD21212046FAF7F4
:10E4680088FD1A4B53F824202121821A2046FAF7F6
:10E4780060FD4FF0007201212046FAF7C2FD104BF3
:10E4880001221A55DFE40222DEE7002283F8242065
:10E49800FBE450212046FAF76CFDA0F5C332A03A00
:10E4A80021212046FAF745FDFDE450212046FAF7E0
:10E4B80060FD00F5C332A032F2E700BF40420F0012
:10E4C800090C00200000408100004080F40B00206F
:10E4D8000C0C0020FAF74DFDD8F80020821AFDE454
:10E4E8000020FAF7BCF8804607E5FAF767F835E543
:10E4F8002A4492F82420002A3FF442AD002B3FF42E
:10E5080042AD0120FAF77AF840E5FAF73FF900281A
:10E518003FF499AD687CFAF727F900287FF493ADAA
:10E52800687C842303FB00631A6AA2B3049A51042B
:10E5380031D593F83C30012B1DD8FAF7AAFD687C39
:10E54800684A4C234343D35C5BB15021FAF711FD71
:10E558006B7C654A52F823202121821A1846FAF763
:10E56800E8FC687C842303FB006393F83C30012BB0
:10E5780001D1FAF7F1F8687C2B1801225A701221A0
:10E588000022FAF7D6FC97F824309A064FF00200DA
:10E598003FD5FAF713F8687C842404FB00635A6AB1
:10E5A800002A3FF450ADDB69DFF84491A3BB01F0CA
:10E5B8002FFB6B7C039A04FB0364801A0028626AB1
:10E5C800B8BF404290427FF63EAD94F83C20012A05
:10E5D80002D81846FAF75DFD687C842303FB0066C1
:10E5E80096F83C30012B01D1FAF7B6F899F81100EA
:10E5F80009EB000301225A7012210022FAF799FC54
:10E6080097F824309B067FF51BAD0220F9F7D6FF5B
:10E6180019E5F9F7F3FFBEE76621FAF7AAFCC8E7A0
:10E62800687C842303FB0066336A002B3FF40BAD40
:10E6380019F4802F3FF407ADFAF72BFD5021687CC1
:10E64800FAF797FC6B7C284A52F823202121821A7A
:10E658001846FAF76EFC4FF48021687CFAF70DFD36
:10E668006B7C224A1533D15C012904BF0221D154A5
:10E67800E9E40120F9F7F3FF012806D1AB6A642B1E
:10E6880010D9AC6285F82600EBE40023AB62E8E41D
:10E698002046F9F7E4FF0028F7D1AB6A642B01D9CB
:10E6A800A862EFE70133F1E7022B7FF4ECAC012A13
:10E6B8007FF4E9AC5021687CFAF75BFC2121024623
:10E6C8000646687CFAF735FC32463721687CFAF74B
:10E6D80030FCFAF755F895F82630237007B0BDE8F6
:10E6E800F08F00BFAC0C00200C0C00203E0D002069
:10E6F80054020020024B03EB80004068704700BFC3
:10E708005402002038B5104A842303FB0023044632
:10E71800DB7D0D46B3B901222021FAF70AFC204619
:10E728004FF080520721FAF75EFC20464FF0006256
:10E738000721FAF766FC2A4620462421BDE838401E
:10E74800FAF7F7BB0222E7E7280C00202DE9F0478B
:10E758000F210446FAF70DFCC54984236343CD18FD
:10E7680088462A7A6F6812F0400F16BF58F80330AF
:10E7780058F80390C3F10009BE4B4FEA10211B8AD9
:10E788004FEAD0100FBF00F0010A01F0010A00F0B3
:10E7980001007F4208BF01F0010002F03F0612F0BD
:10E7A800800F18BF83F400530A2EC3F3403300F2DE
:10E7B800BB810122B24012F4C06F40F02A8212F4E9
:10E7C800F07F40F03F8112F01E0F00F0AD81AA4D9E
:10E7D8002B5D013B0E2B00F2A781DFE813F00F0041
:10E7E8001E002D0039004900530062007000B1007E
:10E7F800E700ED00A5012B011102B402012120461A
:10E80800FAF7B7FB05EB840301225860023E9B4BE5
:10E8180096421A551AD8022332E005EB84035A6847
:10E8280042F0020201212046FAF783FB49462046BE
:10E83800FFF768FF032323E0002800F075812121FA
:10E848002046FAF796FB8E4B43F82400042317E082
:10E8580005EB84035A6842F0010201212046FAF7C9
:10E8680068FBC9F100012046FFF74CFF052307E0CC
:10E87800BAF1000F00F058812046FAF70AFC062387
:10E888002B5551E105EB840301215A68204622F0FB
:10E898000302FAF74EFB39462046FFF733FF0723FA
:10E8A800EEE7BAF1000F40F03F8151462046FFF7EE
:10E8B80029FF79422046FFF725FF0823E0E7BAF150
:10E8C800000F00F0318121212046FAF752FB002188
:10E8D80006462046FFF716FF694A52F824309B1B6C
:10E8E80042F8243005EB840301215A68204622F0BF
:10E8F8000302FAF71EFB842303FB048898F81730F9
:10E90800E3B9052220212046FAF713FB3A462421D1
:10E918002046FAF70EFB4FF0805207212046FAF7FF
:10E9280070FB4FF0006207212046FAF75CFB324685
:10E9380037212046FAF7FDFA0923A1E70622E1E785
:10E948000F212046FAF715FBC00740F1ED80212181
:10E958002046FAF70EFB4B4B002118602046FFF7C4
:10E96800D1FE4C236343484A12F80380B8F1000FE4
:10E9780009D1424637212046FAF7DBFA42462121DF
:10E988002046FAF7D6FA21212046FAF7F2FA3F4B49
:10E99800502143F824002046FAF7EBFA033E3C4B9B
:10E9A800012E43F824004BD87942D0E0BAF1000F89
:10E9B80000F0BA800B2363E7BAF1000F40F0B4808F
:10E9C80021212046FAF7D5FA514606462046FFF798
:10E9D80099FE022396FBF3F605EB840301215A689E
:10E9E800204622F00302FAF7A4FA842303FB0488E2
:10E9F80098F81730E3B9052220212046FAF799FA4A
:10EA08003A4624212046FAF794FA4FF0805207211B
:10EA18002046FAF7F6FA4FF0006207212046FAF787
:10EA2800E2FA324637212046FAF783FA0D2327E720
:10EA38000622E1E70F212046FAF79BFAC10773D5B2
:10EA48000E231DE70C4D2A5D013A0E2A6CD8DFE82B
:10EA580012F02100310042004E005F006B006D0093
:10EA68006B006B0095009F0083004801D7007A0176
:10EA7800280C00200008004880020020090C002013
:10EA8800EC0B0020F80C0020AC0C0020F40B00204C
:10EA98000C0C0020AE4B012120461955FAF769FAF3
:10EAA80005EB8403062E58603FF4B5AE082E7FF4BC
:10EAB800CDAEB0E6062E05D105EB84035A6822F0E8
:10EAC8000302ADE6082E7FF4B1AE05EB84035A6865
:10EAD80022F00302A6E6721F012A05D820B1062EED
:10EAE8003FF4B4AE0F23CBE6F3B10C23C8E6052EF2
:10EAF80005D105EB84035A6822F00302ABE6072E22
:10EB08007FF4AFAE05EB84035A6822F00302A4E653
:10EB1800721F012A05D8BAF1000F02D0052EE1D1E3
:10EB280079E6002B7FF4BBAEBDE8F087002BFBD164
:10EB3800073E012E0AD905EB840301215A6822F009
:10EB4800030242F002022046FAF7F3F9394620465A
:10EB5800FFF7D8FD0A2393E6002BE5D1073E012EE7
:10EB68007FF622AF05EB840301215A6822F00302E5
:10EB780042F001022046FAF7DCF915E7002BD3D062
:10EB880021212046FAF7F5F905EB8403986011E78F
:10EB9800002BC9D1212120464FEA8409FAF7E9F967
:10EBA80005EB090306465A68012122F003022046B4
:10EBB800FAF7BFF9842303FB048898F81730EBB9F8
:10EBC800052220212046FAF7B4F93A4624212046A6
:10EBD800FAF7AFF94FF0805207212046FAF711FAF9
:10EBE8004FF0006220460721FAF7FDF905EB09030B
:10EBF80002229868304490FBF2F213E70622E0E71D
:10EC080005EB840301215A682046FAF792F900239C
:10EC180036E6504D2B5D013B0E2B85D801A252F8EC
:10EC280023F000BF69EC000831EB000831EB000865
:10EC380031EB000831EB000831EB000831EB00083C
:10EC480031EB000831EB00088DEC000831EB0008CF
:10EC580031EB0008EBEC000817EC00084FED00085A
:10EC68003B4B01224FF4102120461A55FAF705FABA
:10EC780040F6682207212046FAF7B5F9092E7FF4F5
:10EC880093AE63E70E212046FAF773F9C2037FF5C6
:10EC98004BAF00212046FFF735FD842303FB048892
:10ECA80098F81730DBB9052220212046FAF741F9F8
:10ECB8003A4624212046FAF73CF94FF080520721C2
:10ECC8002046FAF79EF94FF0006207212046FAF72E
:10ECD8008AF936212046FAF74CF90246A2E60622BE
:10ECE800E2E70F212046FAF744F9C3077FF51CAF86
:10ECF8000E23212120462B55FAF73BF9164B00210C
:10ED080018602046FFF7FEFC4C236343134AD55C8A
:10ED18004DB92A4637212046FAF70BF92A46212110
:10ED28002046FAF706F921212046FAF722F90C4B7A
:10ED3800502143F824002046FAF71BF9094B43F801
:10ED48002400BDE8F08700212046FFF7DBFC77E6CA
:10ED5800090C002080020020F80C0020AC0C0020D8
:10ED6800F40B00200C0C0020024B1A5C0AB901229B
:10ED78001A54704780020020024B1A5C0AB10F2215
:10ED88001A54704780020020014B185C704700BF7E
:10ED980080020020F8B599422DED028B04460D46FD
:10EDA800164632DA5B1A07EE903A331B07EE103A32
:10EDB800F8EEE77AB8EEC77A274B87EE878A2746B8
:10EDC80093ED007ADFED257AB8EEC77A68EE277AF8
:10EDD800F4EEC77AF1EE10FA44BFBDEEE77A17EE0B
:10EDE800102A93ED017A48BF1A60B8EEC77AF4EE9C
:10EDF800C77AF1EE10FAC4BFFDEEE77AC3ED017AE7
:10EE0800B74207DBBDEC028BF8BDFBDDC1F58042E4
:10EE18001344C8E73B1B07EE103A07EE905AB8EECA
:10EE2800C77AF8EEE77AB8B2E8EE077A00F18060C0
:10EE380000F5E0304000FDEEE77A013717EE901A52
:10EE48004B42C3F30D03C1F30D0158BF594289B2B8
:10EE580003F028FAD4E700BF8C02002000007A44AF
:10EE680073B5F9F70FFA0446F9F70CFA001B0028F6
:10EE7800B8BF40426328F7DD4FF4E070F9F732FF7E
:10EE8800044640F2C110F9F72DFF05464FF4E17032
:10EE9800F9F728FF064640F2C310F9F723FF2106C9
:10EEA80005D42A0603D4330601D41F2803D9002029
:10EEB800064605460446009033462A462146002069
:10EEC800F9F7C0FC02B070BD4FF090434FF48012C8
:10EED8009A610D4B4FF426429A811A89D007FCD5C6
:10EEE8009889002100049981074B20F07F421989F5
:10EEF800C907FCD54FF0904110208861988980B2ED
:10EF08001043800A704700BF003C00400C4B0022B1
:10EF180040211A7210465972D9601A615A6103EB7E
:10EF280042010132402A0883F9D14FF48042054951
:10EF3800C3F898200A684968521AC3F89C20704799
:10EF48008C02002048000020024B03EB4000008B9D
:10EF580000B270478C020020684620F007018D46F9
:10EF680031B59D4C00226021204604F0B9FF4FF0D6
:10EF780090431022A1899A61984A92F8A000C0B2E1
:10EF88000128C1F30D01134600F0D88107D30228E8
:10EF98004FF0000300F0D48182F8A03018E192F815
:10EFA800A1201AB1C1F57F513F3189B28C4A107A3C
:10EFB800002800F0F880C3F8A410B3F8A81089B2AC
:10EFC800C3F8AC105969D3F8A40001445961D3F8C7
:10EFD800A410B1F5005F1969D3F8A4000144A8BFD3
:10EFE800A1F580411961197A0131C9B21972197AEA
:10EFF8003F2984BF00211972587AD968884280F263
:10F00800F380D3F8B010002940F0EE80597A01312E
:10F01800C9B25972197AD3F8A40003EB410100B2BE
:10F028000883D3F8A410B1F5805F05DBD3F8A410EA
:10F03800B1F5405FC0F23F811969587A91FBF0F150
:10F04800C3F8B810D3F8B8100029BEBFD3F8B81069
:10F0580001F58041C3F8B810D3F8B810D3F8B01050
:10F068000131C3F8B010D3F8B010402947D1117A54
:10F07800002944D00021C3F8B010D3F8B810D3F851
:10F08800BC00091AC3F8C010D3F8C010B1F5005F6E
:10F09800D3F8C01040F31181A1F58041C3F8C01026
:10F0A800D3F8C010C3F8C410D3F8C010DFED4D6A10
:10F0B8000029BEBFD3F8C0104942C3F8C01093ED71
:10F0C800307AB8EEC77AC6EE877AFDEEE77AC3EDF6
:10F0D800037AD9684029C4BF4021D960D868D1686B
:10F0E8008842BCBFD168D960D3F8B810C3F8BC1047
:10F0F800D3F8C4004FF474714143C3F8C810587A68
:10F108001169884280F21281D3F8C4505169D3F84A
:10F118009840D3F8B800694391FBF4F10144C3F86F
:10F12800CC10D3F8C8005168884280F2CF8051686B
:10F13800D3F8C8004942814280F2C8800022C3F84F
:10F14800D020D3F8D020D3F8CC100A44C3F8CC2070
:10F15800D3F8CC205142C1F30D01C2F30D0258BFC0
:10F168004A42C3F8CC20D3F8CC20002A05DAD3F8D9
:10F17800CC2002F58042C3F8CC205A7A402A40F0CD
:10F18800D880D3F8CC20D3F8D410521A002AB8BFAC
:10F198005242022A00F3CD80D3F8D420C3F8CC2001
:10F1A800D3F8CC1089B293F8D82032B1B1F5804F9A
:10F1B8003CBFD3F8DC2032F81110A3F8A81093F85C
:10F1C800E0202AB193F8E020013AD2B283F8E02097
:10F1D800BDE8314085467047003001408C02002070
:10F1E8004800002000000043197A587A091AC3F829
:10F1F800B410D3F8B4100029BEBFD3F8B41040310E
:10F20800C3F8B4105969D3F8B40003EB4000008B7D
:10F2180000B2091A5961D3F8B41003EB4101098B04
:10F2280009B2B1F5005F1969D3F8B40003EB4000E7
:10F23800008B00B2A1EB0001A8BF01F58041196164
:10F24800587AD96888427FF7E5AED3F8B0108907B5
:10F258007FF4E0AE597A0139C9B25972197A587AED
:10F26800091AC3F8B410D3F8B4100029BEBFD3F8F4
:10F27800B4104031C3F8B4105969D3F8B40003EBA3
:10F288004000008B00B2091A5961D3F8B41003EB9F
:10F298004101098B09B2B1F5005F1969D3F8B400CF
:10F2A80003EB4000008B00B2A1EB0001A8BF01F501
:10F2B80080411961AEE65969BFE611F5005FBFF6F6
:10F2C800EFAED3F8C01001F58041E7E6D3F8C800E7
:10F2D8001168884201DD926931E71168D3F8C800E6
:10F2E8004942814202DD9269524228E7D3F8C800B8
:10F2F800516888420FDDD3F8C800116888420ADADD
:10F30800D3F8C81054689269D3F89C00091B4A4383
:10F3180092FBF0F213E79069D3F8C8405268D3F82B
:10F328009C102244424392FBF1F208E7D3F8B8203C
:10F3380021E7D3F8CC20C3F8D42031E702232BE609
:10F34800A2F8E21028E6684620F007018D4619B5B4
:10F358000121174805F070FBF0B101211448154C44
:10F3680005F074FB4FF090434FF480129A616021CE
:10F378000122204604F0B4FD0F4B93F8A030DBB215
:10F38800012B22460FD001D3022B05D10B4B9B7EBC
:10F3980033B947F6FE739381BDE819408546704737
:10F3A8004FF6FF73F7E74FF6FC73A381F4E700BF4E
:10F3B80000040040003001408C020020280C00208E
:10F3C80007B500214FF4E070F9F747FC002140F23F
:10F3D800C110F9F742FC00214FF4E170F9F73DFC48
:10F3E800002140F2C310F9F738FC002300931A46B5
:10F3F80019461846F9F726FA03B05DF804FBB0F58C
:10F40800804F3DBF034BD3F8DC3033F810004FF684
:10F41800FF7070478C020020824B834A30B501216F
:10F4280083F8A1101488C3F8DC204FF6FF708442DB
:10F4380093B01D4605D047F6FE74125B824240F039
:10F44800E780FFF7BDFF002404F1806000F5E0309D
:10F45800A1B24000013402F025FFB4F5804FF3D18A
:10F4680002F03EFE012385F8D830FFF74FFD6F4BC1
:10F4780001251D72F8F734FF002800F0CC80FFF753
:10F48800EFFC2946022003F0FDFD6948002404F042
:10F4980000FE4FF4616304A965480593ADF8104078
:10F4A800ADF81840ADF8124004F07CFE2A46294613
:10F4B8005F4805F0DCFA29465D4804F01CFF1D236F
:10F4C80003A88DF80C308DF80D508DF80E508DF87E
:10F4D8000F5003F017FB232303A88DF80C308DF889
:10F4E8000D408DF80E508DF80F5003F00BFB294698
:10F4F800284603F0AFFD4F4B08934F4B079310235B
:10F5080009934FF480630E934FF480730D93802317
:10F518000C9320230F9307A94FF4405347481093A7
:10F528001194ADF828500B9402F068FC2A46022189
:10F53800434804F0C1FC2946404802F08AFC0C23E9
:10F548000093C82204230A212046F9F768FD4FF0EA
:10F558000A1256212046F9F7ECFC4FF4FA725821AA
:10F568002046F9F7E6FC4FF4041207212046F9F784
:10F57800E0FC344A08212046F9F7DBFC4FF6FF721D
:10F5880068212046F9F7D5FC4FF440622146204611
:10F59800F9F7CFFC08212046F9F7EBFC2246692150
:10F5A8002046F9F7C6FC4FF6FF7268212046F9F7A6
:10F5B800C0FC4FF4674269212046F9F7BAFC0821DC
:10F5C8002046F9F7D6FC6A212046F9F7D2FC6B21D0
:10F5D8002046F9F7CEFC4FF4804254212046F9F733
:10F5E800A8FC224650212046F9F7A3FC164B4FF4FD
:10F5F800C8625A6483F8404083F841400622019467
:10F608000094402363212046F9F770FC13B030BD05
:10F6180083F8D81029E7FFF723FC0C4B4FF48042FE
:10F62800DA61F3E78C02002000800308480000201C
:10F6380000040040340300200C3800405800024009
:10F64800003800400D081010AC0C0020280C0020D9
:10F6580000B939E400207047024BB3F8E20080B2E9
:10F66800704700BF8C0200204FF480407047062985
:10F6780021D8DFE801F004080C1014181C000F4B07
:10F68800D3F8E40070470D4BD3F8E80070470B4BF4
:10F69800D3F8EC007047094BD3F8F0007047074BDC
:10F6A800D3F8F4007047054BD3F8F8007047034BC4
:10F6B800D3F8FC0070470020704700BF8C02002080
:10F6C80000280ADD054B1A68904206DC58601A6863
:10F6D8005B68D31A024AC2F89C3070474800002081
:10F6E8008C02002000280DDD074B5A68904209DB88
:10F6F800064A904206DC18601A685B68D31A044A06
:10F70800C2F89C30704700BF4800002080841E006B
:10F718008C020020FF2808B509D805F0A3FB044B8C
:10F72800002205F02FFD05F015FE024B986108BD7B
:10F73800000009404800002037B50C230093044618
:10F748000423C8220A210020F9F769FC424D14B3AA
:10F75800002108464FF48052F9F7EBFB3F4B542148
:10F76800DA690020F9F7E5FB002210465021F9F785
:10F77800E0FB6A6CFF21082385F8401085F84130CA
:10F78800019100936321D3B20020C2F30722F9F755
:10F79800ADFB03B030BD20464FF00A125621F9F7F1
:10F7A800C8FB20464FF4C8625821F9F7C2FB20462F
:10F7B8004FF404120721F9F7BCFB2046284A082118
:10F7C800F9F7B7FB20464FF6FF726821F9F7B1FB4E
:10F7D8004FF4406221462046F9F7ABFB082120464A
:10F7E800F9F7C7FB224620466921F9F7A2FB204614
:10F7F8004FF6FF726821F9F79CFB4FF467422046E9
:10F808006921F9F796FB08212046F9F7B2FB6A212E
:10F818002046F9F7AEFB6B212046F9F7AAFB6A6C84
:10F8280085F84040072385F841308DE818002046C8
:10F83800D3B26321C2F30722F9F758FB20464FF4ED
:10F8480080425421F9F775FB22465021204603B027
:10F85800BDE83040F9F76DBBAC0C0020280C002047
:10F868000D081010F7B5D24C94F80031013B042B69
:10F8780067D8DFE813F0050068008E009600540191
:10F88800CC4B00251D7284F8D850F9F709FDF9F71B
:10F8980013FC0120FFF750FF2B462A462946009506
:10F8A8000120F8F7CFFF80222B4601920092062113
:10F8B8002846F9F71BFB012220212846F9F739FBD6
:10F8C8004FF4FA20F9F7FCFC282102462846F9F7FC
:10F8D80030FB2846F9F7F2FC242102462846F9F7BE
:10F8E80028FB012220212846F9F723FB2846F9F7AF
:10F8F800E5FC242102462846F9F71BFB502128463F
:10F90800F9F737FB212102462846F9F712FB2A4668
:10F9180037212846F9F70DFB052220212846F9F75B
:10F9280008FB4FF44840F9F7C9FC24210246284651
:10F93800F9F7FFFAC4F804510223C4F8085184F80F
:10F94800003103B0F0BD0F210020F9F712FBC0070A
:10F95800F7D579210020F9F70CFB7F2805DCC0F1E9
:10F968008000C4F804010323E9E7B0F5C07F02DA98
:10F97800C0F5C070F5E7B0F5207F02DAC0F5207059
:10F98800EFE7B0F5607FB4BFC0F56070C0F5906078
:10F99800E7E7D4F8042137210020F9F7CAFA04234D
:10F9A800CDE70F210020F9F7E4FAC107C9D5D4F84B
:10F9B8000831B3F5C87F28D221210020F9F7D9FAF8
:10F9C8004FF44842D4F8081190FBF2F303FB1200FD
:10F9D800104404EB810190FBF2F302FB1300A1F841
:10F9E8000E01D4F80851FFF76FFAD4F8043103F583
:10F9F8008073C4F80431D4F8083104EB8505013369
:10FA0800A5F80C01C4F80831ADE76B4B997D9A7ADB
:10FA180001915B7A0093002306211846F9F766FAEC
:10FA280000238CE719461D8831F8046FAE4200F1B7
:10FA3800010006D2D1F800E05E889D80C3F800E09E
:10FA4800DE800B469042EDDB013A69D1B4F82A1406
:10FA5800B4F80E51B4F80C016FF000424FF00043B7
:10FA6800A94284E80C00B4F828245DD9C1F5804384
:10FA78002B4407EE903AC2F58043B8EEE77A034488
:10FA880007EE903AF8EEE77A0132C7EE276A0E469B
:10FA98004FF0010E43F6FF7CDFED487A9FED487A80
:10FAA80066EEA77AF4EEC77AF1EE10FA44BFBDEE1F
:10FAB800E77A17EE103A9FED437A48BF2360F4EED9
:10FAC800C77AF1EE10FAC4BFFDEEE77AC4ED017A09
:10FAD800824234D172B6FFF773FC2946B4F80E316E
:10FAE800B4F80C21384D0020FFF754F9FB88BA8888
:10FAF800798837F8040BFFF74DF9BD42F6D1334644
:10FB08004FF48042B4F82A14B4F82804FFF742F9F5
:10FB180062B602F0E5FA012384F8D83080E7C722FC
:10FB28002A4F00203B468DE7C5F580430B4407EE7E
:10FB3800903AC0F58043B8EEE77A1344A0E7EAB9F3
:10FB480007EE90EAB8EEE77A07EE901AF8EE677AD1
:10FB5800E6EE877AFDEEE77A17EE905A6B42C3F32A
:10FB68000D03C5F30D0558BF5D42ADB20132B2F5C4
:10FB7800804F0EF1010EA8BF0022A9E76245F5D11A
:10FB880007EE90EAB8EEE77A07EE901AF8EE677A91
:10FB9800E6EE877AFDEEE77A17EE903A5E4206EADD
:10FBA800020603EA020358BF73429EB2DEE700BFB3
:10FBB8008C02002048000020280C002000007A4415
:10FBC8000000004F000000CFB4060020980300207A
:10FBD800024B012283F80021704700BF8C020020ED
:10FBE800044B93F8002102F0FF0012B1D3F808018A
:10FBF800013070478C020020014B1868704700BF25
:10FC08008C020020014B5868704700BF8C0200200E
:10FC180048B9064B1B7A1BB1054BD3F8C80070478F
:10FC28006621F9F7A6B90020704700BF48000020F8
:10FC38008C020020B0F5C87F3FBF064B03EB800065
:10FC4800B0F80C31B0F80E0134BF40EA03404FF071
:10FC5800FF3070478C020020014B1872704700BFBC
:10FC680048000020014B83F8D80070478C02002020
:10FC780030B501219BB0022003F0ECF901214FF0CF
:10FC8800805003F0E7F901214FF0005003F0E2F94A
:10FC98004FF4887003F06AF9434803F067F90024C9
:10FCA80003236946414800938DF804308DF80740D6
:10FCB80002F0ECFC3E4B10933E4B0F934FF48063E5
:10FCC80016934FF4807315930223ADF848308023C0
:10FCD80014930FA920233848179311941994139457
:10FCE800189402F08BF80121334802F0B2F8012190
:10FCF800324801F0D2F9F8F7C5FA0446F8F7C2FA23
:10FD0800001B0028B8BF40420428F7DD2B4800211B
:10FD180001F0AFF9294801F0A1F9284801F0B1F93B
:10FD280004460028F9D1022502A902900390049004
:10FD38008DF818002148059501F052F907A801F03F
:10FD480025F94FF4005307A91C4807930894099410
:10FD58000A940B940C940D948DF8385001F0F8F82F
:10FD68002946164801F087FB0121144801F07AFB67
:10FD7800032301220C21114801F066FA01210F48E2
:10FD880003232A4601F060FA01210C4801F05DF9CD
:10FD980001210A4801F0E5FB0028F9D0074801F0E5
:10FDA800C1FA1BB030BD00BF00220010000400489B
:10FDB800D8090020400400505804024000040050B4
:10FDC800082808B503D009280CD0002008BD1E4B10
:10FDD800188883B240F2F720584340F6FF7390FB2F
:10FDE800F3F008BD184B588880B207EE900AF8EE79
:10FDF800677A17EE900A05F047F80DA3D3E90023B8
:10FE080005F096F80CA3D3E9002305F0BBF905F03B
:10FE1800C9FA05F039F800220C4B04F0D5FE08A306
:10FE2800D3E9002305F0AEF905F094FA08BD00BF48
:10FE38006666666666660A400000000000FEAF401F
:10FE48007B14AE47E17A843FD80900200000E03FE8
:10FE58002DE9F74305460C4691460C216FF00072D8
:10FE680098469DF828709DF82C60F9F762F80E21E5
:10FE78002846F9F77EF844F08003019300231A46D8
:10FE880000936D212846F9F731F80196009743460B
:10FE98004A466C212846F9F729F80E212846F9F731
:10FEA80068F88301F9D548EA092804F07F0447EA8D
:10FEB80008272C44034B46EA072643F8246003B07E
:10FEC800BDE8F083E009002073B505460C461646E8
:10FED8000C216FF00072F9F72CF80E212846F9F77B
:10FEE80048F844F08003019300231A466D21284600
:10FEF8000093F8F7FBFF32466C212846F9F719F80A
:10FF08000E212846F9F735F88301F9D504F07F0466
:10FF18002C44024B43F8246002B070BDE009002075
:10FF280073B51D4B01F07F0405461B5D73B3F8F7ED
:10FF3800D3FF064650BB6FF000720C212846F8F735
:10FF4800F8FF0E212846F9F714F832466D212846A5
:10FF5800019400963346F8F7C9FF32466C212846CB
:10FF6800F8F7E7FF0E212846F9F703F88201F9D5DB
:10FF78006E212846F8F7FDFF222C01D0422C03D130
:10FF8800030201D540F07F4002B070BD2C44034B02
:10FF980053F82400F8E700BFE3580108E0090020FF
:10FFA80070B50B4C2218054692F800220E465AB935
:10FFB8006C21FFF7B5FF06F00F0320F00F021A437C
:10FFC8006C212846FFF780FF631983F8016270BD32
:10FFD800E009002038B50C466C210546FFF7A0FF64
:10FFE800240104F0700420F07002224328466C219A
:08FFF800BDE83840FFF768BFC7
:020000040801F1
:1000000038B50C466C210546FFF78EFFE40304F477
:10001000C03420F4C032224328466C21BDE8384069
:10002000FFF756BF38B50C466C210546FFF77CFF3D
:10003000240504F4700420F47002224328466C2145
:10004000BDE83840FFF744BF38B50C466C21054683
:10005000FFF76AFF240604F0706420F07062224308
:1000600028466C21BDE83840FFF732BF38B50D4651
:100070006C210446FFF758FF3DB140F08042204616
:100080006C21BDE83840FFF723BF20F08042F6E73F
:1000900038B50D466C210446FFF746FF3DB140F4EC
:1000A000002220466C21BDE83840FFF711BF20F444
:1000B0000022F6E738B50D466C210446FFF734FF01
:1000C0003DB140F4802220466C21BDE83840FFF766
:1000D000FFBE20F48022F6E738B50D466C210446B9
:1000E000FFF722FF3DB140F4804220466C21BDE87D
:1000F0003840FFF7EDBE20F48042F6E738B50D46F4
:100100006C210446FFF710FF3DB140F40052204639
:100110006C21BDE83840FFF7DBBE20F40052F6E763
:1001200038B50D466C210446FFF7FEFE3DB140F4A4
:10013000805220466C21BDE83840FFF7C9BE20F44C
:100140008052F6E738B50C466C210546FFF7ECFE09
:10015000230748BF20F070004FEA04124CBF40F460
:10016000006020F4076002F0700202436C21284610
:10017000BDE83840FFF7ACBE38B50C466C210546EB
:10018000FFF7D2FEE40104F4F06420F4F0622243AD
:1001900028466C21BDE83840FFF79ABEFFF7ECBF58
:1001A00038B50D466C210446FFF7BEFE3DB140F464
:1001B000003220466C21BDE83840FFF789BE20F4AC
:1001C0000032F6E708B5074B034493F800222AB93A
:1001D0006C21FFF7A9FE00F00F0008BD93F80102A3
:1001E00008BD00BFE009002008B56C21FFF79CFEA8
:1001F000C0F3021008BD08B56C21FFF795FEC0F3EF
:10020000C13008BD08B56C21FFF78EFEC0F3035066
:1002100008BD08B56C21FFF787FEC0F3036008BD79
:1002200008B56C21FFF780FEC0F3807008BD08B5EB
:100230006C21FFF779FEC0F3C04008BD08B56C2102
:10024000FFF772FEC0F3804008BD08B56C21FFF7D0
:100250006BFEC0F3803008BD08B56C21FFF764FE6B
:10026000C0F3403008BD08B56C21FFF75DFEC0F358
:10027000003008BD08B56C21FFF756FEC0F302132D
:10028000020548BF43F00803184608BD08B56C21B5
:10029000FFF74AFEC0F3C31008BDFFF7F7BF08B56C
:1002A0006C21FFF741FEC0F3404008BD38B50C4655
:1002B0006D210546FFF738FE640104F0600420F06C
:1002C0006002224328466D21BDE83840FFF700BE9A
:1002D00038B50C466D210546FFF726FE640304F48D
:1002E000C04420F4C042224328466D21BDE8384076
:1002F000FFF7EEBD38B50C466D210546FFF714FE3D
:10030000240204F4706420F47062224328466D21B4
:10031000BDE83840FFF7DCBD38B50C466D21054619
:10032000FFF702FE04F00F0420F00F0222432846DC
:100330006D21BDE83840FFF7CBBD38B50D466D21C6
:100340000446FFF7F1FD20F47F0040EA05426D21ED
:100350002046BDE83840FFF7BBBD38B50D466D21DE
:100360000446FFF7E1FD3DB140F4004220466D2117
:10037000BDE83840FFF7ACBD20F40042F6E738B5E1
:100380000D466D210446FFF7CFFD3DB140F0807270
:1003900020466D21BDE83840FFF79ABD20F08072FD
:1003A000F6E708B56D21FFF7BFFDC0F3411008BDAA
:1003B00008B56D21FFF7B8FDC0F3413008BD08B5A1
:1003C0006D21FFF7B1FDC0F3032008BD08B56D2115
:1003D000FFF7AAFD00F00F0008BD08B56D21FFF77B
:1003E000A3FD0314D8B21B0648BF60F0FF0008BD90
:1003F00008B56D21FFF798FDC0F3C03008BD08B502
:100400006D21FFF791FDC0F3006008BD38B50C46C3
:1004100070210546FFF788FD04F0030420F4401224
:1004200042EA045228467021BDE83840FFF750BD2B
:1004300038B50D4670210446FFF776FD3DB140F416
:10044000002220467021BDE83840FFF741BD20F46E
:100450000022F6E738B50D4670210446FFF764FD2B
:100460003DB140F4802220467021BDE83840FFF7BE
:100470002FBD20F48022F6E738B50C4670210546E2
:10048000FFF752FD04F0030420F4403242EA044234
:1004900028467021BDE83840FFF71ABD38B50D4633
:1004A00070210446FFF740FD20F47F4040EA05221A
:1004B00070212046BDE83840FFF70ABD38B50D462B
:1004C00070210446FFF730FD20F0FF0045EA0002EE
:1004D00070212046BDE83840FFF7FABC08B570210E
:1004E000FFF722FDC0F3015008BD08B57021FFF7EA
:1004F0001BFDC0F3C04008BD08B57021FFF714FD17
:10050000C0F3804008BD08B57021FFF70DFDC0F3B2
:10051000014008BD08B57021FFF706FDC0F30720B4
:1005200008BD08B57021FFF7FFFCC0B208BDF8B5E3
:1005300007460E4615461C46F8F7D2FC78B96C21E2
:100540003846F8F71AFD16B1C0F30903336015B148
:10055000C0F304432B700CB1000E2070F8BD0020D6
:10056000F1E737B5002108464FF00112FFF7B0FC64
:10057000022253238DE80C000022104641236C21F7
:10058000FFF76AFC0A25002300241A4618460921B1
:1005900001950095FFF760FC01232246294620467D
:1005A00001950094FFF758FC1F2301930093224606
:1005B000234610212046FFF74FFC0420F8F7D2F91C
:1005C00001301CD00520F8F7CDF90B21024620465A
:1005D000FFF77EFC0620F8F7C5F9C1B22046FFF709
:1005E000E3FC0720F8F7BEF9C1B22046FFF7F6FC9E
:1005F0000820F8F7B7F9C1B22046FFF7BDFD084A59
:1006000070210020FFF764FC0020FFF7DBFD054BA5
:10061000002283F8010283F8002203B030BD00BF3E
:100620001E000CC4E009002038B5074C044494F8BF
:10063000001241B994F80152FFF7B6FC012384F887
:10064000003284F8015238BDE0090020064B034413
:1006500093F8002232B1002293F8011283F80022AD
:10066000FFF7A2BC704700BFE0090020024B18440E
:1006700090F80002704700BFE0090020684620F0B3
:1006800007018D4631B5264C264B25681B68013580
:10069000082D08BF00259D4286B03BD001AA00214D
:1006A000214801F092F99DF80C302268042B1F4B71
:1006B00003EB021227D1012151702268029903EB4A
:1006C000021251609DF80D20022A226803EB0212EB
:1006D0000CBF01210021917022689DF80E101201BB
:1006E00099540022216801A8104403EB0111114420
:1006F0000132C07A0872082AF4D1256006B0BDE83C
:10070000314085467047002151702268019903EB02
:100710000212D6E70021044801F0A2F9EEE700BF7B
:100720007C120020F011002000640040FC11002029
:10073000684620F007018D4631B5264C264B2568CA
:100740001B680135082D08BF00259D4286B03BD0AF
:1007500001AA0121214801F038F99DF80C302268E6
:10076000042B1F4B03EB021227D101215170226889
:10077000029903EB021251609DF80D20022A2268B3
:1007800003EB02120CBF01210021917022689DF839
:100790000E10120199540022216801A8104403EBA5
:1007A000011111440132C07A0872082AF4D125607F
:1007B00006B0BDE83140854670470021517022687F
:1007C000019903EB0212D6E70121044801F048F930
:1007D000EEE700BF7C120020F01100200064004012
:1007E000FC110020684620F007018D4611B52C4B06
:1007F0002C4A19681268914287B009D10022012160
:10080000294801F0B0F907B0BDE8114085467047AE
:100810001968264A02EB0111497801F0FF0000290E
:1008200032D004218DF80C1000210191196802EBDF
:10083000011149680291196802EB0111897801F0F0
:10084000FF0051B302218DF80D1019680901515CA8
:100850008DF80E100021186802EB00100844047A8D
:1008600001A8084401310829C472F4D11A680E485D
:1008700001321A601A68082A08BF002201A908BFBD
:100880001A6001F010F8BEE719688DF80C0002EB51
:100890000111029049680191CDE78DF80D00D4E770
:1008A000F8110020F41100200064004080120020A4
:1008B000F0B501388BB00E4615460C23072800F220
:1008C0000A81DFE810F00601040102010001FE00C8
:1008D0000801FC00080002228DF8103003238DF877
:1008E00011309448ADF80C2000238DF80F3000F043
:1008F0007FFE01214FF0007002F0C8FB01214FF490
:10090000003002F0ABFB4FF4C053019302230024EC
:100910008DF8083001A903234FF090408DF809307D
:100920008DF80A408DF80B4001F0B4FE09220B212E
:100930004FF0904001F026FF09220C214FF090402B
:1009400001F020FF012703A97A488DF80E408DF8A9
:1009500012408DF813708DF814408DF815408DF805
:1009600016708DF8177000F050FEB6F5006F8DF818
:1009700022408DF823408DF8247080F2AE80730100
:10098000ADF818304FF6FF73ADF81A40ADF81C30D3
:10099000ADF81E30ADF820408DF8257006A800F0A7
:1009A000AEFE012300228DF822308DF823208DF831
:1009B0002430002D00F0A080B5F5006F80F29C80FF
:1009C0006901ADF81A204FF6FF72ADF81810ADF8B6
:1009D0001C20ADF81E20ADF820308DF8253006A87B
:1009E00000F08DFE02238DF822307313F60046F0DE
:1009F000040600270124ADF81A6006A84FF6FF761A
:100A0000ADF818308DF823708DF82440ADF81C60D7
:100A1000ADF81E60ADF820708DF8254000F06FFE37
:100A20000323BD428DF822308DF823708DF82440C9
:100A300071DD6B13ED0045F00405ADF81830ADF82D
:100A40001A50ADF81C60ADF81E60ADF820408DF86E
:100A5000254006A800F053FE012407260025142394
:100A600068468DF800308DF801608DF802508DF8E1
:100A7000034002F04BF8152368468DF800308DF8DE
:100A800001608DF802508DF8034002F03FF8132307
:100A900068468DF800308DF801608DF802508DF8B1
:100AA000034002F033F822460221224801F05BF8AD
:100AB000224610211F4801F056F80BB0F0BD042269
:100AC0000AE7102208E7142206E7282204E7642236
:100AD00002E7C82200E70822FEE64FF6FF73ADF8F2
:100AE0001840ADF81A40ADF81C30ADF81E30ADF826
:100AF00020408DF8254051E74FF6FF71ADF81820E2
:100B0000ADF81A20ADF81C10ADF81E10ADF820306D
:100B10008DF8252063E70423ADF81870ADF81A307E
:100B2000ADF81C60ADF81E60ADF820408DF8257062
:100B30008FE700BF00640040F0B54378426887B09B
:100B40000446002B39D004238DF80C300023029288
:100B50000193A37803B102238DF80D30234606AA32
:100B600013F8081B02F80A1D04F1100113F8010B19
:100B700002F8010F8B42F9D101A9134800F093FE4E
:100B8000042817D1114F124B3D681B680135082D01
:100B900008BF00259D4215D03B680E4E06EB03169C
:100BA00094E80F0086E80F000122114606483D60D8
:100BB00000F0D9FF012007B0F0BD8DF80C30019294
:100BC0000293C6E70020F6E700640040F41100201D
:100BD000F81100208012002030B50C4B0C4C22681C
:100BE0001B689A4205460FD02268531C2360094BAC
:100BF00003EB02130FCB85E80F002368082B01D10C
:100C000000232360012030BD002030BD7C12002075
:100C1000F0110020FC110020F0B510208BB002F084
:100C2000B9F9224D01214FF4001002F02FFA0121F1
:100C30004FF4802002F012FA28460422062101F027
:100C4000A1FD04222846072101F09CFD02230AAEE3
:100C50008DF8083003238DF80930402346F8243DF1
:100C600000240127314628468DF80A708DF80B4084
:100C700001F010FD28460E4D80233146019301F00E
:100C800009FD284601F090FD0AA90A4B41F81C3DD8
:100C900028460694049405940894099401F0A0FD54
:100CA0003946284601F0D7FD0BB0F0BD00040048DE
:100CB000005400407A25E0002DE9F74304468946B8
:100CC00017461D464FF40041204601F0F6FE064649
:100CD0000028F7D14FF41053ADB200933A464FF0CD
:100CE00000732946204601F06AFEC846A8EB0903B6
:100CF0009F4203D8012003B0BDE8F08304212046C1
:100D000001F0DBFE0028F9D0204601F0C9FE4FF0CB
:100D1000007308F8010B3A4600962946204601F078
:100D20004EFEE3E72DE9F7430446894617461D4684
:100D30004FF40041204601F0C0FE06460028F7D1DE
:100D40004FF40053ADB200933A464FF0007329467A
:100D5000204601F034FEC846A8EB09039F4203D8A1
:100D6000012003B0BDE8F0830221204601F0A5FE7A
:100D70000028F9D018F8011B204601F08FFE0096DC
:100D80004FF000733A462946204601F018FEE3E78B
:100D90007047FEE7FEE7FEE7FEE7704770477047E3
:100DA000384AD2F8883043F47003C2F88830364BA2
:100DB0001A6842F001021A605968344A0A405A60BF
:100DC0001A6822F0847222F480321A601A6822F4BF
:100DD00080221A605A6822F4FE025A60DA6A22F00F
:100DE0000F02DA62196B2A4A82B00A401A630022A3
:100DF0009A60009201921A6842F480321A601A686E
:100E000002F400320192009A01320092019A1AB95A
:100E1000009AB2F5A06FF2D11A6812F4003218BF2E
:100E200001220192019A012A04D0164B194A9A60B4
:100E300002B07047184A122111605A685A605A6805
:100E40005A605A6842F480625A605A6822F47C12EE
:100E50005A605A6842F4F8125A601A6842F0807276
:100E60001A601A689201FCD55A6822F003025A608F
:100E70005A6842F002025A605A6802F00C02082ACC
:100E8000FAD1D2E700ED00E0001002400CC07FF87C
:100E9000CCFC00FF00800008002002401549164AE3
:100EA0004B6803F00C03042B10B50CD0082B0CD0AE
:100EB000124B13604B68C3F303131344197913687F
:100EC000CB40136010BD0E4BF3E74B684868C0037E
:100ED00049BFC86A0B480A4C00F00F00C3F38343B4
:100EE00048BF013003F1020348BFB4FBF0F04343B5
:100EF000DFE700BF001002406400002000127A000B
:100F00000024F40000093D00B0F1A04F08B502D064
:100F10000F4B98420BD101214FF0805002F0C2F8E4
:100F200000214FF08050BDE8084002F0BBB8094BEB
:100F3000984203D003F58073984208D101214FF005
:100F4000005002F0AFF800214FF00050EBE708BD71
:100F50000001005000040050C3680D4A10B51A404B
:100F600091E8180023438C682343CC6823430C6921
:100F700023434C6923438C6923431343C360026BAF
:100F80000B7F22F00F02013B1343036310BD00BF30
:100F900007C0FFFD0023036043608360C3600361FB
:100FA00043618361012303777047C36C91E80C00B0
:100FB0001343CA6843EA02230A6943EA82334A694F
:100FC00043EA02538A6943EA82630A7A013A134385
:100FD000C364704700230360436001230372C3604E
:100FE0000361436183617047B0F1A04F10B5114BAD
:100FF00002D0114A904218D1104A94681C4091E8DE
:101000000C0013438A681343CA6843EA02330A7C1C
:10101000B0F1A04F43EA022343EA040302D0064A98
:10102000904204D1054A936010BD054AE5E7044AA1
:10103000F9E700BFE010FCFF000100500003005082
:10104000000700500023036043608360C3600374A3
:101050007047836819B143F001038360704743F020
:101060000203FAE7836843F0004383607047D0F8D7
:10107000B4007047C0F8B4107047836823F0804311
:10108000836083681943816070478068C00F704730
:10109000836843F00203836070478068C0F34000B8
:1010A0007047836823F040538360836819B143F02D
:1010B00080538360704743F00053FAE7012332B155
:1010C000D0F8B0208B401343C0F8B0307047D0F850
:1010D000B0208B4022EA0303F6E7C36819B143F45A
:1010E0000013C360704723F40013FAE7C36819B113
:1010F00043F48043C360704723F48043FAE7C36836
:1011000023F0E0731943C1607047036A23F07F63E3
:1011100023F470230362036A43EA01410162036A14
:1011200023F47F6323F00F030362036A1A4302620E
:101130007047436A23F47F034362436A43EA0141F1
:101140004162436A23F0FF034362436A1A434262E7
:101150007047836A23F47F038362836A43EA014111
:101160008162836A23F0FF038362836A1A43826287
:101170007047C36823F0F84343EA8161C160704758
:1011800010B5D0F8A020D0F8A040012303FA01F157
:10119000A3F50023214313401943C0F8A01010BD4C
:1011A00010B5D0F8A420D0F8A440012303FA01F12F
:1011B000A3F50023214313401943C0F8A41010BD28
:1011C000B0F1A04F02D0074B984206D1064B9A6867
:1011D00029B142F400029A607047044BF7E722F409
:1011E0000002F8E700010050000300500007005023
:1011F000B0F1A04F02D0074B984206D1064B9A6837
:1012000029B142F480029A607047044BF7E722F458
:101210008002F8E700010050000300500007005072
:10122000B0F1A04F02D0074B984206D1064B9A6806
:1012300029B142F080729A607047044BF7E722F0C0
:101240008072F8E7000100500003005000070050D2
:10125000042A30B51CD802EB4202046B52001F2551
:10126000954024EA050401FA02F2224302630929A7
:1012700039D90A398269826901EB410107248C401E
:1012800022EA0402826182698B401343836130BD8C
:10129000092A0CD80624053A6243456B1F24944062
:1012A00025EA040401FA02F222434263DFE70E2A30
:1012B0004FF006040BD80A3A6243856B1F24944012
:1012C00025EA040401FA02F222438263CFE70F3ACF
:1012D0006243C56B1F24944025EA040401FA02F21C
:1012E0002243C263C3E701394269426901EB41010C
:1012F00038248C4022EA040242614269033103FA35
:1013000001F11143416130BD036B23F00F0303630F
:10131000036B0139194301637047C36823F47C638D
:10132000C360C3680A431A43C2607047836843F0CE
:101330000403836070478068C0F38000704783684F
:1013400043F0100383607047C368013923F46023BE
:1013500043EA4143C3607047C36819B143F4803323
:10136000C360704723F48033FAE7006C80B27047A3
:10137000B0F1A04F02D0044B984202D1034BD86881
:101380007047034BFBE700BF000100500003005013
:1013900000070050036E23F0F8430366036E43EA30
:1013A00081610166036E23F47F6323F00F030366FC
:1013B000036E1A4302667047436E23F0F843436698
:1013C000436E43EA81614166436E23F47F6323F0F9
:1013D0000F034366436E1A4342667047836E23F0E1
:1013E000F8438366836E43EA81618166836E23F4EA
:1013F0007F6323F00F038366836E1A438266704710
:10140000C36E23F0F843C366C36E43EA8161C166CD
:10141000C36E23F47F6323F00F03C366C36E1A43C6
:10142000C2667047036E19B143F00043036670470C
:1014300023F00043FAE7436E19B143F000434366DB
:10144000704723F00043FAE7836E19B143F000437D
:101450008366704723F00043FAE7C36E19B143F087
:101460000043C366704723F00043FAE7C36819B12D
:1014700043F00103C360704723F00103FAE7C36838
:1014800023F00203C360C3681943C1607047092990
:1014900070B519D9A1F10A04856904EB4404072643
:1014A000A64025EA060503FA04F42C438461541E81
:1014B00006226243C36C4FF4F854944023EA0403B9
:1014C00091401943C16470BD456901EB4106072491
:1014D000B44025EA040503FA06F42C434461E6E728
:1014E000C36C013923F003031943C1647047C36C13
:1014F00023F0FC03C364C36C0A431A43C2647047FD
:10150000836843F0080383607047836843F02003D7
:10151000836070478068C0F3C0007047C36819B12A
:1015200043F00073C360704723F00073FAE7C368A9
:1015300019B143F48013C360704723F48013FAE7B2
:1015400082B0002301930190019B803319440191E3
:10155000019B186880B202B07047436812B119430A
:101560004160704723EA0101FAE703680B4214BFA8
:1015700001200020704701607047B0F1A04F02D0F9
:10158000054B984206D1054B1B680B4214BF012046
:1015900000207047024BF7E70001005000030050A5
:1015A00000070050B0F1A04F02D0064B984204D182
:1015B000054B1A68114319607047044A13681943B0
:1015C00011607047000100500003005000070050F8
:1015D0000368426889B211EA030003D0114214BFC4
:1015E000012000207047036819430160704700BF65
:1015F00008B501214FF0007001F06CFD00214FF0A3
:101600000070BDE8084001F065BD82B00023019381
:10161000036823F002030360036843F001030360DF
:101620006FF07F424368DB0702D4019B93425CD199
:10163000436813F0010360D08B79012B03680CBF62
:1016400043F0800323F080030360CB79012B036810
:101650000CBF43F0400323F0400303600B7A012BDF
:1016600003680CBF43F0200323F0200303604B7A90
:10167000012B03680CBF43F0100323F01003036039
:101680008B7A012B03680CBF43F0080323F0080397
:101690000360CB7A012B03680CBF43F0040323F0F3
:1016A00004030360CB788A781B0643EA82730A79C5
:1016B00043EA02434A7943EA02530A88013A134350
:1016C000C361036823F001030360002301936FF0FB
:1016D0007F424368DB0702D5019B934209D14068F2
:1016E000C04300F0010002B07047019B0133019339
:1016F00098E7019B01330193EBE71846F3E7374A7C
:10170000837AD2F8001241F0010130B5C2F800121C
:101710000125D2F81C129D40EC432140C2F81C1256
:10172000017B002934D1D2F80C122140C2F80C12EE
:10173000C2884188DB0041EA024103F1804202F5A0
:10174000C8420388C2F84012818843EA0143C2F8C4
:101750004432C37A2149A3BBD1F804322340C1F8F3
:10176000043203891D4A83BBD1F814321C40C1F8EE
:101770001442437B012B02BFD2F81C322B43C2F828
:101780001C32D2F8003223F00103C2F8003230BD1F
:101790000129DED1D2F80C12DB002943C2F80C1269
:1017A00003F180430188428803F5C84342EA0142BD
:1017B000C3F840228188C28842EA0142C3F8442229
:1017C000C7E7D1F804322B43C9E7012B02BFD2F897
:1017D00014322B43C2F81432CBE700BF0064004040
:1017E00000238371C371037243728372C372837067
:1017F000C3700323037102234371012303807047E5
:101800000D4BD3F8002242F00102C3F80022D3F8B6
:10181000002222F47C5222F00E02C3F80022D3F8F8
:10182000002242EA0020C3F80002D3F8002222F08E
:101830000102C3F80022704700640040036819B138
:1018400043F480330360704723F48033FAE703687E
:10185000A9B143F080030360D0F8843143F480736E
:10186000C0F88431D0F8943143F48073C0F89431D7
:10187000D0F8A43143F48073C0F8A431704723F04A
:1018800080030360D0F8843123F48073C0F884317E
:10189000D0F8943123F48073C0F89431D0F8A43197
:1018A00023F48073E8E78368F0B55C0102462FD427
:1018B0008368180140D49368DB003FD40420F0BD56
:1018C0000C68D3F8806145EA44543443C3F880413E
:1018D0008C7A04F00F048C72D3F8845125F00F0534
:1018E000C3F88451D3F884512C43C3F8844102EBEC
:1018F0000012D1F80B40C2F88841D1F80F10C2F89D
:101900008C11D3F8802142F00102C3F88021F0BD90
:10191000002002EB0013D3F8804104F00104C3F867
:1019200080410C7A4D7A002CCAD04F68D3F8806180
:1019300044EAC7042C43C8E70120EAE70220E8E7AD
:10194000012915D003D3022916D0022070478368DD
:1019500023F07B4323F47F0323F47F4323F0FC0332
:101960000D4A934216D00FD8002BEED000207047BE
:1019700082680A4B1340F3E7836823F06F4323F434
:101980007C031B0C1B04EBE7044A934202D0044A7D
:101990009342EBD1012070470300000400030008CC
:1019A00000000310012908D002D3022909D0704792
:1019B000836843F0800383607047836843F4004387
:1019C000F9E7836843F40003F5E700EB011310B572
:1019D000D3F8B04104F004041472BCBBD3F8B04196
:1019E000640D1460D3F8B04104F002045472D3F8CB
:1019F000B44104F00F049472D3F8B4311B0AD374C9
:101A000000EB0113D3F8B841D472D3F8B841240ADB
:101A10001473D3F8B841240C5473D3F8B841240E8E
:101A20009473D3F8BC41D473D3F8BC41240A147422
:101A3000D3F8BC41240C5474D3F8BC311B0E9374FE
:101A400049B9C36843F02003C36010BDD3F8B04167
:101A5000E4085460C6E7036943F02003036110BD46
:101A600021B9C36843F02003C3607047036943F0A2
:101A700020030361704719B9C06800F00300704784
:101A8000012901D10069F8E700207047B1B9036866
:101A900023F0030343F0010303604FF080734268B7
:101AA00002F00302012A01D0013BF8D1406800F0A6
:101AB0000300012814BF002001207047012911D123
:101AC000036823F0030303604FF0807342689207BA
:101AD00001D0013BFAD1436813F0030F0CBF012082
:101AE00000207047022913D1036823F0030343F059
:101AF000020303604FF08073426802F00302022A7F
:101B000001D0013BF8D1406800F003000228D1E782
:101B100000207047036823F0030343F002030360CF
:101B2000406800F00300831E584258417047036824
:101B300023F0020303604FF080734268920701D5DF
:101B4000013BFAD1406880F00200C0F340007047CA
:101B5000806900F0700070478069000E70478069EE
:101B6000C0F307407047436912B1194341617047A0
:101B700023EA0101FAE711F4700F07D08369C3F378
:101B800013030B4214BF012000207047CB0101D585
:101B90004368F4E70A0101D58368F0E78B014CBF85
:101BA000C3680369EBE70A4B994202D100238361C2
:101BB00070478A01C1F3130301D5C36070474A011E
:101BC00001D5036170470A014CBF836043607047D1
:101BD0007000F03043690B4009D0402946D012D83C
:101BE00004293BD005D8012929D0022930D0002072
:101BF0007047102936D0202936D00829F7D1C0687F
:101C0000C0F300107047B1F5006F3DD00CD8B1F5AE
:101C1000007F31D0B1F5806F32D0B1F5807FE6D151
:101C2000806900F001007047B1F5803F20D0B1F528
:101C3000003F1FD0B1F5004FD9D1406821E0806846
:101C400000F0013020F08070003018BF0120704794
:101C5000C06810F0030018BF01207047C068C0F3CF
:101C6000C00070470069F4E70069F8E70069C7E75A
:101C70004068F4E74068C3E78069C0F340007047FC
:101C80008069C0F380007047836913F0700F14BF40
:101C9000012000207047B1F5807F23D00CD808299F
:101CA00028D004D801291FD0042920D0704720292A
:101CB00022D0402923D07047B1F5006F10D006D84C
:101CC000B1F5007F0ED0B1F5806F0BD07047B1F544
:101CD000803F16D0B1F5003F16D0B1F5004F12D1BC
:101CE0000023836104230DE0084B836070470823C1
:101CF000C36070471023FBE708230361704710237C
:101D0000FBE70823436070471023FBE70101010054
:101D1000036823F001031B041B0C03600023036012
:101D200043608360C360294B984204D1284A5368BA
:101D300043F00F0326E0274B984204D1244A53680E
:101D400043F0F0031EE0244B984204D1204A53682C
:101D500043F4706316E0214B984204D11C4A536847
:101D600043F470430EE01E4B984204D1184A536866
:101D700043F4702306E01B4B984205D1144A536884
:101D800043F4700353607047174B984204D1104AD4
:101D9000536843F07063F5E7144B984201D1144A3D
:101DA000C5E7144B984201D1114AC8E7124B98423B
:101DB00001D10F4ACBE7114B984201D10C4ACEE733
:101DC0000F4B9842DFD10A4AD1E700BF080002401A
:101DD000000002401C00024030000240440002406B
:101DE000580002406C00024080000240080402409B
:101DF000000402401C04024030040240440402403B
:101E0000580402408B68026810B50C6A23430C69C1
:101E100023434C6923438C692343CC6923434C6A95
:101E200023438C6A22F4FF4222F0700223431343BF
:101E300003608B8943600B6883604B68C36010BD8F
:101E40000023036043608360838103614361836196
:101E5000C3610362436283627047036819B143F050
:101E600001030360704723F001031B041B0CF8E718
:101E700041607047406880B27047036812B11943EF
:101E80000160704723EA0101FAE7C3004CBF044B2D
:101E9000044B1B68034214BF01200020704700BFA1
:101EA0000004024000000240FFF7EFBFC3004CBF38
:101EB000014B024B58607047000402400000024092
:101EC000FFF7F4BF0A4B4FF0FC521A606FF0FC5161
:101ED00000225A609A60DA601A6159610C21196215
:101EE0005A629A62DA621A6303225A63704700BF29
:101EF000000401408279036870B50479002A64D037
:101F000023F01F0101F1804101F5823103F01F022E
:101F10000D68012303FA02F225EA02020A60016851
:101F2000324D21F01F0601F01F01725903FA01F131
:101F300022EA01017151016804F1804221F01F057C
:101F400002F5823201F01F01AC5803FA01F121437E
:101F5000A9500268264D22F01F0402F01F026159A9
:101F600003FA02F221EA020262510268214C22F0D5
:101F70001F0602F01F02315903FA02F221EA02029F
:101F8000417932511029026812D122F01F0102F06A
:101F90001F024E5903FA02F232434A51026822F0FC
:101FA0001F0102F01F020859934003430B5170BDFB
:101FB00001F1804122F01F0001F5823102F01F0281
:101FC000445893402343435070BD04F1804223F0B2
:101FD0001F0502F5823203F01F03A958012000FA01
:101FE00003F321EA0303AB5070BD00BF04040140BA
:101FF000080401400C040140002310220360037117
:1020000042718371704720F01F0110B5044A00F03F
:102010001F038C58012098402043885010BD00BFFA
:102020001004014020F01F02054B00F01F00D258A1
:10203000012303FA00F0104214BF18460020704735
:102040001404014020F01F0303F1804303F58233A1
:1020500000F01F000122824019685869104003D027
:10206000114214BF01200020704720F01F020123FD
:1020700000F01F0003FA00F0014BD050704700BF82
:1020800014040140FFF7F1BF034A136823F0030370
:1020900018431060704700BF00200240044B1A68CC
:1020A00018B142F008021A60704722F00802FAE7FD
:1020B00000200240044B1A6818B142F010021A6066
:1020C000704722F01002FAE700200240044B1A6920
:1020D000120641BF034A5A6002F188325A607047C3
:1020E0000020024023016745024A136943F0800340
:1020F0001361704700200240044B1A6992055FBFCC
:10210000034A9A6002F188329A60704700200240C8
:1021100023016745024A136923F400731361704772
:1021200000200240024A136943F4005313617047D0
:1021300000200240024BD869C0F30720704700BF5F
:1021400000200240014B186A704700BF0020024087
:10215000034BDB6913F0060F14BF0120002070470A
:1021600000200240044B1A6911B1104318617047F6
:1021700022EA0000FAE700BF00200240034BDB68C0
:10218000034214BF01200020704700BF002002401E
:10219000014BD860704700BF00200240084BDA684E
:1021A000D10709D4DA68D20608D4DB6813F0040F2B
:1021B00014BF03200420704701207047022070479D
:1021C0000020024010B50446FFF7E8FF012806D1C1
:1021D0000CB9052010BDFFF7E1FF013CF6E7002C2C
:1021E00008BF052010BD38B505464FF43020FFF775
:1021F000E9FF042811D1094C236943F0020323614C
:102200006561236943F0400323614FF43020FFF7F9
:10221000D9FF236923F00203236138BD0020024067
:1022200010B54FF43020FFF7CDFF042810D1094C32
:10223000236943F004032361236943F040032361CE
:102240004FF43020FFF7BEFF236923F0040323611E
:1022500010BD00BF0020024073B5002306464FF4B6
:1022600030200D460193FFF7ADFF042819D10E4C25
:10227000236943F001032361ABB233804FF4302074
:10228000FFF7A0FF042808D102360196019B2D0C10
:102290001D804FF43020FFF795FF236923F00103E1
:1022A000236102B070BD00BF0020024070B505463A
:1022B0004FF430200E46FFF785FF04280DD1074C60
:1022C000236943F0010323614FF430202E80FFF790
:1022D00079FF236923F00103236170BD00200240D0
:1022E00038B5FFF735FF00284FF430200CBFAA2582
:1022F0000025FFF767FF042822D1124C236943F021
:1023000020032361236943F0400323614FF430200D
:10231000FFF758FF04280DD1236923F02003236120
:10232000236943F010032361074B4FF430201D80D5
:10233000FFF748FF05281EBF236923F01003236120
:1023400038BD00BF0020024000F8FF1F10B5044652
:102350004FF43020FFF736FF04281DD11249E44323
:102360000B69E2B243F01003FF2A0B610AD1C4F3F8
:102370000724FF2C11D104200B4A136923F010030A
:10238000136109E0094B4FF430201A81FFF71AFF5F
:102390000428ECD00528EFD110BD044B4FF43020B9
:1023A0005C81FFF70FFFF5E70020024000F8FF1FF8
:1023B00038B505464FF43020FFF704FF042823D139
:1023C000154C236943F020032361236943F0400344
:1023D00023614FF43020FFF7F5FE042815D123695F
:1023E00023F020032361236943F0100323610B4B87
:1023F000ADB21D804FF43020FFF7E4FE052803D076
:10240000236923F01003236138BD0528FCD023691C
:1024100023F02003F7E700BF0020024000F8FF1F71
:10242000F8B5124C124BA36003F188330546A36044
:102430004FF430200E461746FFF7C4FE042814D18F
:10244000236967F0070743F010033E4323613543D8
:10245000084BEDB25D804FF43020FFF7B3FE052846
:102460001EBF236923F010032361F8BD0020024042
:102470002301674500F8FF1F38B5104C104BA360CF
:1024800003F188330546A3604FF43020FFF79AFE2E
:10249000042811D1236943F010032361094B45F04F
:1024A000EF055D804FF43020FFF78CFE05281EBF3E
:1024B000236923F01003236138BD00BF00200240D0
:1024C0002301674500F8FF1F38B5104C104BA3607F
:1024D00003F188330546A3604FF43020FFF772FE06
:1024E000042811D1236943F010032361094B45F0FF
:1024F000DF055D804FF43020FFF764FE05281EBF26
:10250000236923F01003236138BD00BF002002407F
:102510002301674500F8FF1F38B505464FF430200A
:10252000FFF750FE042812D1094C236943F0100331
:102530002361084B45F0BF055D804FF43020FFF765
:1025400041FE05281EBF236923F01003236138BD17
:102550000020024000F8FF1F38B5104C104BA3605C
:1025600003F188330546A3604FF43020FFF72AFEBD
:10257000042811D1236943F010032361094B45F06E
:1025800088055D804FF43020FFF71CFE05281EBF34
:10259000236923F01003236138BD00BF00200240EF
:1025A0002301674500F8FF1F70B506464FF4302041
:1025B0000D46FFF707FE042810D1094C2369ADB280
:1025C00043F0100323614FF430203580FFF7FAFD0C
:1025D00005281EBF236923F01003236170BD00BFCF
:1025E00000200240B0F1904F08B50BD101214FF40B
:1025F000003000F057FD00214FF40030BDE80840E6
:1026000000F050BD1E4B984208D101214FF48020AC
:1026100000F048FD00214FF48020EFE7194B98426D
:1026200008D101214FF4002000F03CFD00214FF4BF
:102630000020E3E7144B984208D101214FF48010A9
:1026400000F030FD00214FF48010D7E70F4B984287
:1026500008D101214FF4001000F024FD00214FF4B7
:102660000010CBE70A4B984208D101214FF48000BB
:1026700000F018FD00214FF48000BFE708BD00BF47
:102680000004004800080048000C00480010004802
:10269000001400482DE9F04100230F681D464FF05B
:1026A000010E03260EFA05FC3CEA070234D10C7930
:1026B000621E012A19D8826806FA03F822EA080283
:1026C00082604A79D0F808809A4042EA0802826023
:1026D000828892B222EA0C0282808A79B0F804C021
:1026E000AA4042EA0C0292B28280D0F800C006FAF8
:1026F00003F2D24302EA0C0CC0F800C0D0F800C0CC
:102700009C4044EA0C040460C4682240C260CA7958
:10271000C4689A402243C2600135102D03F10203C0
:10272000C0D1BDE8F0814FF6FF73036001220023A2
:10273000037142718371C371704741F48033C36187
:10274000C161C361C369C3697047038A194214BF79
:10275000012000207047008A80B27047838A1942A6
:1027600014BF012000207047808A80B270478161C9
:102770007047018570470AB18161704701857047D4
:102780008182704701F00703C90800EB810010B592
:10279000016A9B000F249C4021EA04010162016A46
:1027A0009A400A43026210BD08B50C4B98424FF0A4
:1027B00001010AD14FF4001000F08CFC00214FF40D
:1027C0000010BDE8084000F085BC4FF4800000F028
:1027D00081FC00214FF48000F3E700BF005400406B
:1027E0000368164A23F001030360036810B51A401A
:1027F0008C684B6843EA0423134303600B680A693F
:1028000023F070630361036843F001030360002356
:102810008360C3608B69134383608368CA6843F431
:102820000043836003681343036043684A6923F0ED
:10283000784323F400431343436010BDFFE0CF000F
:1028400000234FF40042036043608360C360036170
:10285000426183617047036819B143F0010303606B
:10286000704723F00103FAE7036823F001030360D4
:102870000368036843F0010303607047036819B1FC
:1028800023F400330360704743F40033FAE703682E
:1028900019B143F480230360704723F48023FAE7DF
:1028A000C36819B143F40043C360704723F4004385
:1028B000FAE7C368120223F4FF6302F4E06201F056
:1028C000FE0123F006030A431A43C26070470368FF
:1028D00019B143F400230360704723F40023FAE79F
:1028E000036819B143F480330360704723F48033E5
:1028F000FAE7436823F47F7323F00303C1F309016C
:102900000B4343607047436819B143F4006343606D
:10291000704723F40063FAE7436819B143F000738A
:102920004360704723F00073FAE7436819B143F03E
:1029300080734360704723F08073FAE7436823F4A1
:102940007F0343EA014141607047436819B923F4AA
:1029500080634360704743F48063FAE7436819B1CA
:1029600043F400534360704723F40053FAE743688D
:1029700019B143F480434360704723F48043FAE77E
:10298000436819B143F480534360704723F4805384
:10299000FAE7436819B123F400434360704743F4F6
:1029A0000043FAE78069000C00F0FE00704783697D
:1029B00013F4803F14BF4FF480600020704730B59F
:1029C0004468039D24F07F7424F45934C1F3090151
:1029D0002B4324F47F74194324F0030441EA024199
:1029E0002143416030BD036819B143F480030360A3
:1029F000704723F48003FAE7436919B143F40043B5
:102A00004361704723F40043FAE7436919B143F087
:102A100000434361704723F00043FAE7436919B16B
:102A200043F480534361704723F48053FAE74369CA
:102A300023F47F6323F00F03C1F30B010B434361C6
:102A400070474269044B22F07F6222F4702203EA4D
:102A500001411143416170470000FF0F036819B144
:102A600043F400030360704723F40003FAE70368AC
:102A700019B143F080630360704723F08063FAE785
:102A8000006AC0B2704782B0002301930190019B9D
:102A900019440191019B186802B070478162704728
:102AA000406AC0B27047036812B1194301607047B1
:102AB00023EA0101FAE7FFF7F6BF83690B4214BF6F
:102AC000012000207047C161704711F47C5F0368EA
:102AD00008D003F080038069084002D0181C18BF9A
:102AE0000120704711F0C00F14BF03F040030B40EA
:102AF000F1E7C161704700BF40F0BF60024B40F496
:102B00000030D860704700BF00ED00E010B5C2781B
:102B10000378E2B1124AD16842788078C943C1F3A0
:102B20000221C1F10404A2400F2424FA01F1014062
:102B30000A430C491201C818D2B280F8002303F0EE
:102B40001F005A090123834041F8223010BD5A0961
:102B5000012103F01F0301FA03F320320149F3E7D7
:102B600000ED00E000E100E021F0604121F07F0194
:102B7000014B01439960704700ED00E0044B1A6976
:102B800011B110431861704722EA0000FAE700BF54
:102B900000ED00E0044B1A6804280CBF42F0040268
:102BA00022F004021A60704710E000E0114B1A682E
:102BB00042F001021A6059680F4A0A405A601A68C6
:102BC00022F0847222F480321A601A6822F4802281
:102BD0001A605A6822F4FE025A60DA6A22F47F52BE
:102BE00022F03F02DA62196B044A0A401A6300229B
:102BF0009A6070470010024000C0FFF8CCFC000F44
:102C0000024B00221A701870704700BF0210024079
:102C1000034A136823F0F80343EAC00010607047CA
:102C200000100240014B1860704700BF0000424294
:102C3000064B1A6A22F001021A621A6A22F0040292
:102C40001A621A6A10431862704700BF00100240EF
:102C5000044B1A6A22F018021A621A6A10431862A8
:102C6000704700BF00100240014B1860704700BF62
:102C700080044242044A536823F474135360536837
:102C8000194301435160704700100240014B186026
:102C9000704700BF60004242034AD36A23F00F032B
:102CA0001843D062704700BF00100240014B18600B
:102CB000704700BF4C004242014B1870704700BF84
:102CC00007100240034A536823F00303184350607F
:102CD000704700BF00100240024B586800F00C0023
:102CE000704700BF00100240034A536823F0F0030E
:102CF00018435060704700BF00100240034A5368F9
:102D000023F4E06318435060704700BF0010024096
:102D1000034A536823F4605343EAC000506070478D
:102D2000001002408E4B5A6802F00C02042AF0B5E3
:102D300078D0082A7AD08B490160002A74D159686A
:102D4000894CC1F3031114F801E001685FFA8EFEAB
:102D500021FA0EF545605E68C6F30226A65D25FAE7
:102D600006F686605F68C7F3C227E75DFFB2FD40E5
:102D7000C560D3F82CC0CCF3041C04EB4C0CBCF89D
:102D800010C01FFA8CFC1CF0100F0EBF0161B2FBCB
:102D9000FCFCC0F810C0D3F82CC0CCF3442C04EBDE
:102DA0004C04248AA4B214F0100F0EBF4161B2FB90
:102DB000F4F444611C6BE4065ABF6A4C846181617F
:102DC0001C6BA4065ABF674CC461C1611C6BE4054F
:102DD00041D58A423FD1BE453DD1540004621C6BAF
:102DE000A4053AD58A4238D1BE4536D14A0042625E
:102DF0001A6B920733D185621A6B12F4403F45D1AA
:102E0000C6621A6B12F4402F5AD106631A6B12F481
:102E1000401F6FD146631A6B12F4400F40F085805B
:102E20008663F0BD514A0260002288E75A685968FB
:102E3000C90349BFD96A4E494C4C01F00F01C2F396
:102E4000834248BF013102F1020248BFB4FBF1F1F5
:102E50004A43026073E70562C1E74562C8E71A6B3F
:102E600002F00302012A01D18162C5E71A6B02F068
:102E70000302022A03D14FF400428262BCE71A6BBC
:102E800002F00302032AB7D1364AF6E71A6B02F4BE
:102E90004032B2F5803F01D1C162B2E71A6B02F451
:102EA0004032B2F5003F03D14FF40042C262A8E7BE
:102EB0001A6B02F44032B2F5403FA2D1294AF5E73D
:102EC0001A6B02F44022B2F5802F01D101639DE715
:102ED0001A6B02F44022B2F5002F03D14FF40042E6
:102EE000026393E71A6B02F44022B2F5402F8DD1B2
:102EF0001C4AF5E71A6B02F44012B2F5801F01D1AB
:102F0000416388E71A6B02F44012B2F5001F03D147
:102F10004FF4004242637EE71A6B02F44012B2F5AE
:102F2000401F7FF478AF0F4AF4E71A6B02F44002B7
:102F3000B2F5800F01D18163F0BD1A6B02F440023B
:102F4000B2F5000F03D14FF400438363F0BD1B6B58
:102F500003F44003B3F5400FF8D1024BF5E700BF8F
:102F60000010024000127A00780000200024F400D3
:102F700000093D00030F064BDA6A14BF22F47852B1
:102F800022F4F872DA62DA6A1043D862704700BF3E
:102F900000100240030F064B1A6B14BF22F02002F0
:102FA00022F010021A631A6B10431863704700BFB7
:102FB00000100240030F064B1A6B14BF22F400727C
:102FC00022F480721A631A6B10431863704700BFB3
:102FD00000100240020F013A0F4B042A08D8DFE824
:102FE00002F0030B0F1317001A6B22F003021A638F
:102FF0001A6B1043186370471A6B22F44032F6E7DD
:103000001A6B22F44022F2E71A6B22F44012EEE728
:103010001A6B22F44002EAE700100240014B1860EC
:10302000704700BFD8004242024A136A1843106238
:10303000704700BF00100240014B1860704700BF8E
:10304000DC004242014B1860704700BF3C04424222
:10305000014B1860704700BF40044242044B5A695C
:1030600011B110435861704722EA0000FAE700BF2F
:1030700000100240044B9A6911B1104398617047E7
:1030800022EA0000FAE700BF00100240044BDA69B0
:1030900011B11043D861704722EA0000FAE700BF7F
:1030A00000100240044B9A6A11B1104398627047B5
:1030B00022EA0000FAE700BF00100240044BDA6881
:1030C00011B11043D860704722EA0000FAE700BF50
:1030D00000100240044B1A6911B110431861704787
:1030E00022EA0000FAE700BF00100240044B1A7801
:1030F00011B110431870704722EA0000FAE700BFD0
:10310000091002404209094B07D11B6800F01F005B
:1031100023FA00F000F001007047012A01D11B6A78
:10312000F4E7042A0CBF5B685B6AEFE7001002401B
:1031300007B5002301931120FFF7E4FF019B013342
:103140000193019BB3F5A06F01D00028F3D01120AB
:10315000FFF7D8FF003018BF012003B05DF804FB73
:10316000024A536A43F08073536270470010024072
:10317000034B9B68184214BF01200020704700BF1A
:1031800000100240014B1870704700BF0A10024047
:1031900000230928DAB203F1010303D840EA021040
:1031A000C0B270470A38C0B2F3E7030903EB8303E8
:1031B00000F00F0000EB4300C0B2704700217F22F7
:1031C000FF2380E80E007047044B10B1FF225A62C3
:1031D0007047CA225A625322F9E700BF0028004014
:1031E00082B0002301930D4BDA68520614D44FF0DD
:1031F000FF32DA601846DA680199013101910199CC
:10320000B1F5005F02F0400201D0002AF3D0C0689F
:10321000C0F3801002B070470120FBE70028004097
:10322000024AD36823F08003D3607047002800402F
:1032300038B50F4CCA236362532363620546FFF718
:10324000CFFF88B1A36823F04003A360A3682A6876
:103250001343A360AB68236123696A6843EA0243AE
:103260002361FFF7DDFF0120014BFF225A6238BDC9
:103270000028004013B500230193114B9A68920671
:103280001BD4CA225A6253225A62DA6822F0A00280
:10329000DA601C46DA680199013101910199B1F5B2
:1032A000004F02F0200201D0002AF3D0E068FF2393
:1032B000C0F34010636202B010BD0120FBE700BF05
:1032C0000028004037B51F4CCA23002501956362D2
:1032D00053236362FFF784FF28B90020194BFF22B4
:1032E0005A6203B030BD42F2011325606360A368E7
:1032F00003F00703A3602346E268019901310191BD
:103300000199B1F5005F02F0040201D0002AF3D068
:10331000DA685207E1D59A684FF6FF7100229A6089
:10332000596109491961DA611A62DA62DA635A6429
:103330009A64DA601A64FFF79DFF003018BF01201D
:10334000CCE700BF00280040FF007F0038B50B4CE1
:10335000CA236362532363620546FFF741FF38B116
:10336000A36845B143F01003A360FFF759FF0120A4
:10337000FF23636238BD23F01003F5E70028004007
:10338000074BCA225A6253225A629A6828B142F005
:1033900020029A60FF225A62704702F0DF02F8E7CB
:1033A00000280040224B0A789B6870B54D788C78D5
:1033B000B0B913F0400300D1CB701046FFF7E8FE20
:1033C00006462846FFF7E4FE05462046FFF7E0FEE6
:1033D000CB7840EA034040EA064040EA05240AE090
:1033E00013F0400300D1CB70280240EA0240204392
:1033F000CC7840EA04440E4DCA236B6253236B62BF
:10340000FFF7EEFE70B104F07F3424F0FE442C6030
:10341000FFF706FFAB689B0608D4FFF72BFF0030D1
:1034200018BF0120024BFF225A6270BD0120F9E74C
:10343000002800400023C3700370437083707047FE
:10344000104B70B51C6804F07F3323F0FE431D0C55
:1034500005F03F06C3F3062204F07F0405F04005A3
:103460000E704A708C70CD7058B93046FFF79DFED3
:1034700008701046FFF799FE48702046FFF795FE4A
:10348000887070BD00280040014B986A5B687047E7
:103490000028004070B54B78CA788D780C780028E9
:1034A00033D1D80603D523F010030A334B701046EE
:1034B000FFF76EFE06464878FFF76AFE014628468B
:1034C000FFF766FE40EA443040EA064040EA012445
:1034D000114DCA236B6253236B62FFF781FE70B1FB
:1034E00024F07F4424F0C0046C60FFF799FEAB68C1
:1034F0009B0608D4FFF7BEFE003018BF0120064B24
:10350000FF225A6270BD0120F9E7180240EA02402A
:10351000284340EA4434DBE70028004001230370DD
:10352000837043700023C370704738B50F4B5A68DF
:1035300022F07F4323F0C0031D0CC3F3042402F0E8
:103540003F02C3F34233CD704C708A700B7058B990
:103550002846FFF72AFEC8702046FFF726FE48706F
:103560001046FFF722FE887038BD00BF00280040DB
:103570002DE9F047264B9468D2F804A0977892F88A
:1035800000E092F80180167B154600BB9B6813F0A3
:10359000400300D1D3707046FFF7FAFD81464046E4
:1035A000FFF7F6FD80463846FFF7F2FD0746304646
:1035B000FFF7EEFDEB7844EA0A0444EA03433B4399
:1035C00043EA094343EA082343EA006010E09A68AB
:1035D00012F0400200D1EA7044EA0A00384340EA9F
:1035E0000E40EB7840EA082040EA034040EA0660DB
:1035F000074BCA225A6253225A62B1F5807F4FF0BC
:10360000FF020CBFD86118625A62BDE8F08700BFA4
:103610000028004000230122C370037043708370B0
:103620008360027343607047F8B5174BB1F5807F34
:103630000CBFDB691B6AC3F30741064601F03F007C
:1036400001F04001C3F3062503F07F0403F0804737
:10365000D170C3F3056103F080331070557094701E
:1036600011739760536076B9FFF79FFD107028467D
:10367000FFF79BFD50702046FFF797FD90700846BE
:10368000FFF793FD1073F8BD0028004013B5002329
:103690000193134BCA225A6253225A629A6839B173
:1036A0001043986001200E4BFF225A6202B010BDF9
:1036B00022EA00029A60000A1C46DA680199013188
:1036C00001910199B1F5005F02EA000205D1E368BA
:1036D000184214BF01200020E5E7002AEDD0F6E7EC
:1036E0000028004010B5074BCA245C620A43B0F5BD
:1036F000807F4FF053045C620CBF5A649A64FF22CF
:103700005A6210BD00280040044BB0F5807F0CBF0A
:10371000586C986CC0F30E00704700BF0028004042
:10372000074BCA225A6253225A629A6822F0070251
:103730009A609A681043FF2298605A62704700BFEF
:1037400000280040044BCA225A6253225A62FF22C8
:1037500058615A62704700BF00280040014B586909
:1037600080B270470028004082B000230193124BC2
:10377000CA225A6253225A629A6840B142F4806265
:103780009A6001200C4BFF225A6202B0704722F46B
:1037900080629A601846DA680199013101910199B5
:1037A000B1F5005F02F0040201D0002AF3D0C06836
:1037B000C0F38000E6E700BF00280040074BCA22A4
:1037C0005A6253225A629A6822F480229A609A6856
:1037D00011430143FF2299605A627047002800405C
:1037E000024B986800F48020704700BF002800401A
:1037F000074BCA225A6253225A629A6822F4E002A4
:103800009A609A6811430143FF2299605A62704797
:1038100000280040074BCA225A6253225A629A6813
:1038200028B142F400029A60FF225A62704722F4E3
:103830000002F8E700280040074BCA225A625322D0
:103840005A629A6822F400229A609A681043FF2212
:1038500098605A62704700BF002800400E4B30B598
:10386000CA245C6253245C62DC68E40306D541F23E
:103870000104DD68ED0301D5013CFAD1064BDC689B
:10388000E4035CBF114308434FF0FF0256BFD86307
:10389000002001205A6230BD00280040084A936889
:1038A00023F4006323F0080309B143F40063CA2141
:1038B00051620343532151629360FF235362704767
:1038C00000280040204B2DE9F0411E6B5D6B06F097
:1038D0007F3727F0FE473C0C25F07F4304F03F0E76
:1038E00004F04004CC7023F0C0030024C7F3062783
:1038F00006F07F0681F800E04F708E70C3F3042855
:10390000D47005F03F05C3F3423482F8018095700E
:103910001470B8B97046FFF748FC08703846FFF7D6
:1039200044FC48703046FFF740FC88704046FFF783
:103930003CFC50702846FFF738FC90702046FFF79B
:1039400034FC1070BDE8F08100280040014B986BFA
:10395000704700BF00280040044B40001A6C19B9A2
:1039600022EA0000186470471043FBE7002800407B
:10397000044B1A6C11B110431864704722EA00001E
:10398000FAE700BF00280040044B1A6C22F4C05232
:103990001A641A6C10431864704700BF0028004076
:1039A000044B1A6C22F4E0621A641A6C1043186417
:1039B000704700BF00280040044B1A6C22F4C0423C
:1039C0001A641A6C10431864704700BF0028004046
:1039D000044B1A6C18B142F080021A64704722F04E
:1039E0008002FAE700280040044B1A6C18B122F458
:1039F00000421A64704742F40042FAE7002800408F
:103A000082B000230193054B0193019B03EB8000DF
:103A10000190019B196002B0704700BF5028004020
:103A200082B000230193054B0193019B03EB8000BF
:103A30000190019B186802B0704700BF50280040F9
:103A4000044B1A6C22F480221A641A6C1043186416
:103A5000704700BF00280040134BCA2210B55A62BD
:103A600053225A62DA68120706D542F20102DC6874
:103A7000240701D5013AFAD10B4AD36813F00803A1
:103A80000DD19468E4060CD40143D162FFF7F2FB38
:103A9000003018BF0120044BFF225A6210BD0020E5
:103AA000F9E71846F7E700BF002800400D4BCA228F
:103AB0005A6253225A6220F0040200F0040049B115
:103AC00099680A439A601A6C10431864054BFF22E8
:103AD0005A627047996821EA02029A601A6C22EAD7
:103AE0000000F2E700280040044BDA68044B134062
:103AF000034214BF01200020704700BF002800408F
:103B00007FFF01000549064ACB68024042F080026F
:103B100003F0800363EA0203CB6070470028004093
:103B20007FFF01000B490B6C8A68C96810B5840CD3
:103B300020FA04F403F0040303EAD43302401343ED
:103B400006D08BB213EA101314BF0120002010BD61
:103B5000184610BD00280040054AD368C0F30F1076
:103B600040F0800003F0800363EA0003D3607047F5
:103B70000028004008B5154B98420BD101214FF4A5
:103B80008050FFF79BFA00214FF48050BDE80840B9
:103B9000FFF794BA0E4B98420BD101214FF48040AD
:103BA000FFF798FA00214FF48040BDE80840FFF786
:103BB00091BA084B984208D101214FF40040FFF719
:103BC00089FA00214FF40040EFE708BD00300140C2
:103BD00000380040003C00400023038043804FF445
:103BE000E062C380038143818381C3810723828094
:103BF000038270472DE9F0474C88B1F800A0B1F876
:103C00000680B1F808C0B1F80AE08F89CE898D88A6
:103C1000B4F5827F22D1028802F4415242EA0A02BC
:103C200042F4827242EA080343EA0C0343EA0E03B9
:103C30003B4333439BB20380838823F470631B04AC
:103C40001B0C1D43ADB28580838B23F400631B04E2
:103C50001B0C83830B8A0382BDE8F087B0F80490C5
:103C600029F470694FEA09494FEA194949EA0505FB
:103C7000ADB28580038803F44153234343EA0A032A
:103C800043EA080343EA0C0343EA0E033B4333438E
:103C90009BB20380D8E70023022203804380838005
:103CA000C380826083817047838B23F47B6323F01E
:103CB0000F031B04F0B51B0C8383022303848B6862
:103CC000868B022B91B005460C46B6B239D08B8854
:103CD00001A8002B14BF02270127FFF723F8E38870
:103CE0000199A068B3F5007F4FF00A0216BF7B016F
:103CF0000B0AB1FBF3F35343B3FBF0F305330A2292
:103D00009BB2B3FBF2F303F001021202C3F34F03C1
:103D1000991E89B2FE2924BF002202231343E288A0
:103D200013439BB262882B8423881343A28843F4F5
:103D300000631343A28913431E43B6B2AE8311B08E
:103D4000F0BD0022E4E7038821B19BB243F04003B9
:103D50000380704723F040031B041B0CF8E78388A3
:103D600021B19BB243F010038380704723F010030E
:103D70001B041B0CF8E7838B21B19BB243F48063D7
:103D80008383704723F480631B041B0CF8E783884C
:103D900023F470631B041B0C1943818070478388D4
:103DA00023F480531B041B0C838083889BB219432C
:103DB000818070470388B1F5804F15BF23F480439D
:103DC0009BB21B0443F4804318BF1B0C0380704755
:103DD0004FF6FF63994203880BBF23F480739BB2B5
:103DE0001B0443F4807308BF1B0C03807047838B54
:103DF0000A8823F47B6323F00F031B041B0C8383CB
:103E00000223038430B54B888D888989848B2B43AA
:103E100022F4007243F4006392B20B43002A43EA97
:103E200004030CBF4FF4807200229BB213438383C0
:103E300030BD838821B19BB243F004038380704777
:103E400023F004031B041B0CF8E7838821B19BB209
:103E500043F008038380704723F008031B041B0C06
:103E6000F8E70173704781817047007B7047808954
:103E700080B27047038823F400631B041B0C03808B
:103E800003889BB2194301807047038821B19BB21C
:103E900043F400530380704723F400531B041B0CAE
:103EA000F8E703889BB243F48053038070470129ED
:103EB00014BF008B808A80B27047008A80B270473E
:103EC00083889BB212B119438180704723EA0101B4
:103ED000FAE7838823F4C0431B041B0C8380838888
:103EE0009BB21943818070470B0901219940838857
:103EF00089B29BB212B119438180704723EA010154
:103F0000FAE7008900F4C0507047008900F4C060EF
:103F100070470389194214BF012000207047C9432C
:103F200089B20181704710B58488008901F00F02C1
:103F3000012380B203FA02F21040A4B205D00909AD
:103F40008B401C4214BF0120002010BD084B1A6892
:103F500002F003021A601A6842F0F8421A60002266
:103F60005A609A60DA601A615A619A61704700BFBC
:103F700000000140034A136823F003031843106054
:103F8000704700BF00000140044B1A6822F4400251
:103F90001A601A6810431860704700BF00000140A3
:103FA000014B1860704700BF14002042044B1A6890
:103FB00011B110431860704722EA0000FAE700BF11
:103FC00000000140FFF7F2BFFFF7F0BFFFF7EEBFC1
:103FD00001F0030301F0FC0101F1804101F58031A2
:103FE00010B58A689B000F249C4022EA04028A6074
:103FF0008A6898401043886010BD024B01221A6005
:10400000704700BF10032042024A536818435060B3
:10401000704700BF00000140024B9869C0F30020C8
:10402000704700BF00000140024A93691843906145
:10403000704700BF00000140FFF7F6BF30B5046ACB
:1040400024F0010404628569046A25F0F30542EA5C
:10405000031324F00A0441F001012B43214383613F
:10406000016230BD30B5046A24F010042404240C2D
:1040700004628569046A090124F0A0041202240480
:1040800041F0100125F4734542EA0333240C89B250
:104090002B4321438361016230BD08B53A4B9842FE
:1040A0000BD101214FF40060FFF708F800214FF415
:1040B0000060BDE80840FFF701B8B0F1804F09D1BA
:1040C00001210846FFF706F800210120BDE808405D
:1040D000FFF700B82D4B984206D101210220FEF7D0
:1040E000F9FF00210220F1E7294B984206D1012176
:1040F0000420FEF7EFFF00210420E7E7254B98425C
:1041000006D101211020FEF7E5FF00211020DDE798
:10411000214B984206D101212020FEF7DBFF002130
:104120002020D3E71D4B984208D101214FF40050C5
:10413000FEF7C4FF00214FF40050BAE7184B984235
:1041400008D101214FF48030FEF7B8FF00214FF471
:104150008030AEE7134B984208D101214FF4003074
:10416000FEF7ACFF00214FF40030A2E70E4B98425F
:1041700008D101214FF48020FEF7A0FF00214FF469
:10418000802096E708BD00BF002C014000040040DD
:1041900000080040001000400014004000340140BE
:1041A000004001400044014000480140204A03888B
:1041B00090429BB20ED002F5006290420AD0B0F15C
:1041C000804F07D0A2F59832904203D002F580626A
:1041D000904203D14A8823F070031343154A90425A
:1041E00008D002F5806290421FBF23F440730A8911
:1041F0009BB2134303804B68C3620B8803850C4B4F
:1042000098420FD003F5006398420BD003F540634A
:10421000984207D003F58063984203D003F580638A
:10422000984201D18B7A038601234361704700BF16
:10423000002C0140001000404FF0FF33436000238A
:104240000380038143808372704701854261704718
:10425000038823F070031B041B0C19430180704773
:1042600041627047C1627047406A7047008D80B2FA
:104270007047038821B19BB243F00203038070476B
:1042800023F002031B041B0CF8E7038821B19BB247
:1042900043F004030380704723F004031B041B0C4A
:1042A000F8E7038821B19BB243F4006303807047B1
:1042B00023F400631B041B0CF8E7038821B19BB2B5
:1042C00043F080030380704723F080031B041B0C22
:1042D000F8E7038823F008031B041B0C0380038802
:1042E0009BB2194301807047038823F440731B0479
:1042F0001B0C038003889BB219430180704703881D
:1043000021B19BB243F001030380704723F0010306
:104310001B041B0CF8E7036A23F00103036270B56A
:10432000056A426884690B688E8824F4803424F01E
:1043300073041C438B89334325F002059BB22B4346
:10434000134DA8420FD005F50065A8420BD005F526
:104350004065A84207D005F58065A84203D005F561
:104360008065A8420ED123F00805CB894E8A2B43E5
:10437000CD8823F004032B4322F440750A8A32438C
:1043800092B22A4342608A6884614263036270BDCC
:10439000002C0140036A23F010030362036A4268A1
:1043A00030B584690D6824F0807424F4E64444EA4E
:1043B00005248D8923F0200343EA05138D8843EA01
:1043C00005130F4DA84203D005F50065A84211D191
:1043D000CD8923F0800343EA0513CD8823F0400301
:1043E00043EA05130D8A22F4406242EA85024D8AAF
:1043F00042EA850242608A6884618263036230BD5A
:10440000002C0140036A23F480730362036A42684C
:1044100030B5C4690D6824F073042C438D8923F4EE
:10442000007343EA05238D8843EA05230F4DA84214
:1044300003D005F50065A84211D1CD8923F40063AE
:1044400043EA0523CD8823F4806343EA05230D8ADC
:1044500022F4405242EA05124D8A42EA05124260B5
:104460008A68C461C263036230BD00BF002C014092
:10447000036A23F480530362036A30B54468C26957
:104480000D6822F4E64242EA05228D8923F40053A6
:1044900043EA05338D8843EA0533094DA84203D02A
:1044A00005F50065A84204D10D8A24F4804444EA4D
:1044B00085144460C2618A680264036230BD00BF33
:1044C000002C0140036A23F480330362036A30B591
:1044D0004468426D0D6822F070022A438D8923F4EE
:1044E000003343EA05438D8843EA0543084DA8425B
:1044F00003D005F50065A84204D10D8A24F4803468
:1045000044EA0544446042658A688265036230BDBE
:10451000002C0140036A23F480130362036A30B560
:104520004468426D0D6822F4E04242EA05228D891A
:1045300023F4001343EA05538D8843EA0553074DDE
:10454000A84203D005F50065A84201D124F4003447
:10455000446042658A68C265036230BD002C014038
:10456000836D19B143F000538365704723F0005306
:10457000FAE7836D19B143F080438365704723F0F8
:104580008043FAE7836D19B143F0004383657047B8
:1045900023F00043FAE7002303608380C380836035
:1045A0008381C38103824382704701238B4030B5EE
:1045B000DB43056A9BB22B40036221F0080300F144
:1045C000180453B949080B5923F4803323F07003BE
:1045D0000B510B591A430A5130BD043949081202D4
:1045E0000B5923F0807323F4E0430B5192B20B5923
:1045F000F0E74163704781637047C16370470164AE
:10460000704781657047C1657047836923F48033C3
:1046100023F07003194381617047836923F080732D
:1046200023F4E04343EA012181617047C36923F029
:1046300070031943C1617047C36923F4E04343EA3F
:104640000121C1617047436D23F070031943416537
:104650007047436D23F4E04343EA0121416570470D
:10466000836923F00803194381617047836923F448
:10467000006343EA012181617047C36923F00803A5
:104680001943C1617047C36923F4006343EA012100
:10469000C1617047436D23F00803194341657047BA
:1046A000436D23F4006343EA012141657047836948
:1046B00023F00403194381617047836923F4806305
:1046C00043EA012181617047C36923F00403194360
:1046D000C1617047C36923F4806343EA0121C1616A
:1046E0007047836923F080031943816170478369B0
:1046F00023F4004343EA012181617047C36923F039
:1047000080031943C1617047C36923F4004343EA3E
:104710000121C1617047436D23F080031943416556
:104720007047436D23F4004343EA0121416570471C
:10473000836823F008031B041B0C83608368194300
:1047400081607047036A23F00203194301627047D6
:10475000036A23F00803194301627047036A23F0D8
:10476000200343EA011101627047036A23F08003CA
:1047700043EA011101627047036A23F4007343EABC
:10478000012101627047036A23F4006343EA0121B7
:1047900001627047036A23F4005343EA0131016266
:1047A0007047036A23F4003343EA01410162704712
:1047B000036A23F4001343EA015101627047036A5C
:1047C00010B501248C4023EA04030362036A8A4083
:1047D0001A43026210BD036A10B504248C4023EA18
:1047E00004030362036A8A401A43026210BD002375
:1047F0000122038043808280C38003817047406B25
:104800007047806B7047C06B7047006C704783695E
:1048100023F00C03836183691943816170478369C5
:1048200023F440638361836943EA01218161704716
:10483000F8B50C464988A288B4F800E0238900291D
:104840000CBF02260026012A0CBF02270127BEF159
:10485000000F0ED1FFF7F2FBE188FFF7D8FF3146DA
:1048600023893A46FFF7FEFBE188BDE8F840FFF7F1
:10487000D6BFFFF7F7FBE188FFF7D1FF3146238969
:104880003A46FFF7DBFBE188BDE8F840FFF7BFBF22
:10489000C36923F00C031B041B0CC361C3691943D8
:1048A000C1617047C36923F440631B041B0CC361DF
:1048B000C369090289B21943C1617047F8B50E880E
:1048C0000B898A880D46498836B9FFF7B7FBE98816
:1048D000BDE8F840FFF79BBF042E06D1FFF7C2FBEF
:1048E000E988BDE8F840FFF79ABF082EEF88056A0F
:1048F0001CD125F480752D042D0C0562C669056A4E
:10490000B6B2ADB226F0F30646EA031625F42063EC
:1049100043EA0123B6B29BB2324343F48073C261CF
:1049200039460362BDE8F840FFF7B2BF25F4805571
:104930002D042D0C0562C669056A26F4407625F41F
:10494000005536056D04360D6D0C46EA022245EA27
:10495000013189B242EA03339BB241F48051C36111
:1049600001623946BDE8F840FFF79CBF4A880B88D2
:1049700013438A881343CA8813430A8913434A8915
:1049800013438A8913439BB243647047436C23F4F7
:1049900072234364436C43EA02420A434264704711
:1049A000436C23F03C734364436C43EA02520A4372
:1049B00042647047436C19B143F4805343647047B9
:1049C00023F48053FAE7436C19B143F080734364D6
:1049D000704723F08073FAE70023038043808380CD
:1049E000C3800381438183817047436C19B143F4D1
:1049F000004343647047C3F30E03FAE7436819B1F9
:104A000043F004034360704723F004031B041B0CB2
:104A1000F8E7436819B143F001034360704723F09E
:104A200001031B041B0CF8E74161704703690B424B
:104A300014BF012000207047C94389B2016170474B
:104A40000369C26811EA030003D0114214BF0120B8
:104A500000207047C94389B2016170470A43A0F83A
:104A600048207047C36812B11943C1607047C943F9
:104A700089B21940F9E7FFF7F5BF436819B143F070
:104A800008034360704723F008031B041B0CF8E77E
:104A9000836823F007031B041B0C83607047826844
:104AA0004FF68F73134019438160836843F0070307
:104AB0008360704738B50D46602D114604464FF0AF
:104AC00001020CD1FFF7CEFAA2684FF68F731340A4
:104AD0001D43A560A36843F00703A36038BDFFF73B
:104AE000ADFAF1E782684FF68F7313401943816086
:104AF0007047436823F070031B041B0C436043683A
:104B0000194341607047436823F47003436043686E
:104B1000194341607047836823F4803323F007030F
:104B200083608368194381607047836823F0800342
:104B30001B041B0C8360836819438160704710B5A8
:104B400084680A43E4B242EA03231C43A4B28460AB
:104B500010BD10B5FFF7F3FF836823F077039BB216
:104B600043F07703836010BD10B5FFF7E8FF83685B
:104B700043F48043836010BDF0B585688469076A9B
:104B80004FF6F8762E404FF6FC4525404FF6DD7483
:104B90003C4042EA031345F480751C43314345F021
:104BA0000105A4B2816085610462F0BD436819B15A
:104BB00043F080034360704723F080031B041B0C09
:104BC000F8E7A0F85010704781F0004102E000BF04
:104BD00083F0004330B54FEA41044FEA430594EABD
:104BE000050F08BF90EA020F1FBF54EA000C55EAF8
:104BF000020C7FEA645C7FEA655C00F0E2804FEAC9
:104C00005454D4EB5555B8BF6D420CDD2C4480EAAA
:104C1000020281EA030382EA000083EA010180EADA
:104C2000020281EA0303362D88BF30BD11F0004F28
:104C30004FEA01314FF4801C4CEA113102D040425E
:104C400061EB410113F0004F4FEA03334CEA133399
:104C500002D0524263EB430394EA050F00F0A780B1
:104C6000A4F10104D5F1200E0DDB02FA0EFC22FAAC
:104C700005F2801841F1000103FA0EF2801843FAA0
:104C800005F359410EE0A5F120050EF1200E012A91
:104C900003FA0EFC28BF4CF0020C43FA05F3C018CF
:104CA00051EBE37101F0004507D54FF0000EDCF148
:104CB000000C7EEB00006EEB0101B1F5801F1BD3F1
:104CC000B1F5001F0CD349085FEA30004FEA3C0CF5
:104CD00004F101044FEA445212F5800F80F09A80EB
:104CE000BCF1004F08BF5FEA500C50F1000041EBEF
:104CF000045141EA050130BD5FEA4C0C404141EBF3
:104D0000010111F4801FA4F10104E9D191F0000F19
:104D100004BF01460020B1FA81F308BF2033A3F19C
:104D20000B03B3F120020CDA0C3208DD02F1140C93
:104D3000C2F10C0201FA0CF021FA02F10CE002F1CE
:104D40001402D8BFC2F1200C01FA02F120FA0CFCC7
:104D5000DCBF41EA0C019040E41AA2BF01EB045110
:104D6000294330BD6FEA04041F3C1CDA0C340EDC0E
:104D700004F11404C4F1200220FA04F001FA02F351
:104D800040EA030021FA04F345EA030130BDC4F10F
:104D90000C04C4F1200220FA02F001FA04F340EA04
:104DA0000300294630BD21FA04F0294630BD94F0B5
:104DB000000F83F4801306BF81F480110134013D9C
:104DC0004EE77FEA645C18BF7FEA655C29D094EA0D
:104DD000050F08BF90EA020F05D054EA000C04BF8B
:104DE0001946104630BD91EA030F1EBF0021002076
:104DF00030BD5FEA545C05D14000494128BF41F015
:104E0000004130BD14F580043CBF01F5801130BD78
:104E100001F0004545F0FE4141F470014FF0000003
:104E200030BD7FEA645C1ABF194610467FEA655CB4
:104E30001CBF0B46024650EA013406BF52EA033556
:104E400091EA030F41F4002130BD00BF90F0000F44
:104E500004BF0021704730B54FF4806404F1320480
:104E60004FF000054FF0000150E700BF90F0000F39
:104E700004BF0021704730B54FF4806404F1320460
:104E800010F0004548BF40424FF000013EE700BF30
:104E900042004FEAE2014FEA31014FEA02701FBFC0
:104EA00012F07F4393F07F4F81F06051704792F092
:104EB000000F14BF93F07F4F704730B54FF460740C
:104EC00001F0004521F0004120E700BF50EA010257
:104ED00008BF704730B54FF000050AE050EA010204
:104EE00008BF704730B511F0004502D5404261EB74
:104EF00041014FF4806404F132045FEA915C3FF4B5
:104F0000DCAE4FF003025FEADC0C18BF03325FEA4D
:104F1000DC0C18BF033202EBDC02C2F1200300FA02
:104F200003FC20FA02F001FA03FE40EA0E0021FA27
:104F300002F11444C1E600BF70B54FF0FF0C4CF411
:104F4000E06C1CEA11541DBF1CEA135594EA0C0FC7
:104F500095EA0C0F00F0DEF82C4481EA030621EA02
:104F60004C5123EA4C5350EA013518BF52EA03353D
:104F700041F4801143F4801338D0A0FB02CE4FF0EF
:104F80000005E1FB02E506F00042E0FB03E54FF01F
:104F90000006E1FB03569CF0000F18BF4EF0010E17
:104FA000A4F1FF04B6F5007F64F5407404D25FEA13
:104FB0004E0E6D4146EB060642EAC62141EA5551C6
:104FC0004FEAC52040EA5E504FEACE2EB4F1FD0C08
:104FD00088BFBCF5E06F1ED8BEF1004F08BF5FEA86
:104FE000500E50F1000041EB045170BD06F0004638
:104FF00046EA010140EA020081EA0301B4EB5C04E5
:10500000C2BFD4EB0C0541EA045170BD41F48011DC
:105010004FF0000E013C00F3AB8014F1360FDEBF01
:10502000002001F0004170BDC4F10004203C35DADD
:105030000C341BDC04F11404C4F1200500FA05F360
:1050400020FA04F001FA05F240EA020001F0004201
:1050500021F0004110EBD37021FA04F642EB060177
:105060005EEA430E08BF20EAD37070BDC4F10C04A1
:10507000C4F1200500FA04F320FA05F001FA04F265
:1050800040EA020001F0004110EBD37041F1000151
:105090005EEA430E08BF20EAD37070BDC4F120055C
:1050A00000FA05F24EEA020E20FA04F301FA05F2C4
:1050B00043EA020321FA04F001F0004121FA04F26C
:1050C00020EA020000EBD3705EEA430E08BF20EA3C
:1050D000D37070BD94F0000F0FD101F00046400076
:1050E00041EB010111F4801F08BF013CF7D041EAF8
:1050F000060195F0000F18BF704703F000465200FC
:1051000043EB030313F4801F08BF013DF7D043EACC
:105110000603704794EA0C0F0CEA135518BF95EA82
:105120000C0F0CD050EA410618BF52EA4306D1D109
:1051300081EA030101F000414FF0000070BD50EA28
:10514000410606BF1046194652EA430619D094EAB2
:105150000C0F02D150EA013613D195EA0C0F05D19C
:1051600052EA03361CBF104619460AD181EA0301F0
:1051700001F0004141F0FE4141F470014FF00000A8
:1051800070BD41F0FE4141F4780170BD70B54FF043
:10519000FF0C4CF4E06C1CEA11541DBF1CEA1355C3
:1051A00094EA0C0F95EA0C0F00F0A7F8A4EB0504A5
:1051B00081EA030E52EA03354FEA013100F088809C
:1051C0004FEA03334FF0805545EA131343EA126365
:1051D0004FEA022245EA111545EA10654FEA00261A
:1051E0000EF000419D4208BF964244F1FD0404F5D3
:1051F000407402D25B084FEA3202B61A65EB03052F
:105200005B084FEA32024FF480104FF4002CB6EBEB
:10521000020E75EB030E22BFB61A754640EA0C006B
:105220005B084FEA3202B6EB020E75EB030E22BFAB
:10523000B61A754640EA5C005B084FEA3202B6EBEC
:10524000020E75EB030E22BFB61A754640EA9C00AB
:105250005B084FEA3202B6EB020E75EB030E22BF7B
:10526000B61A754640EADC0055EA060E18D04FEA39
:10527000051545EA16754FEA06164FEAC30343EAD9
:1052800052734FEAC2025FEA1C1CC0D111F4801FA6
:105290000BD141EA00014FF000004FF0004CB6E79F
:1052A00011F4801F04BF01430020B4F1FD0C88BF3E
:1052B000BCF5E06F3FF6AFAEB5EB030C04BFB6EB49
:1052C000020C5FEA500C50F1000041EB045170BD3C
:1052D0000EF0004E4EEA113114EB5C04C2BFD4EB69
:1052E0000C0541EA045170BD41F480114FF0000EED
:1052F000013C90E645EA060E8DE60CEA135594EA69
:105300000C0F08BF95EA0C0F3FF43BAF94EA0C0F6B
:105310000AD150EA01347FF434AF95EA0C0F7FF4E0
:1053200025AF104619462CE795EA0C0F06D152EA34
:1053300003353FF4FDAE1046194622E750EA410618
:1053400018BF52EA43067FF4C5AE50EA41047FF429
:105350000DAF52EA43057FF4EBAE12E74FEA41028C
:1053600012F5001215D211D56FF47873B3EB6252B7
:1053700012D94FEAC12343F0004343EA505311F0DE
:10538000004F23FA02F018BF404270474FF0000070
:10539000704750EA013005D111F0004008BF6FF0AE
:1053A000004070474FF00000704700BF4FEA4102D5
:1053B000B2F1E04324BFB3F5001CDCF1FE5C0DD973
:1053C00001F0004C4FEAC0024CEA5070B2F1004FBD
:1053D00040EB830008BF20F00100704711F0804FC0
:1053E00021D113F13872BCBF01F00040704741F485
:1053F00080114FEA5252C2F11802C2F1200C10FA89
:105400000CF320FA02F018BF40F001004FEAC1236C
:105410004FEAD32303FA0CFC40EA0C0023FA02F310
:105420004FEA4303CCE77FEA625307D150EA0133E6
:105430001EBF4FF0FE4040F44000704701F00040B6
:1054400040F0FE4040F40000704700BF80F0004094
:1054500002E000BF81F0004142001FBF5FEA41034C
:1054600092EA030F7FEA226C7FEA236C6AD04FEA4C
:105470001262D2EB1363C1BFD21841404840414091
:10548000B8BF5B42192B88BF704710F0004F40F443
:10549000000020F07F4018BF404211F0004F41F45F
:1054A000000121F07F4118BF494292EA030F3FD02B
:1054B000A2F1010241FA03FC10EB0C00C3F120033E
:1054C00001FA03F100F0004302D5494260EB4000CD
:1054D000B0F5000F13D3B0F1807F06D340084FEA38
:1054E000310102F10102FE2A51D2B1F1004F40EB2D
:1054F000C25008BF20F0010040EA03007047490095
:1055000040EB000010F4000FA2F10102EDD1B0FA5F
:1055100080FCACF1080CB2EB0C0200FA0CF0AABF54
:1055200000EBC25052421843BCBFD04018437047F2
:1055300092F0000F81F4000106BF80F400000132F8
:10554000013BB5E74FEA41037FEA226C18BF7FEACF
:10555000236C21D092EA030F04D092F0000F08BF11
:105560000846704790EA010F1CBF0020704712F0F8
:105570007F4F04D1400028BF40F00040704712F137
:1055800000723CBF00F50000704700F0004343F09C
:10559000FE4040F4000070477FEA226216BF0846D2
:1055A0007FEA23630146420206BF5FEA412390EA95
:1055B000010F40F4800070474FF0000304E000BF8B
:1055C00010F0004348BF40425FEA000C08BF70473C
:1055D00043F0964301464FF000001CE050EA010200
:1055E00008BF70474FF000030AE000BF50EA010215
:1055F00008BF704711F0004302D5404261EB410102
:105600005FEA010C02BF84460146002043F0B64326
:1056100008BFA3F18053A3F50003BCFA8CF2083A4B
:10562000A3EBC25310DB01FA02FC634400FA02FC54
:10563000C2F12002BCF1004F20FA02F243EB02005B
:1056400008BF20F00100704702F1200201FA02FCBD
:10565000C2F1200250EA4C0021FA02F243EB0200B0
:1056600008BF20EADC707047002103E00A4B5B585A
:105670004350043109480A4B42189A42F6D3094A6A
:1056800002E0002342F8043B074B9A42F9D3FBF7B0
:1056900087FB00F00DF870478C59010800000020CE
:1056A000A4000020A400002000130020FEE700005A
:1056B0002F49CA6822F4E06208B512042D4B120C7F
:1056C0001343CB604FF080500121FDF7DFFC012137
:1056D0000846FDF7CFFC62B6F2F721FEF3F74AF970
:1056E000F2F7BAFDFAF7C8FAFBF796FAF3F797FB69
:1056F000F2F73AFF204B1A6999685879FBF7D8F806
:10570000F3F7DEFCFAF72DFFF9F78AFE1B4BDC6995
:105710009CB10120FAF714F8F7F7C0FFF8F768F822
:10572000174B4FF000629A61F7F79AFDF8F761F8AE
:10573000F8F7DCF9FAF79AF8F6E7124D2246204618
:105740006021F3F7FAFB224620466121F3F7F5FBCF
:10575000EA891C212046F3F7F0FB6868F9F7B4FFEB
:10576000A868F9F7C3FF287BF9F7D8FFD4E700BF93
:1057700000ED00E00007FA0504000020280C0020DE
:1057800000040048AC0C002010B5431E0A449142AE
:1057900000D110BD11F8014B03F8014FF7E761404C
:1057A00001AA80000020C08000002B2001AA8000F8
:1057B0000020C0800000000000000000E093040012
:1057C000C0270900FF00FE000000000032FF0000BB
:1057D000E80300001027000088130000D007000035
:1057E0000A0000000000000000C2EB0B00000100F6
:1057F000640000006400000000070000F4010000E5
:105800000000000000000000E0930400C027090031
:10581000FF00FE000000000064F00000E80300004C
:105820001027000010270000140000000A000000EC
:1058300000000000FFFFFF3F0000010064000000C7
:105840006400000000070000F401000000000000F8
:105850000050C30000881300014008080000000049
:1058600000000000C800000001000000000000006F
:10587000000000000000000000C8000000C8000098
:105880000000000000000000000000000001000116
:105890000000000000000000000000000000000008
:1058A00000000000000000000000000000000000F8
:1058B00000000000000000000000000000000000E8
:1058C00000000000000000000000000000000000D8
:1058D00000000000A7A6A5A2A3A4A8A9AAABACADEE
:1058E000AEB800000101000100000001000000014D
:1058F00000000000000100000000000000000000A7
:105900000000000101010000000000000000000094
:10591000010000000000000101010001010001017F
:105920000000000000000000000000000000000077
:105930000000000000000000000000000000000067
:105940000000000000000000000000000001010055
:105950000000010001010100000000000000000043
:10596000000000313337385631333800F8B500BF06
:10597000F8BC08BC9E467047F8B500BFF8BC08BC30
:045980009E46704788
:04598400AD810008E9
:045988008981000809
:10598C00635901080001020000080000010000003A
:10599C0002000000000000000000000000000000F9
:1059AC0000000000000000000000000000000000EB
:1059BC0000000000000000000000000000000000DB
:1059CC000000000002000000C0270900E093040062
:1059DC0001000000010000000A000000200300008C
:1059EC005100000000A24A0400000000000000006A
:1059FC000102030406070809000000000102030469
:105A0C00010203040607080900000100020004005B
:105A1C00060008000A000C00100020004000800066
:045A2C000001000075
:04000005080156692F
:00000001FF
